:020000040800F2
:10000000183600209D0100087D640008154C00088A
:1000100079640008B1140008799700080000000016
:1000200000000000000000000000000005010008C2
:10003000551B000800000000490100080F8B000854
:10004000B7010008B7010008B7010008B7010008B0
:10005000B7010008B7010008B7010008B7010008A0
:10006000B7010008B7010008B7010008B701000890
:10007000C91A0008D91A0008E91A0008F91A000874
:10008000091B0008191B0008B7010008B701000888
:10009000B7010008B7010008B7010008631B00089A
:1000A000B7010008B7010008B7010008B701000850
:1000B000B7010008B7010008B7010008B701000840
:1000C000B7010008B7010008B70100084D65000836
:1000D0005D6500086596000875960008B701000880
:1000E000571B0008B7010008B7010008DFF810D05F
:1000F00000F05CFE00480047B5A80008AFF30080A0
:1001000018360020224B19680868B0E8F00F80F319
:100110000988BFF36F8F4FF0000080F311884EF015
:100120000D0E70470000000006480068006880F36C
:10013000088862B661B6BFF34F8FBFF36F8F00DFE1
:1001400000BF00BF08ED00E0EFF30980BFF36F8F41
:100150000F4B1A6820E9F00F106008B54FF05000FF
:1001600080F31188BFF34F8FBFF36F8F0FF080F9CB
:100170004FF0000080F31188BDE808401968086856
:10018000B0E8F00F80F30988BFF36F8F704700BFAE
:1001900018000020EFF305807047000006488047F4
:1001A00006480047FEE7FEE7FEE7FEE7FEE7FEE75C
:1001B000FEE7FEE7FEE7FEE7898B0008ED0000089A
:1001C0002DE9F05F0546002092469B46884606468C
:1001D000814640241BE0284641464746224600F01F
:1001E00020F853465A46C01A914110D3114618467A
:1001F000224600F0A3FB2D1A67EB01084F4622466A
:100200000120002100F09AFB17EB00094E41201E4F
:10021000A4F10104DFDC484631462A464346BDE8E6
:10022000F09F202A04DB203A21FA02F000217047D7
:1002300021FA02F3D040C2F120029140084319464E
:10024000704740EA01039B0703D009E008C9121F69
:1002500008C0042AFAD203E011F8013B00F8013B80
:10026000521EF9D27047D2B201E000F8012B491EAC
:10027000FBD270470022F6E710B513460A46044643
:100280001946FFF7F0FF204610BD10B5044604E004
:100290000B7800F8013B03B1491C521EF8D22046EE
:1002A00010BD421C10F8011B0029FBD1801A7047B9
:1002B00030B505460020034600E05B1C934205D2A2
:1002C000EC5CC85C201A01D1002CF6D130BD2DE9C0
:1002D000F0410E460546002400E0641C285D00F055
:1002E0004AFB0746305D00F046FB381A02D1295D13
:1002F0000029F2D1BDE8F0810FB400B58DB010A98E
:1003000009900B9000914FF0FF300A9000200C9064
:1003100005480690054807906A4609A80F9900F01D
:1003200045FB0DB05DF814FBC9090008E70900089A
:100330002DE9FF5F1D464FF0FF3BD5E90146914691
:100340005F464FF00008A9697F1C01988847296A19
:10035000824688470028F6D1BAF1FF3F0CD024F43A
:10036000C064002E19DD600614D5BAF12B0F09D038
:10037000BAF12D0F0ED103E0584604B0BDE8F09F4E
:1003800044F48064A9697F1C01988847761E8246E0
:10039000002E02DDBAF1300F03D0B9F1000F26D0E4
:1003A00032E0A969761E44F400747F1C01988847E6
:1003B0008246002E05DDBAF1780F06D0BAF1580F4B
:1003C00003D0B9F1000F10D01EE0B9F1000F02D038
:1003D000B9F1100F18D1A969761E24F400747F1C9E
:1003E000019888478246102002E0082000E00A2099
:1003F000814609E008FB0908A969761E44F40074E7
:100400007F1C019888478246002E05DD49465046EC
:1004100000F0B7FA0028EDDAE96901988847A005ED
:1004200002D46FF00100A8E7E00725D1600613D5DC
:10043000600502D5C8F1000000E0404629680A1DA9
:100440002A600968220501D5087015E0220701D548
:10045000088011E008600FE02868011D296000682D
:10046000210502D580F8008006E0210702D5A0F81A
:10047000008001E0C0F8008038467EE72DE9F047B3
:1004800091460F4680460446002614F8015B2DB1C4
:1004900000F064FA0068405DC007F6D12B2D02D051
:1004A0002D2D18D0641E4A463946204600F0ACFA7D
:1004B00027B13968A14201D1C7F8008071054FF01A
:1004C00002040BD54042002803DD09F0A3FB0460C1
:1004D000A007BDE8F08746F48066E4E70028F8DA74
:1004E00009F098FB04606FF00040F2E72DE9F05F3F
:1004F00093460F4680460446002609F08BFBD0F851
:100500000090824614F8015B2DB100F027FA0068D4
:10051000405DC007F6D12B2D02D02D2D1AD0641EC0
:100520000021CAF800105A463946204600F06CFAFD
:10053000014627B13868A04201D1C7F80080DAF837
:100540000000022809D0CAF80090700505D548427D
:10055000BDE8F09F46F48066E2E70846F8E7F0B4AD
:1005600080EA0102D40F4200B2EB410F02D20246F0
:10057000084611464A0042D0C30DDDB2C1F3C7524E
:10058000AD1A202D35DAC1F3160141F4000204B191
:100590005242C5F1200602FA06F12A411044B3EB9B
:1005A000D05F23D0C4B1012DA0EBC35009DCF0BC57
:1005B0004FF0004202EAC352DBB200F5000000F047
:1005C0007BBA400000F1807000EBC350A0F1807056
:1005D00040EAD170490009E0490841EAC071A0EB46
:1005E000C35000F50000400800EBC350F0BC00F021
:1005F0005ABA6142012202EB4101001BF6E7F0BC4E
:10060000704781F00041AAE780F00040A7E730B4CE
:1006100080EA010202F0004530F0004221F0004083
:1006200013D090B1C30DD40DC2F31601C0F3160060
:10063000E41A41F4000140F400027D34914201D3F8
:10064000641C00E04900002C02DA30BC0020704736
:100650004FF400000023914201D3891A034340085C
:100660004FEA4101F7D151B1914202D14FF000411F
:1006700005E002D24FF0010101E06FF0010103EB50
:10068000C450284430BC00F00EBA2DE9FE4F81EA78
:10069000030404F0004421F0004100944FF0000BEB
:1006A00023F0004350EA01045ED052EA03045BD019
:1006B000C3F30A54C1F30A552C44A4F2F334019451
:1006C000A0FB0254C1F3130141F48011C3F31303DF
:1006D00043F4801301FB024400FB034E840A970A93
:1006E00044EA815447EA8357A4FB076802958D0AC0
:1006F00005FB07854FEA932C04FB0C542705029D4C
:100700004FEA065847EA1637B5EB08056EEB070CBB
:10071000870E920E47EA811742EA8312A7FB020175
:10072000B6EB0B0164EB00042B0D43EA0C335E18AF
:1007300044EB1C50DA465146E7FB0201C5F31304B3
:100740004FEA0B3343EA14534FEA0432019C43EA65
:100750000603A4F10C040294009CCDE900B400F05F
:10076000E8F903B0BDE8F08F00200146F9E72DE974
:10077000F04D81EA030404F0004B21F000451446DB
:100780004FF0000A23F0004150EA050220D054EA5D
:1007900001021DD0C5F30A570246C5F31303C1F386
:1007A0001300C1F30A5640F4801543F48013A7EBFD
:1007B0000608101BD64608F2FD3873EB050002D37D
:1007C00008F1010801E092185B41B8F1000F03DA6B
:1007D00000200146BDE8F08D00204FF48011064650
:1007E00084460EE0171B73EB050705D3121B63EB62
:1007F000050306434CEA010C49084FEA3000921801
:100800005B4150EA0107EDD152EA030012D082EABF
:10081000040083EA0501084305D0101BAB4106D252
:100820000122002306E000224FF0004302E06FF0B7
:10083000010253101AEB06004CEB085110EB0A00B2
:1008400041EB0B01BDE8F04D00F064B930B4044653
:1008500096230800214604D0B62330BC002200F0C5
:100860002BB920460021F8E70EB5C10F80EAE070F1
:100870000844CA07002140F233438DE80E000A46BF
:100880000B4600F056F903B000BD0EB540F23341FF
:1008900002910021CDE900110A460B4600F049F90A
:1008A00003B000BDC1F30A5210B5C1F3130140F209
:1008B000FF3341F480119A4201DA002010BD40F26A
:1008C00033439A42A2F2334203DC5242FFF7A9FCBF
:1008D00010BD904010BD00F0004230F000400AD042
:1008E000C10D01F56071C0F3160042EA0151C20862
:1008F000400711437047002001467047002801DB84
:10090000C0F10040002901DBC1F10041884270477D
:1009100030B50B46014600202022012409E021FACF
:1009200002F59D4205D303FA02F5491B04FA02F5CC
:100930002844151EA2F10102F1DC30BD202A04DB9F
:10094000203A00FA02F1002070479140C2F12003E2
:1009500020FA03F3194390407047000000487047A5
:10096000CC4D010810B50446FFF7F8FF0068005DA4
:1009700000F0010010BDA0F14101192900D820307C
:1009800070473A2800D2303820F02002412A01D3A3
:10099000A2F13700884201D34FF0FF3070470000CA
:1009A000026811441378016018467047D160044909
:1009B00051610449116200211161114600F01ABA17
:1009C000A109000865090008426842B1016811F8F0
:1009D000013B23B1521EC0E90012184670470121A5
:1009E000C160881E704742685AB1C368016843B944
:1009F00083688B4205D0491E521CC0E900120020BA
:100A000070474FF0FF3070472DE9F05F8246007865
:100A1000002715468B460AF10104B946302801D05B
:100A20009DB113E014F8010B0127782803D0582852
:100A300001D045B10AE00DB1102D07D100271025D6
:100A400014F8010B02E0082500E00A250026B04654
:100A50000EE005FB080005FB06F1012701EB10463F
:100A60001FFA80F8B6F5803F00D3B94614F8010BA1
:100A70002946FFF786FF0028EBDABBF1000F05D00F
:100A80000FB1641E00E05446CBF80040B9F1000FEE
:100A900006D009F0BFF802210160C81EBDE8F09F32
:100AA00048EA0640FAE70029A8BF7047401C490001
:100AB00008BF20F00100704710B4B0FA80FC00FAC3
:100AC0000CF050EA010404BF10BC704749B1CCF1EE
:100AD000200421FA04F411FA0CF118BF012121437A
:100AE0000843A3EB0C01CB1D4FEA00614FEA102035
:100AF00042BF002010BC704700EBC35010440029D7
:100B0000A4BF10BC7047401C490008BF20F0010082
:100B100010BC704710B5141E73F1000408DA401CB5
:100B200041F1000192185B411A4301D120F001000C
:100B300010BD2DE9F04D92469B4611B1B1FA81F2FC
:100B400002E0B0FA80F220329046FFF7F7FE04464A
:100B50000F4640EA0A0041EA0B0153465A46084351
:100B600013D0114653EA010019D0C8F14002504693
:100B7000FFF757FB05460E46504659464246FFF7DB
:100B8000DDFE084305D0012004E020463946BDE8DB
:100B9000F08D0020054346EAE0762C4337430A985F
:100BA0006305E40AA0EB08000022FD0A44EA47546A
:100BB0000A3002D500200146E9E701051019694114
:100BC000DDE9084500196941BDE8F04DA2E72DE9CE
:100BD000FE4F804681EA0300C00F0C46009021F0D2
:100BE000004123F00045B8EB0200A94105D2404680
:100BF000214690461C460B46024623F00040104317
:100C000047D0270DC7F30A00C3F30A510290401AD8
:100C1000019040286BDAC3F3130040F4801B009866
:100C2000924620B10023D2EB030A63EB0B0B019831
:100C30005946C0F140025046FFF780FE06460D4679
:100C400050465946019A00F0C3F810EB0800614184
:100C5000002487EA115284EAE7731A4340D0009ACD
:100C600062B3019A012A4FEA075215DC001B61EBBF
:100C700002014FF0004202EA0752CDE90042001C97
:100C800041F5801132462B46FFF753FF03B0BDE814
:100C9000F08F40462146F9E7001B61EB0201001C82
:100CA00041F5801300185B412018A2F5001747EBAF
:100CB000030140EAD570B6196D4111E06D084FEAA5
:100CC000360645EAC0754FEA0752001B61EB020188
:100CD000001C41F5801149084FEA300000195141CC
:100CE00032462B4603B0BDE8F04FFFF713BF009824
:100CF000012240000023D0EB020263EBE073009876
:100D000021464FEAE074B8EB000061EB0401E9E72B
:100D100083F000435BE781F0004158E770B521F0B4
:100D2000004303430CD0C1F30A550024D5EB04055E
:100D300064EB0403D617AD1AB34102DB0020014671
:100D400070BD201841EB025170BDC1F30A52C1F3CE
:100D5000130140F2FF3341F480119A4202DA00207D
:100D60000146704740F233439A42A2F2334202DC1A
:100D70005242FFF756BAFFF7E1BD000030B5041E3E
:100D800071F1000404DB4FF00044404264EB0101C8
:100D9000141E73F1000405DB1C464FF00043524261
:100DA00063EB0403994208BF904230BD064C074DE7
:100DB00006E0E06840F0010394E80700984710342B
:100DC000AC42F6D3FFF796F9F45501081456010822
:100DD000202A06DBCB17203A41FA02F043EAE073FF
:100DE00006E041FA02F3D040C2F1200291400843EC
:100DF000194670472DE9F34F8BB04FF0000801F111
:100E00000C000C464FF0010B46460DF1080A01900C
:100E10006269012101989047051E2DD0252D2CD007
:100E2000216A8847C0B16269012101989047216A0F
:100E300088470028F7D1411E62690198904700E079
:100E4000761CA1690B988847216A88470028F7D14A
:100E5000E1690B988847DBE7A1690B98884707464B
:100E6000A84201D1761CD3E7E1690B9888477F1C23
:100E700002D1B8F1000F6FD047E1002762693D460B
:100E80003946019890472A2804D1626901210198C6
:100E900090470125DFF88892626901210198904707
:100EA000A0F130010A290AD24F45E5DC07EB8701A2
:100EB00000EB4107303FDFD445F01005ECE7E906D1
:100EC00001D46FF000476C280AD04C2814D0682851
:100ED00015D06A280DD074281CD07A281AD01DE0AD
:100EE00062690121019890476C2802D045F0040501
:100EF00014E045F002050DE045F020050AE06269C6
:100F0000012101989047682802D045F0080505E0C6
:100F100045F400656269012101989047C4E90157D1
:100F200065283DD019DC58287AD00CDC452837D00C
:100F300004DC252826D0412831D131E046282FD0A5
:100F400047282CD12CE05B2877D0612828D0632853
:100F50007CD0642823D15AE0D1E06F2848D008DC47
:100F600066281DD067281BD0692821D06E2816D18D
:100F700027E0702845D0732868D0752847D0782896
:100F80000DD14DE0A1690B988847054625283FF40F
:100F900069AFE1690B9888476D1C3FF46AAFB4E014
:100FA00023466A466FF001000B99AFF300809FE083
:100FB00045F040006060A80723464FF0000236D499
:100FC0003EE0E8077FF447AF2068011D216000681C
:100FD000290501D506701BE7290701D5068017E70B
:100FE000A90703D5F117C0E9006111E706600FE713
:100FF00045F040006060A80723464FF0080216D471
:101000001EE040F60E0125EA0100606016E045F0A2
:1010100040006060A80723464FF00A0207D40FE0A3
:1010200045F040006060A80708D5234610226FF005
:1010300001000B99AFF300805AE007E0234610222D
:101040006FF001000B99FFF773F951E04FF00009C1
:101050004F464B46632802D05B2807D041E02079F9
:10106000C00601D40120A06001273AE06269012195
:10107000019890475E2805D14FF001096269494601
:1010800001989047216939B900210A46534643F82F
:101090002120491C0829FADBB0B3216969B9C117BD
:1010A00000EBD16253110AEB830122F01F02821A76
:1010B00001200B68904003430B6062690121019895
:1010C00090475D28E8D1B9F1000F09D000205146C2
:1010D00051F82020D24341F82020401C0828F7DB9B
:1010E00002AB224600976FF001000B99AFF300802E
:1010F00000280CDA401C08D1BBF1000F05D04FF0DE
:10110000FF300DB0BDE8F08FFFE74046F9E7E90793
:1011100001D108F1010806444FF0000B78E6000009
:10112000CCCCCC0C2DE9F04D00231A461B1A8A4179
:1011300003DB00200146BDE8F08DC1F30A52C1F384
:10114000130141F480154FF0000BD10702D10018B4
:101150006D41521E0027044640F2FF11384601EB54
:10116000620A3E468046024600204FF48011FFF797
:1011700058F8C2197141BB1846EB0100B4EB030CDF
:1011800075EB000C04D3E41A65EB000517460E4618
:10119000241908F101006D4180463428E3DDF91976
:1011A00046EB0600091BA84103D24FF0FF3213465D
:1011B00001E0002213461BEB070046EB0A51BDE895
:1011C000F04DFFF7A7BC70B58C1810F8015B15F057
:1011D000070301D110F8013B2A1106D110F8012BA9
:1011E00003E010F8016B01F8016B5B1EF9D12B07CE
:1011F00005D40023521E0DD401F8013BFAE710F884
:10120000013BCB1A921C03E013F8015B01F8015B70
:10121000521EF9D5A142D8D3002070BD70B5044646
:101220000D461646012C02DB4FF0FF3070BD064A1A
:1012300002EBC4029188044A52F8340033462A462D
:1012400002F0FEFE0020F1E7E402010810B50446BA
:10125000012C02DB4FF0FF3010BD054A02EBC40247
:101260009188034A52F8340002F0F4FF0020F3E7BB
:10127000E402010810B50446012C02DB4FF0FF30F8
:1012800010BD054A02EBC4029188034A52F83400AB
:1012900003F02EF80020F3E7E4020108014611B143
:1012A000012904D101E0034870470348FCE700200E
:1012B000FAE70000300100208801002070B50546E3
:1012C000022D01DBFF2070BD2846FFF7E7FF044633
:1012D0000CB9FF20F7E7204601F07EFEF3E700009F
:1012E000034612B96FF001007047034800EB43104A
:1012F00040F821200020F7E7A82300202DE9F04145
:1013000005460F4690461E46022D03DB4FF0FF3088
:10131000BDE8F0812846FFF7C1FF044614B94FF03D
:10132000FF30F5E74EB142463946204602F016FB43
:1013300008B10120ECE70020EAE7142342463946D1
:10134000204602F055F808B10120E1E70020DFE770
:101350002DE9F84305460E4617469846DDF82090DD
:10136000022D03DB4FF0FF30BDE8F8832846FFF77E
:1013700095FF044614B94FF0FF30F5E7B9F1000FBF
:101380000AD043463A463146204602F035FA08B1C3
:101390000120E9E70020E7E7142043463A463146BA
:1013A0000090204602F003F908B10120DCE700209C
:1013B000DAE72DE9F04109F031FF05460EF01AFD9C
:1013C0004FF47A71B1FBF5F100FB01F64FF0E0202C
:1013D00087690EF00FFD4FF47A71B1FBF5F100FB58
:1013E00001F44FF0E020D0F81880A64214D14FF459
:1013F0007A7078434FF0E0214969491CB0FBF1F065
:1014000004EB4401C1EBC4114FF47A7202EBC10149
:10141000081A0021BDE8F0814FF47A7008FB00F053
:101420004FF0E0214969491CB0FBF1F004EB4401A5
:10143000C1EBC4114FF47A7202EBC101081A00210A
:10144000E8E70000014611B1012904D101E0034899
:1014500070470348FCE70020FAE700008005002001
:10146000380500202DE9F04104460D4616461F467A
:10147000022C03DB4FF0FF30BDE8F08105B116B957
:101480006FF00100F8E74FB12046FFF7DBFF804621
:101490003246294603F02AFB40B2EDE72046FFF72B
:1014A000D1FF80463246294603F066FB40B2E3E7AF
:1014B00000BFFEE700487047702C002010B53822AE
:1014C0000649074805F012FA0448083000F0EAF827
:1014D00008B1012010BD0020FCE70000702C0020A6
:1014E00000F8000889B001216348A0F86410A0F852
:1014F00066100221A0F868100321A0F86A100021EC
:1015000080F860106E21A0F8621001205A4908721C
:101510005A4A00215848C0E914210D2180F858107A
:10152000002180F8591003214172022180F85A10DD
:1015300080F85B10002180F85C1080F85D104C2171
:1015400080F84710012180F84810202180F84910C8
:10155000042180F83B10202180F83910102180F8F8
:101560003A10002180F83C10C02180F8411034214D
:1015700080F84210072180F843100C2180F82D10CC
:10158000002180F82E107F2180F82F10202180F874
:101590003010402180F83110EF2180F83E100121F9
:1015A00080F83F10202180F84010702180F826102C
:1015B000082180F82710102180F82810202180F8B9
:1015C00029107F2180F82A10302180F82B1000216B
:1015D00080F82C10EB2180F84410002180F8451091
:1015E000102180F84610702180F83210042180F814
:1015F0003310102180F83410202180F835107F211D
:1016000080F83610302180F83710082180F8381023
:101610001BA103C9CDE907011BA103C9CDE9050140
:101620001BA103C9CDE9030113480799C0F80A10AB
:101630009DF8201081730599C0F80F109DF81810BF
:10164000C174039941619DF81010017612A00068E1
:10165000029012A00068019011A000680090064856
:101660000299C0F819100199C0F81D100099C0F82E
:10167000211009B070470000702C002080D2999092
:10168000123456789A00000023456789AB000000A9
:101690003456789ABC000000122334455667788986
:1016A0009AABBCCD10B504460CB9002010BDB4F8FF
:1016B0005C00002805DDB4F85C004FF6FF7188423D
:1016C00001DB0020F2E7FB4AD4E912309A1A70F1EC
:1016D000000006D3F8490020D4E91223891A984162
:1016E00001D20020E2E794F9500010F1120F03DB61
:1016F00094F950000D2801DD0020D7E794F8580038
:10170000022801DB0020D1E7B4F85A00012803DBEE
:10171000B4F85A007A2801DD0020C7E794F8510098
:1017200000F01F0181B9401108280DD2DFE800F058
:101730000405060708090A0B00BF00BF00BF00BF71
:1017400000BF00BF00BF01E00020AFE700BF94F87A
:101750005200042801DB0020A8E75320005D082880
:1017600001DB0020A2E75420005D052801DB0020FA
:101770009CE75520005D052801DB002096E794F8E2
:101780003500D0B101282DD0032844D0042857D1EA
:1017900094F83F0009F026F808B9002086E794F88D
:1017A00040000F2801DD002080E794F8410009F097
:1017B00074F808B9002079E744E03621085D09F0A3
:1017C00011F808B9002071E794F837000F2801DDFF
:1017D00000206BE794F8380009F05FF808B90020A2
:1017E00064E72FE094F8390009F03EF808B90020CA
:1017F0005CE794F83A0009F027F808B9002055E7AB
:1018000094F83B00012803DB94F83B00072801DD36
:1018100000204BE716E094F83C0008F0C4FF08B93C
:10182000002043E794F83D00042801DD00203DE757
:1018300094F83E0009F031F808B9002036E701E0DD
:10184000002033E700BF607F20B3012877D0032852
:1018500076D0042875D194F83300802801DD00206B
:1018600024E794F83100802801DD00201EE794F879
:101870003200102804D094F8320008B1002015E797
:1018800094F8340028B194F83400082801D00020DE
:101890000CE702E1A07F00F00F0181B900110828D8
:1018A0000DD2DFE800F00405060708090A0B00BFA7
:1018B00000BF00BF00BF00BF00BF00BF01E00020AD
:1018C000F4E600BFE07F09280BD2DFE800F0050A4C
:1018D000060A070A080A090000BF00BF00BF00BFD0
:1018E00001E00020E2E600BF94F8200000F00F01C4
:1018F00081B9001108280DD2DFE800F004050607C1
:1019000008090A0B00BF00BF00BF00BF00BF00BF37
:1019100000BF01E00020C9E600BF94F821002028A4
:1019200004D094F8210008B10020BFE694F822000A
:1019300018B194F82200FF2804DD0020B6E61CE070
:101940004AE0A8E094F8230030B1102805D0202800
:1019500004D0302804D102E000BF00BF00BF01E086
:101960000020A3E600BF94F8240028B194F82400D6
:10197000082801D0002099E68FE094F8250020B1D6
:1019800094F82500B0F5803F01DB00208EE694F846
:10199000260028B194F82600802801D0002085E692
:1019A00094F8270018B194F82700FF2801DD0020E3
:1019B0007CE694F82800202804D094F8280008B188
:1019C000002073E694F82900402804D094F82900F8
:1019D00008B100206AE660E094F82A0000F00F01E8
:1019E00081B9001108280DD2DFE800F004050607D0
:1019F00008090A0B00BF00BF00BF00BF00BF00BF47
:101A000000BF01E0002051E600BF94F82B0028B190
:101A100094F82B00042801D0002047E694F82C000D
:101A200000F00F0181B9001108280DD2DFE800F0A5
:101A30000405060708090A0B00BF00BF00BF00BF6E
:101A400000BF00BF00BF01E000202FE600BF94F8F8
:101A50002D00202804D094F82D0008B1002025E6A0
:101A600094F82E0018B194F82E00FF2801DD002014
:101A70001CE694F82F0030B1102805D0202804D09F
:101A8000302804D102E000BF00BF00BF01E0002009
:101A90000CE600BF01E0002008E600BF00210EE0D8
:101AA00004F15E0030F811004FF6FF72904205D14C
:101AB0000020FBE500180D8F00F90295491C032951
:101AC000EEDB0120F2E5000010B5024800F090FACC
:101AD00010BD0000E001002010B5024800F088FAB7
:101AE00010BD00002402002010B5024800F080FA6A
:101AF00010BD0000F402002010B5024800F078FA92
:101B000010BD00006802002010B5024800F070FA15
:101B100010BD0000C805002010B5024800F068FAAA
:101B200010BD00000C06002030B590F84050012494
:101B3000AC40C56B6C60046863604468102C04D1D1
:101B40000468A2600468E16003E00468A1600468BE
:101B5000E26030BD704710B54FF4805000F03EFC9D
:101B600010BD10B5202000F039FC402000F036FCFC
:101B7000802000F033FC10BD72B600BFFEE700000D
:101B80000022054BDA61054A126942F00102034B5B
:101B90001A610180704700005006002000200240BA
:101BA00000201E49C96801F0100139B11C49C969FA
:101BB00041F002011A4AD16140F010001749C9688A
:101BC00001F0040139B11649C96941F00101144A13
:101BD000D16140F004001149C96901F0010169B106
:101BE0000F49C96941F004010D4AD16100BF0B4999
:101BF000C96921F00101094AD16100BF00BF40F26B
:101C00000111884206D10549C96921F00101034A41
:101C1000D16101E00149C86000BF70470020024067
:101C20005006002070B5044600F084FD054609E02A
:101C3000601C38B124B100F07DFD401BA04201D9E9
:101C4000032070BD1248C06800F001000028EFD1E9
:101C50000F48C06800F0200020B100BF20200C49D0
:101C6000C86000BF0A48C06800F0100048B90848C2
:101C7000C06900F0010020B90548C06800F0040008
:101C800018B1FFF78DFF0120DBE70020D9E7000046
:101C9000002002400021074AD1610749096941F04B
:101CA0000201054A116111464861096941F040018C
:101CB00011617047481F00200020024030B50346E4
:101CC000002400200025156022E000E05B1C1D7848
:101CD00015B11D78202DF9D100E05B1C1D7815B1E0
:101CE0001D78202DF9D01D788DB1641C8C420FD148
:101CF000184603E015686D1C15605B1C1D7815B156
:101D00001D78202DF6D1156805B9002002E001E00C
:101D10008C42DAD300BF30BD2DE9F0470546884636
:101D2000914601262E48006898BB2E482C49086031
:101D30002AE02B480068006807683846FEF7B1FAC9
:101D40000446285D202801D0285DC0B922463946C6
:101D50002846FEF7ADFA90B921480068006890F96E
:101D60000C0000280ADB28460AF05AFA1C490968C8
:101D7000096891F90C10884200D0002608E0184844
:101D80000068406816490860154800680028D0D1EE
:101D900000BF1348006848B146B94A461249404658
:101DA000FEF773FA00200E49086016E00C48006840
:101DB00068B10B48006800682A4649468368404677
:101DC000984706464EB900200549086005E04A4696
:101DD00006494046FEF759FA00263046BDE8F0872E
:101DE00000010020F4000020DC4D0108344E010801
:101DF00070B50546002655B900BF502080F3118804
:101E0000BFF34F8FBFF36F8F00BF00BFFEE7082007
:101E10000AF0CEFD044654B900BF502080F311886B
:101E2000BFF34F8FBFF36F8F00BF00BFFEE764B1FA
:101E30000DF0B4F82560002060600548006844603B
:101E4000034804600DF0D4F80126304670BD000050
:101E5000FC0000200146002001F47F420AB140F05E
:101E600008004FF2F0020A400AB140F004004CF6BC
:101E7000CC420A400AB140F002004AF6AA220A40C7
:101E80000AB140F00100704770B504460D4629467E
:101E9000204600F041FC70BD2DE9F04781460D461B
:101EA00016461C462846FFF7D5FF074674B108487A
:101EB00040F82740284604F0C7F880460022314603
:101EC000404600F0C3FC404600F0B0FCBDE8F0879F
:101ED0003024002070B505460E461446E2B2314665
:101EE000284600F021FC70BD0146002291F8210037
:101EF000022808D00420886300BF002081F8200059
:101F000000BF012070470868006820F00E000B68D1
:101F100018600868006820F001000B68186091F8EC
:101F2000403001209840CB6B5860012081F821009F
:101F300000BF002081F8200000BF1046E2E700004B
:101F400070B50446002594F82100022803D004202F
:101F5000A063012548E02068006820F00E00216899
:101F600008602068006820F00100216808601F49AF
:101F70002068884201D1012026E01C4914312068E4
:101F8000884201D110201FE018492831206888427A
:101F900001D1801518E015493C312068884201D1F3
:101FA000801411E0114950312068884202D14FF469
:101FB000803009E00D4964312068884202D14FF435
:101FC000801001E04FF08070084908394860012016
:101FD00084F8210000BF002084F8200000BF606B5F
:101FE00010B12046616B8847284670BD080002404A
:101FF00070B50446E06B05682068066894F84010E8
:10200000042088402840002846D006F0040000281C
:1020100042D02068006800F0200028B920680068DD
:1020200020F004002168086057492068884201D1E7
:10203000042027E0544914312068884201D140200F
:1020400020E0514928312068884201D1001519E06B
:102050004D493C312068884202D14FF4804011E064
:10206000494950312068884202D14FF4802009E06C
:10207000454964312068884202D14FF4800001E074
:102080004FF08060404908394860E06A00287AD003
:102090002046E16A884776E094F8401002208840A4
:1020A0002840A0B306F0020088B32068006800F062
:1020B000200040B92068006820F00A00216808600C
:1020C000012084F8210030492068884201D1022093
:1020D00028E02D4914312068884201D1202021E0D8
:1020E000294928312068884201D140151AE0264943
:1020F0003C312068884202D14FF4005012E022495E
:1021000050312068884203D14FF400300AE017E0D4
:102110001D4964312068884202D14FF4001001E06B
:102120004FF0007018490839486000BF002084F85B
:10213000200000BFA06A30B32046A16A884722E091
:1021400094F84010082088402840E0B106F00800CC
:10215000C8B12068006820F00E002168086094F87B
:10216000401001208840E16B48600120A06384F8A2
:10217000210000BF002084F8200000BF206B10B1B8
:102180002046216B884770BD0800024001460022AE
:1021900009B901207047164B0868C01A1423B0FB18
:1021A000F3F08000086412480838C863022081F800
:1021B00021000868026843F6F0708243D1E9010308
:1021C0001843CB6818430B6918434B6918438B6954
:1021D0001843CB69184302430868026000208863F3
:1021E000012081F82100002081F8200000BFD1E704
:1021F000080002402DE9F04104460D4616461F46F0
:102200004FF0000800BF94F82000012802D10220FE
:10221000BDE8F081012084F8200000BF94F821007F
:1022200001282CD1022084F821000020A06320681E
:10223000006820F00100216808603B4632462946CC
:102240002046FFF771FCE06A30B12068006840F07A
:102250000E00216808600BE02068006820F0040090
:10226000216808602068006840F00A002168086062
:102270002068006840F001002168086006E000BFA7
:10228000002084F8200000BF4FF002084046BFE75E
:1022900070B5044600F04EFA06462546681C10B19B
:1022A00004480078054400BF00F044FA801BA842AF
:1022B000FAD370BD100000200348006940F0800090
:1022C0000149086100207047002002402DE9FE4FBF
:1022D00005468B46174698460126002400200290AA
:1022E00000BF2448007E012802D10220BDE8FE8FF5
:1022F00001202049087600BF4CF25030FFF792FCD5
:10230000064686BB012D02D10120029006E0022D77
:1023100002D10220029001E00420029000241EE07D
:102320002201B946C24648465146FDF77AFF80B2BF
:102330000190022000FB04B000900199FFF720FCFF
:102340004CF25030FFF76EFC06460B48006920F057
:1023500001000949086106B104E0601CC4B202989A
:102360008442DDDB00BF00BF00200249087600BFC9
:102370003046BBE7500600200020024000200849FC
:10238000096901F0800151B10649054A51600649C9
:1023900051601146096901F0800101B101207047C7
:1023A0000020024023016745AB89EFCD70B505469B
:1023B00000240DE00120A040284038B1064850F824
:1023C000240018B1044951F824008047601CC4B2AD
:1023D000102CEFDB70BD00006823002010B5044610
:1023E00004480068204020B1024804602046FFF7FE
:1023F000DDFF10BD140401402DE9F847034600221B
:1024000094466EE14FF0010808FA02F4D1F800801A
:1024100008EA0400A0427DD1DFF8DCA2D1F80480F4
:10242000A8EB0A09D0453AD014DCB8F1030F50D01C
:1024300009DCB8F1000F31D0B8F1010F1CD0B8F1B0
:10244000020F49D120E0B8F1110F18D0B8F1120FE6
:1024500042D11EE0B9F5881F25D006DCB9F5803FD2
:1024600020D0B9F5801F37D11AE0B9F5001F18D078
:10247000B9F5041F30D117E0D1F80CC02DE0D1F828
:102480000C8008F1040C28E0D1F80C8008F1080C4D
:1024900023E0D1F80C8008F10C0C1EE000BF00BF57
:1024A00000BF00BF00BF00BFD1F80880B8F1000F27
:1024B00002D14FF0040C0BE0D1F80880B8F1010F05
:1024C00003D14FF0080C1C6102E04FF0080C5C6176
:1024D00003E04FF0000C00E000BF00BFFF2801D870
:1024E000984601E003F104084646FF2802D84FEA67
:1024F000820803E0A2F108084FEA88084746D6F8A8
:1025000000804FF00F0909FA07F928EA09080CFAC8
:1025100007F900E088E048EA0908C6F80080D1F829
:10252000048008F08058B8F1805F7DD100BFDFF8EB
:10253000CC81D8F8188048F00108DFF8C091C9F8BC
:102540001880C846D8F8188008F00108CDF8008037
:1025500000BF00BF4FEAB9384FEA920958F8295036
:102560004FEA82784FEA18794FF00F0808FA09F815
:1025700025EA0805DFF88881434502D14FF00008BD
:1025800016E0DFF88081434502D14FF001080FE0EB
:10259000DFF87481434502D14FF0020808E0DFF80C
:1025A0006C81434502D14FF0030801E04FF004086D
:1025B0004FEA82794FEA197908FA09F848EA0505DD
:1025C000DFF84C814FEA920948F82950D1F804808D
:1025D00008F48018B8F5801F0AD1DFF83881D8F8E0
:1025E000008048EA0008DFF82C91C9F8008009E073
:1025F000DFF82081D8F8008028EA0008DFF814917D
:10260000C9F80080D1F8048008F40018B8F5001F5C
:1026100010D1DFF8008108F10408D8F8008048EAFA
:102620000008DFF8F09000E05AE009F10409C9F869
:1026300000800DE0DFF8DC8008F10408D8F80080A5
:1026400028EA0008DFF8CC9009F10409C9F80080F5
:10265000D1F8048008F40038B8F5003F0ED1DFF857
:10266000B480A8F10408D8F8008048EA0008DFF830
:10267000A490A9F10409C9F800800DE0DFF8948066
:10268000A8F10408D8F8008028EA0008DFF8849050
:10269000A9F10409C9F80080D1F8048008F4803851
:1026A000B8F5803F0ED1DFF86C80A8F10808D8F8A3
:1026B000008048EA0008DFF85C90A9F10809C9F831
:1026C00000800DE0DFF84C80A8F10808D8F8008001
:1026D00028EA0008DFF83C90A9F10809C9F8008051
:1026E000521CD1F8008028FA02F8B8F1000F7FF4EC
:1026F00089AEBDE8F887000000001110001002400C
:1027000000080140000C014000100140001401408D
:102710000800014008040140024693680B400BB1D9
:10272000012000E0002070470AB1016101E00B04C4
:1027300003617047014800687047000008000020EE
:102740000348006803490978084401490860704754
:10275000080000201000002010B50848006840F074
:10276000100006490860032000F0AEF80F2000F0CA
:1027700007F800F02BF8002010BD000000200240F8
:1027800070B504460E4800784FF47A71B1FBF0F052
:102790000C490968B1FBF0F5284601F0C7F908B10A
:1027A000012070BD102C07D200222146501E00F0DF
:1027B0004DF80548046001E00120F2E70020F0E751
:1027C00010000020140000200C00002008B500BFFD
:1027D0001448806940F00100124988610846806908
:1027E00000F00100009000BF00BF00BF0846C069B4
:1027F00040F08050C8610846C06900F080500090E9
:1028000000BF00BF00220F21901E00F01FF800BF84
:102810000549486820F0E06040F00070486000BF63
:1028200008BD0000001002400000014001460846BB
:10283000002809DB00F01F0301229A4043099B0096
:1028400003F1E023C3F8002100BF70472DE9F05FDA
:1028500080460D461646002707F0C0F90746394660
:102860002A46334601F00700C0F1070ABAF1040F07
:1028700002D94FF0040A01E0C0F1070AD14600F185
:10288000040ABAF1070F02D24FF0000A01E0A0F1EA
:10289000030AD4464FF0010A0AFA09FAAAF1010A1A
:1028A0000AEA020A0AFA0CFA4FF0010B0BFA0CFBC7
:1028B000ABF1010B0BEA030B4AEA0B04214640463D
:1028C00007F094F9BDE8F09F00BF00F00702064B47
:1028D00019684FF6FF031940044B0B4343EA0221EA
:1028E000014B196000BF70470CED00E00000FA05D5
:1028F00070B504460D460CB9012070BD5A480068F9
:1029000000F00700A8420ED25748006820F00700E8
:102910002843554908600846006800F00700A842AF
:1029200001D00120E9E7207800F0020002281DD143
:10293000207800F00400042805D14C48406840F499
:10294000E0604A494860207800F00800082805D176
:102950004648406840F460504449486043484068F5
:1029600020F0F000A168084340494860207800F05A
:10297000010078B36068012806D13C48006800F483
:10298000003090B90120B8E76068022806D13748C6
:10299000006800F0007040B90120AEE733480068DD
:1029A00000F0020008B90120A7E73048406820F095
:1029B0000300616808432D494860FFF7BBFE0646E7
:1029C00009E0FFF7B7FE801B41F28831884202D947
:1029D000032092E707E02548406800F00C0061689A
:1029E000B0EB810FEDD12048006800F00700A8424D
:1029F0000ED91D48006820F0070028431A490860D6
:102A00000846006800F00700A84201D0012074E7E2
:102A1000207800F00400042807D11448406820F40E
:102A2000E060E168084311494860207800F0080040
:102A3000082808D10D48406820F46050216940EA18
:102A4000C1000A49486000F03FF808494968C1F3ED
:102A50000311074A515CC8400649086006480068EF
:102A6000FFF78EFE002048E70020024000100240E1
:102A7000CA020108140000200C0000200148006870
:102A8000704700001400002000B5FFF7F7FF04496D
:102A90004968C1F30221034A515CC84000BD0000EF
:102AA00000100240DA02010800B5FFF7E7FF044911
:102AB0004968C1F3C221034A515CC84000BD00000F
:102AC00000100240DA02010870B500210022002443
:102AD00000230020134D696801F00C05F5B1042DA9
:102AE00002D0082D19D101E00F4819E00F4DC1F3B4
:102AF0008346AB5D01F4803555B10A4D6D68C5F371
:102B000040450B4E725D084D5D43B5FBF2F402E0AB
:102B1000084D03FB05F4204602E000BF064800BF55
:102B200000BF70BD001002400024F400B80201088C
:102B3000C802010800093D0000127A00F8B50446F9
:102B40000CB90120F8BD207800F00100002878D0F1
:102B5000F848406800F00C0004280CD0F5484068A4
:102B600000F00C00082811D1F248406800F48030D1
:102B7000B0F5803F0AD1EF48006800F4003000282B
:102B80005FD0606800285CD10120DBE700BF60688F
:102B9000B0F5803F06D1E748006840F48030E54951
:102BA000086028E0606858B9E248006820F4803086
:102BB000E04908600846006820F4802008601AE0B8
:102BC0006068B0F5A02F0BD1DA48006840F480208F
:102BD000D84908600846006840F4803008600AE080
:102BE000D448006820F48030D24908600846006864
:102BF00020F48020086000BF606888B1FFF79AFD6C
:102C0000054606E0FFF796FD401B642801D9032026
:102C100098E7C848006800F400300028F2D010E0BF
:102C2000FFF788FD054606E0FFF784FD401B64289A
:102C300001D9032086E7BF48006800F4003000286F
:102C4000F2D1207800F00200022857D1B94840683C
:102C500000F00C0050B1B748406800F00C000828A4
:102C600018D1B448406800F4803098B9B148006881
:102C700000F0020020B12069012801D0012061E7A5
:102C8000AC48006820F0F800616940EAC100A94939
:102C9000086033E02069E8B10120A7490860FFF728
:102CA00049FD054606E0FFF745FD401B022801D916
:102CB000032047E79F48006800F002000028F2D098
:102CC0009C48006820F0F800616940EAC100994919
:102CD000086013E0002098490860FFF72BFD0546C7
:102CE00006E0FFF727FD401B022801D9032029E752
:102CF0009048006800F002000028F2D1207800F02F
:102D0000080008282DD1A069B8B101208B490860BE
:102D1000FFF710FD054606E0FFF70CFD401B0228FB
:102D200001D903200EE78348406A00F00200002822
:102D3000F2D0012003F0F6FB13E000207F49086089
:102D4000FFF7F8FC054606E0FFF7F4FC401B0228FD
:102D500001D90320F6E67748406A00F00200002817
:102D6000F2D1207800F00400042873D100277148C4
:102D7000C06900F0805070B900BF6E48C06940F073
:102D800080506C49C8610846C06900F080500090CE
:102D900000BF00BF01276A48006800F48070B0B926
:102DA0006748006840F4807065490860FFF7C2FC1E
:102DB000054606E0FFF7BEFC401B642801D903204E
:102DC000C0E65F48006800F480700028F2D000BFC1
:102DD000E068012806D15748006A40F001005549D3
:102DE000086227E0E06858B95248006A20F0010004
:102DF000504908620846006A20F00400086219E0A1
:102E0000E06805280BD14B48006A40F004004949AE
:102E100008620846006A40F0010008620AE045487E
:102E2000006A20F00100434908620846006A20F069
:102E30000400086200BFE068A0B1FFF77BFC054614
:102E400009E0FFF777FC401B41F28831884202D944
:102E5000032077E622E03748006A00F002000028ED
:102E6000EFD012E0FFF766FC054608E0FFF762FCD2
:102E7000401B41F28831884201D9032062E62D4887
:102E8000006A00F002000028F0D1012F05D1294886
:102E9000C06920F080502749C86100BFE069C8B30D
:102EA0002448406800F00C00082860D0E06902283F
:102EB00048D1002020490866FFF73CFC054606E0A3
:102EC000FFF738FC401B022801D903203AE61948D5
:102ED000006800F000700028F2D1206AB0F5803F51
:102EE00007D11448406820F40030A1680843114914
:102EF0004860D4E9080108430E49496821F4741177
:102F000008430C49486001200B490866FFF712FC92
:102F1000054607E03DE0FFF70DFC401B022801D904
:102F200003200FE60348006800F000700028F2D08C
:102F30002FE00000001002400000424280044242A4
:102F400000700040002014490866FFF7F3FB0546B7
:102F500006E0FFF7EFFB401B022801D90320F1E553
:102F60000E48006800F000700028F2D111E0E0691E
:102F7000012800D1E6E50948466806F48031206A58
:102F8000814204D106F47011606A814201D00120AF
:102F9000D8E50020D6E500000000424200100240C3
:102FA00070B50446204603F021FC0546032D0FD0E2
:102FB000204603F01BFC074901EB4010806938B143
:102FC000204603F013FC034901EB40108669B0472B
:102FD00070BD0000A8230020014691F85100704701
:102FE000F8B504462068466820688568C5F38010F7
:102FF00048B905F0010030B1C6F3801018B1204681
:10300000216C8847F8BDC5F3400030B1C6F3C0104D
:1030100018B12046616C8847F4E7C5F3401018B931
:10302000C5F38010002871D0C6F3401000286DD081
:10303000C5F38010F0B194F8510003280ED0606DF4
:1030400040F00400606500BF002000902068C06868
:10305000009020688068009000BF0BE000BF002057
:1030600000902068C068009020688068009000BFD1
:1030700000BFC7E7C5F3401088B1606D40F00100A4
:10308000606500BF00200090206880680090206884
:10309000006820F040002168086000BF00BF606D3C
:1030A00070B32068406820F0E0002168486001208B
:1030B00084F8510006F0020010B906F0010000B3D8
:1030C0002068406820F0030021684860E06C50B13F
:1030D0000F48E16C4863E06CFEF732FF18B1606D99
:1030E00040F040006065A06C50B10948A16C486395
:1030F000A06CFEF725FF18B1606D40F040006065E0
:1031000002E02046FFF74CFF7CE7FFE700BF79E7CE
:103110006D65000810B504460CB9012010BD606A49
:1031200038B96068B0F5827F00D105E00021E16127
:1031300002E00021216161610021A16294F8510047
:1031400028B9002084F85000204600F043F80220FF
:1031500084F851002068006820F040002168086071
:10316000A08800F48270218901F404410843A189F8
:1031700001F400610843217C01F002010843217D34
:1031800001F001010843218B01F400710843217F04
:1031900001F0380108432021095D01F08001084356
:1031A000218D01F400510843216808600421A069C1
:1031B00001EA1040216848602068C06920F400607E
:1031C0002168C86100206065012084F8510000205A
:1031D000A4E7000010B586B00446002002900390DA
:1031E000049005905D492068884269D100BF5C4821
:1031F000806940F480505A4988610846806900F42B
:103200008050019000BF00BF00BF0846806940F0B9
:10321000040088610846806900F00400019000BF46
:1032200000BFA0200290022003900320059002A975
:103230004C48FFF7E1F840200290002003900490F2
:1032400002A94848FFF7D8F84748484908600020D5
:1032500048600021454881608021C16000210161F2
:1032600041618161C161FEF791FF08B1FEF784FC05
:1032700000BF3E48E064446200BF3B4814303C4914
:103280000860102048600021394881608021C160B9
:103290000021016141618161C161FEF777FF08B1E1
:1032A000FEF76AFC00BF3248A064446200BF0022FF
:1032B00005212320FFF7CAFA2320FFF7B7FA4BE0D6
:1032C0002C492068884247D100BF2548C06940F496
:1032D00080402349C8610846C06900F480400190DD
:1032E00000BF00BF00BF0846806940F00800886149
:1032F0000846806900F00800019000BF00BF4FF44D
:1033000020400290022003900320059002A91A4851
:10331000FFF772F814483C301849086010204860E4
:103320000021164881608021C16000210161416156
:103330008161C161FEF72AFF08B1FEF71DFC00BFE5
:103340000E48A064446200BF002205212420FFF73C
:103350007DFA2420FFF76AFA06B010BD0030014064
:1033600000100240000801401C000240E001002063
:103370002402002000380040000C014068020020B8
:1033800070B50446204603F031FA0546032D0FD0F0
:10339000204603F02BFA074901EB4010406838B192
:1033A000204603F023FA034901EB40104668B0477A
:1033B00070BD0000A823002070B50446204603F02D
:1033C00015FA0546032D0FD0204603F00FFA0749E2
:1033D00001EB4010006938B1204603F007FA0349B9
:1033E00001EB40100669B04770BD0000A823002023
:1033F0002DE9F84304460F4616461D46FFF79AF995
:103400008046B14694F85100012802D00220BDE860
:10341000F88307B10EB90120F9E700BF94F8500016
:10342000012801D10220F2E7012084F8500000BFFA
:10343000032084F85100002060652763A686E68695
:10344000A063A087E08760642064A068B0F5004FA7
:103450000BD12068006820F04000216808602068D7
:10346000006840F48040216808602068006800F02F
:103470004000402805D02068006840F040002168E6
:103480000860E068B0F5006F37D1606810B1B9F13D
:10349000010F09D1206B00882168C860206B801C57
:1034A0002063E08E401EE08623E02068806800F004
:1034B000020002280AD1206B00882168C860206BB6
:1034C000801C2063E08E401EE08612E0FFF732F998
:1034D000A0EB0800A84201D3681C00B94DB9012037
:1034E00084F8510000BF002084F8500000BF032082
:1034F0008DE7E08E0028D8D136E0606810B1B9F1D0
:10350000010F09D1206B007821680873206B401CE3
:103510002063E08E401EE08623E02068806800F093
:10352000020002280AD1206B007821680873206B02
:10353000401C2063E08E401EE08612E0FFF7FAF8A0
:10354000A0EB0800A84201D3681C00B94DB90120C6
:1035500084F8510000BF002084F8500000BF032011
:1035600055E7E08E0028D8D142462946204603F090
:103570001BF908B120206065A06850B900BF002089
:1035800000902068C068009020688068009000BFAC
:1035900000BF012084F8510000BF002084F85000D3
:1035A00000BF606D08B1012031E700202FE72DE951
:1035B000FE4F04460F4690461D460C9E012001908A
:1035C000FFF7B8F8814694F851B060680290AA46B7
:1035D000BBF1010F0BD00298B0F5827F04D1A06837
:1035E00010B9BBF1040F02D00220BDE8FE8F1FB15D
:1035F000B8F1000F00D00DB90120F6E700BF94F834
:103600005000012801D10220EFE7012084F850008A
:1036100000BF94F85100042802D0052084F851001E
:1036200000206065C4F83880E587A5872763E586B4
:10363000A586206460642068006800F0400040288F
:1036400005D02068006840F0400021680860E0680C
:10365000B0F5006F52D1606810B1BAF1010F09D115
:10366000206B00882168C860206B801C2063E08E7E
:10367000401EE0863BE02068806800F002000228DF
:1036800010D1E08E70B1019801280BD1206B008819
:103690002168C860206B801C2063E08E401EE0869D
:1036A000002001902068806800F0010068B1E08F80
:1036B00058B12068C068A16B0880A06B801CA06313
:1036C000E08F401EE08701200190FFF733F8A0EB68
:1036D0000900B0420BD3701C48B1012084F851009E
:1036E00000BF002084F8500000BF03207DE7E08E7B
:1036F0000028C0D1E08F0028BDD152E0606810B131
:10370000BAF1010F09D1206B007821680873206B92
:10371000401C2063E08E401EE0863CE0206880680C
:1037200000F00200022810D1E08E70B1019801284B
:103730000BD1206B007821680873206B401C20633C
:10374000E08E401EE086002001902068806800F036
:10375000010068B1E08F58B12068C068A16B0870A3
:10376000A06B401CA063E08F401EE0870120019009
:10377000FEF7E0FFA0EB0900B04201D3701C00B9D6
:103780004EB9012084F8510000BF002084F8500099
:1037900000BF032029E7E08E0028BFD1E08F00287A
:1037A000BCD14A463146204602F0FEFF40B12020FF
:1037B000606500BF002084F8500000BF012014E7BE
:1037C000A06850B900BF002000902068C068009039
:1037D00020688068009000BF00BF012084F851007D
:1037E00000BF002084F8500000BF606D08B10120C8
:1037F000FBE60020F9E600002DE9F04704460E46FE
:1038000017461D4694F85180D4F80490B8F1010F82
:103810000AD0B9F5827F04D1A06810B9B8F1040FBD
:1038200002D00220BDE8F0870EB107B10DB901202A
:10383000F8E700BF94F85000012801D10220F1E719
:10384000012084F8500000BF94F85100042802D0F1
:10385000052084F85100002060652663A586E58672
:10386000A763A587E5872064606494F85100042865
:1038700006D13548E16CC8623448E16C886205E0E5
:103880003348E16CC8623348E16C88623248E16CCD
:1038900008630020E16C4863E38FD4F800C00CF1AA
:1038A0000C01A26BE06CFEF7A5FC50B1606D40F01E
:1038B0001000606500BF002084F8500000BF0120A8
:1038C000B0E72068406840F00100216848600020AF
:1038D000A16CC862A16C8862A16C0863A16C48638A
:1038E000E38ED4F800C00CF10C02216BA06CFEF743
:1038F00081FC50B1606D40F01000606500BF002099
:1039000084F8500000BF01208CE72068006800F0B8
:103910004000402805D02068006840F04000216841
:10392000086000BF002084F8500000BF2068406895
:1039300040F02000216848602068406840F00200A4
:103940002168486000206DE7A9650008D36500087C
:10395000C5650008CB660008816500082DE9F041C7
:1039600004460E46154694F85100012802D0022064
:10397000BDE8F08106B10DB90120F9E700BF94F868
:103980005000012801D10220F2E7012084F8500004
:1039900000BF032084F85100002060652663A586DF
:1039A000E586A06360642064A087E087A068B0F526
:1039B000004F0BD12068006820F0400021680860AB
:1039C0002068006840F48040216808601F48A16CAE
:1039D000C8621F48A16C88621E48A16C0863002061
:1039E000A16C4863E38E276807F10C02216BA06C81
:1039F000FEF700FC50B1606D40F01000606500BF44
:103A0000002084F8500000BF0120B1E72068006862
:103A100000F04000402805D02068006840F04000D9
:103A20002168086000BF002084F8500000BF2068B3
:103A3000406840F02000216848602068406840F0FD
:103A4000020021684860002092E70000B765000886
:103A50004D6600088165000870B50546284602F0ED
:103A6000C5FE0446032C09D0054800EB441000684D
:103A700020B1034901EB44110868804770BD000084
:103A8000A823002070B50446204602F0AFFE05468C
:103A9000032D0FD0204602F0A9FE074901EB40108C
:103AA000C06838B1204602F0A1FE034901EB401086
:103AB000C668B04770BD0000A823002070B504465A
:103AC000204602F093FE0546032D0FD0204602F05B
:103AD0008DFE074901EB4010806838B1204602F0A6
:103AE00085FE034901EB40108668B04770BD0000B9
:103AF000A823002070B50446204602F077FE054654
:103B0000032D0FD0204602F071FE074901EB401053
:103B1000406938B1204602F069FE034901EB4010CC
:103B20004669B04770BD0000A823002070B5044668
:103B30002546681EB0F1807F01D301200FE0681E8A
:103B40004FF0E02148610F214FF0FF3006F04EF8B2
:103B500000204FF0E021886107200861002070BD3F
:103B600010B50346002200BF93F83C00012801D1A4
:103B7000022010BD012083F83C0000BF22F0FF00AE
:103B8000CC6840EA040222F440708C6840EA0402E7
:103B900022F480604C6840EA040222F400600C6861
:103BA00040EA040222F480500C6940EA040222F444
:103BB00000504C6940EA040222F48040CC6940EA9B
:103BC00004021868426400BF002083F83C0000BF74
:103BD00000BFCEE730B502460B4600BF92F83C006E
:103BE000012801D1022030BD012082F83C0000BF35
:103BF000022082F83D00106844681068816824F053
:103C000070041868044310684460104D1068A8429E
:103C10000BD01068B0F1804F07D00D4D1068A8424E
:103C200003D00C4D1068A84205D121F080015868DE
:103C3000014310688160012082F83D0000BF002030
:103C400082F83C0000BF00BFCDE70000002C01401F
:103C5000000400400008004010B504460CB90120E3
:103C600010BD94F83D0028B9002084F83C0020469F
:103C700000F026F8022084F83D00211D206804F0A1
:103C800085FF012084F8460000BF84F83E00012132
:103C90003F200155402001554120015500BF00BF84
:103CA000012084F84200432001554420015545205D
:103CB000015500BF012084F83D000020D0E700003E
:103CC00038B504461B492068884231D100BF1A48E4
:103CD000806940F40060184988610846806900F4F2
:103CE0000060009000BF00BF144815490860102014
:103CF00048600021124881608021C1608900016113
:103D00008900416100218161C161FEF73FFA08B17C
:103D1000FDF732FF00BF0A4921630846446200BF35
:103D200000BFA163446200BF00BF6163446200BF83
:103D300038BD0000002C0140001002404400024049
:103D4000F40200202DE9F04104460D46002700BF93
:103D500094F83C00012802D10220BDE8F081012046
:103D600084F83C0000BF022084F83D00206886688B
:103D700026F0770626F47F4620688660286850285B
:103D800033D00CDC202850D004DC00284BD0102885
:103D900051D149E0302849D040284CD139E0602841
:103DA0002DD0702807D0B0F5805F03D0B0F5005F4C
:103DB00041D10DE041E0D5E902136A68206804F0C2
:103DC000BBFF2068866846F077062068866034E08E
:103DD000D5E902136A68206804F0AEFF20688068A5
:103DE00040F480402168886027E0EA6869682068BC
:103DF00005F072F85021206804F0A9FF1DE0EA6880
:103E00006968206805F07BF86021206804F09FFF56
:103E100013E0EA686968206805F05EF840212068D0
:103E200004F095FF09E000BF00BF00BF29682068CB
:103E300004F08DFF01E0012700BF00BF012084F8DE
:103E40003D0000BF002084F83C0000BF384684E7F6
:103E50007047000010B586B0044600200290039021
:103E6000049005900E492068884216D100BF0D4885
:103E7000806940F004000B4988610846806900F0C1
:103E80000400019000BF00BFC814029002200390FC
:103E9000059002A90448FEF7AFFA06B010BD000075
:103EA000002C014000100240000801402DE9F041C3
:103EB00004460D461646002700BF94F83C00012832
:103EC00002D10220BDE8F081012084F83C0000BF4F
:103ED00036B1042E1BD0082E31D00C2E5ED145E019
:103EE0002946206804F03CFF2068806940F0080003
:103EF000216888612068806920F004002168886159
:103F000020688069296908432168886148E029465A
:103F1000206804F055FF2068806940F40060216843
:103F200088612068806920F4806021688861206849
:103F30008069296940EA01202168886130E02946CA
:103F4000206804F071FF2068C06940F00800216813
:103F5000C8612068C06920F004002168C861206839
:103F6000C069296908432168C86119E029462068A9
:103F700004F08EFF2068C06940F400602168C861C9
:103F80002068C06920F480602168C8612068C06929
:103F9000296940EA01202168C86101E0012700BFCA
:103FA00000BF00BF002084F83C0000BF384689E70E
:103FB00010B504460CB9012010BD94F83D0028B995
:103FC000002084F83C00204600F025F8022084F808
:103FD0003D00211D206804F0D9FD012084F8460031
:103FE00000BF84F83E0001213F20015540200155CB
:103FF0004120015500BF00BF012084F8420043204A
:104000000155442001554520015500BF012084F889
:104010003D000020D0E7704710B5044605492068F0
:10402000884206D10020044908700C21204600F087
:104030005FF910BD002C0140DF0000207047000038
:104040002DE9F04704460D4616461F464FF000087E
:1040500015B994F83E000BE0042D02D13F20005D1D
:1040600006E0082D02D14020005D01E04120005D06
:10407000022801D1BDE8F08715B994F83E000BE0A5
:10408000042D02D13F20005D06E0082D02D1402022
:10409000005D01E04120005D012818D106B10FB993
:1040A0000120E7E71DB9022084F83E0011E0042D4D
:1040B00003D102213F2001550BE0082D03D102213D
:1040C0004020015505E002214120015501E0012079
:1040D000D0E735B1042D1FD0082D38D00C2D6CD170
:1040E00050E05649606A81625549606AC16255492B
:1040F000606A0163216801F134023B463146606A1F
:10410000FEF778F808B10120B4E72068C06840F4F1
:1041100000702168C86053E04849A06A816248493C
:10412000A06AC1624749A06A0163216801F13802AF
:104130003B463146A06AFEF75DF808B1012099E7D9
:104140002068C06840F480602168C86038E03B495E
:10415000E06A81623A49E06AC1623A49E06A016311
:10416000216801F13C023B463146E06AFEF742F825
:1041700008B101207EE72068C06840F40060216833
:10418000C8601DE02D49206B81622D49206BC16202
:104190002C49206B0163216801F140023B46314606
:1041A000206BFEF727F808B1012063E72068C0689C
:1041B00040F480502168C86002E04FF0010800BF61
:1041C00000BFB8F1000F36D101222946206804F063
:1041D0001FFD1D492068884201D1012000E0002018
:1041E00028B12068406C40F40040216848641649BA
:1041F000206888420BD02068B0F1804F07D0134967
:104200002068884203D01249206888420DD1206876
:10421000806800F00709B9F1060F0CD0206800682B
:1042200040F001002168086005E02068006840F067
:1042300001002168086040461CE70000338C00083C
:104240009B8C0008DB8C0008002C0140000400401F
:104250000008004030B504460D460022294620687B
:1042600004F0D6FC21492068884201D1012000E0F9
:10427000002090B100BF2068006A41F2111108408F
:1042800050B92068006A8910084028B92068406C3D
:1042900020F400402168486400BF00BF2068006A25
:1042A00041F21111084050B92068006A8910084095
:1042B00028B92068006820F001002168086000BF6C
:1042C0001DB9012084F83E000EE0042D03D1012128
:1042D0003F20015508E0082D03D101214020015560
:1042E00002E0012141200155002030BD002C014099
:1042F00070B504460D46002635B1042D0ED0082DAC
:1043000016D00C2D28D11DE02068C06820F4007064
:104310002168C860606AFDF713FE1FE02068C0686E
:1043200020F480602168C860A06AFDF709FE15E0EE
:104330002068C06820F400602168C860E06AFDF76A
:10434000FFFD0BE02068C06820F480502168C86041
:10435000206BFDF7F5FD01E0012600BF00BF002E38
:1043600046D100222946206804F052FC21492068E9
:10437000884201D1012000E0002090B100BF2068F8
:10438000006A41F21111084050B92068006A891092
:10439000084028B92068406C20F400402168486437
:1043A00000BF00BF2068006A41F21111084050B9F7
:1043B0002068006A8910084028B92068006820F049
:1043C00001002168086000BF1DB9012084F83E008B
:1043D0000EE0042D03D101213F20015508E0082DF6
:1043E00003D101214020015502E001214120015566
:1043F000304670BD002C0140704770B50446002562
:1044000020684069C0F3C01594F84100212817D1F5
:10441000B5B100BF00BF2168143151E8001F21F081
:1044200080002168143141E80002002AF3D100BF66
:10443000A06B10B1A06BFDF757FD204604F015FFEF
:1044400020684069C0F3801594F84200222817D1F3
:10445000B5B100BF00BF2168143151E8001F21F041
:1044600040002168143141E80002002AF3D100BF66
:10447000E06B10B1E06BFDF737FD204604F0AFFEB6
:10448000002070BD70B50546284604F001FF0446C3
:10449000032C0DD004EBC400064901EB8000006939
:1044A00030B104EBC401034A02EB81010869804783
:1044B00070BD0000E82300202DE9F84F0446206875
:1044C00005682068C668206847694FF00009CA4639
:1044D00005F00F09B9F1000F0AD105F0200038B13D
:1044E00006F0200020B1204604F0E6FEBDE8F88F7B
:1044F000B9F1000F7BD007F0010018B906F49070F5
:10450000002874D005F0010030B106F4807018B1B5
:10451000606C40F00100606405F0040030B107F009
:10452000010018B1606C40F00200606405F0020008
:1045300030B107F0010018B1606C40F00400606415
:1045400005F0080048B106F0200010B907F001009E
:1045500018B1606C40F008006064606C002845D0C1
:1045600005F0200028B106F0200010B1204604F02C
:10457000A3FE20684069C0F3801A606C00F0080058
:1045800010B9BAF1000F2CD0204604F028FE2068A4
:10459000406900F0400000B300BF00BF2168143143
:1045A00051E8001F21F040002168143141E8000269
:1045B000002AF3D100BFE06B50B17748E16B48634C
:1045C000E06BFDF7BDFC88B1E06B416B88470DE007
:1045D0002046FFF757FF09E009E02046FFF752FFAA
:1045E00004E02046FFF74EFF002060647EE7206B6A
:1045F000012877D105F01000002873D006F01000D4
:104600000028FAD000BF00200090206800680090C9
:1046100020684068009000BF00BF2068406900F03B
:10462000400000285FD0E06B006840681FFA80F807
:10463000B8F1000F55D0A08D404552DDA4F82E8072
:10464000E06B8069202843D000BF00BF21680C3197
:1046500051E8001F21F4807021680C3141E800020C
:10466000002AF3D100BF00BF00BF2168143151E818
:10467000001F21F001002168143141E80002002AE6
:10468000F3D100BF00BF00BF2168143151E8001F03
:1046900021F040002168143141E80002002AF3D1E2
:1046A00000BF202084F842000020206300BF00BF2C
:1046B00021680C3151E8001F21F0100021680C31F5
:1046C00041E80002002AF3D100BFE06BFDF70CFCCB
:1046D00002206063A08DE28D801A81B22046FFF730
:1046E0008BFE03E742E0A08DE18D401A1FFA80F8AF
:1046F000E08DD0B3B8F1000F37D000BF00BF216804
:104700000C3151E8001F21F4907021680C3141E810
:104710000002002AF3D100BF00BF00BF216814319E
:1047200051E8001F21F001002168143141E8000226
:10473000002AF3D100BF202084F84200002020632B
:1047400000BF00BF21680C3151E8001F21F01000AC
:1047500021680C3141E80002002AF3D100BF022099
:10476000606341462046FFF747FEBFE605F0800044
:1047700030B106F0800018B1204604F0FDFEB5E629
:1047800005F0400030B106F0400018B1204604F0BA
:104790005CFDABE600BFA9E63D90000810B50446FD
:1047A0000CB9012010BDA06900B100E000BF94F871
:1047B000410028B9002084F84000204600F02AF883
:1047C000242084F841002068C06820F4005021684B
:1047D000C860204604F0EEFD2068006920F4904097
:1047E000216808612068406920F02A00216848613A
:1047F0002068C06840F400502168C86000206064F0
:10480000202084F8410084F842000020606300BF4B
:10481000C8E7000010B586B004460020029003905F
:104820000490059055492068884237D100BF54480C
:10483000806940F48040524988610846806900F4EC
:104840008040019000BF00BF00BF0846806940F073
:10485000040088610846806900F00400019000BFF0
:1048600000BF48150290022003900320059002A982
:104870004448FDF7C1FD4FF4806002900020039092
:10488000049002A93F48FDF7B7FD0022052125202D
:10489000FDF7DCFF2520FDF7C9FF6CE03A492068F1
:1048A000884268D100BF3648C06940F400303449BE
:1048B000C8610846C06900F40030019000BF00BF25
:1048C00000BF0846806940F004008861084680699E
:1048D00000F00400019000BF00BF042002900220FD
:1048E00003900320059002A92648FDF785FD0820C6
:1048F000029000200390049002A92248FDF77CFD5D
:104900002248234908600020486000212048816037
:104910008021C1600021016141618161C161FDF7B8
:1049200035FC08B1FDF728F900BF1948E06344627F
:1049300000BF164814301749086010204860002155
:10494000144881608021C160002101614161816161
:10495000C161FDF71BFC08B1FDF70EF900BF0D4862
:10496000A063446200BF002205212620FDF76EFFF0
:104970002620FDF75BFF06B010BD000000380140A7
:104980000010024000080140004400406C0002405A
:10499000C80500200C06002070B504460D461646DA
:1049A00094F8420020280BD105B10EB9012070BD4A
:1049B0000020206332462946204604F079FDF6E7C0
:1049C0000220F4E770B50546284604F061FC044671
:1049D000032C0DD004EBC400064901EB8000C06835
:1049E00030B104EBC401034A02EB8101C86880477F
:1049F00070BD0000E823002070B50546284604F08D
:104A000047FC0446032C0DD004EBC400064901EB1F
:104A10008000806830B104EBC401034A02EB8101DD
:104A20008868804770BD0000E82300202DE9F84F1A
:104A300004460E46174699464FF0000A94F8410086
:104A4000202850D106B117B90120BDE8F88F002009
:104A50006064212084F84100FDF76CFE8246A78443
:104A6000E784A068B0F5805F04D1206910B9002503
:104A7000B04602E035464FF000081EE053460022E3
:104A800080212046CDF8009004F0A6FD20B1202022
:104A900084F841000320D8E745B9B8F80000C0F316
:104AA00008002168486008F1020803E028782168BE
:104AB00048606D1CE08C401EE084E08C0028DDD155
:104AC0005346002240212046CDF8009004F084FD9A
:104AD00020B1202084F841000320B6E7202084F88C
:104AE00041000020B1E70220AFE70000F7B504461F
:104AF000154694F84100202836D1019800B10DB92F
:104B00000120FEBD01982062A584E5840020606438
:104B1000212084F841001548A16B88621448A16BDC
:104B2000C8621448A16B08630020A16B486301AE02
:104B300023681A1D31682B46A06BFDF75BFB6FF0F5
:104B400040002168086000BF00BF2168143151E8AF
:104B5000001F41F080002168143141E80002002A62
:104B6000F3D100BF0020CCE70220CAE7799100080A
:104B7000D19100085190000810B5034693F8410008
:104B8000202813D101B10AB9012010BD19629A84FD
:104B9000DA8400205864212083F841001868C06836
:104BA00040F080001C68E0600020EEE70220ECE7A7
:104BB00070B50546284604F06BFB0446032C0DD067
:104BC00004EBC400064901EB8000406830B104EBFF
:104BD000C401034A02EB81014868804770BD0000B0
:104BE000E823002070B50546284604F051FB044632
:104BF000032C0BD004EBC400054951F8200028B168
:104C000004EBC401024A52F82100804770BD000045
:104C1000E823002000BFFEE7F8B5054628128DF80E
:104C20000000E8B28DF80100F02387220021084639
:104C300000F00AFC4FF48776304605F055FE044636
:104C400014B96FF00100F8BD002007E09DF80010D6
:104C500021549DF80120411C6254801CB042F5D3C0
:104C6000002704E0B1B2204600F07AFC7F1CF02F50
:104C7000F8D3204605F024FD0020E4E72DE9FF5F8E
:104C800007468A469346984627B96FF0010004B05C
:104C9000BDE8F09F08F10700C11700EB5171C1F3A7
:104CA000CF0900263FE006FB09700390002436E0A0
:104CB0000398005D029000252CE005EBC40080B253
:104CC00001900198404500DB26E0002000901098FC
:104CD000012809D1802028410299084008B101200B
:104CE00000E00020009008E00120A8400299084060
:104CF00008B1012000E000200090009840B10BEBCB
:104D0000060291B2019A524490B20F9A00F002FA50
:104D1000681CC5B2082DD0DB00BF601C84B24C45B6
:104D2000C6DB701C86B20E988642BCDB0020AEE764
:104D30002DE9FF4F87B0804689461546202D01DBBF
:104D40007E2D04DD4FF0FF300BB0BDE8F08FA5F1F4
:104D50002000C0B206904FF0000A00260020059007
:104D6000049014980C2806D0102805D0182839D0A3
:104D7000202871D18EE091E04A49069801EB001A93
:104D8000082610200590002728E01AF80700039055
:104D900000241FE008EB040080B2029009EB07003A
:104DA00080B201901598012806D1C4F1070103983B
:104DB000084100F0010B03E00398204100F0010BD3
:104DC000BBF1000F04D00A9ADDE9011000F0A2F94E
:104DD000601CC4B2B442DDDB781CC7B205988742C0
:104DE000D3DB5BE0069800EB40002F4901EB001A93
:104DF0000C2618200590F01DC11700EB5171C91049
:104E00000491002742E000243CE008EB040080B25B
:104E1000039009EB070080B202902046E11704EBF3
:104E20005171C1F3C70101910499019807FB010079
:104E30001AF800000090159801280ED12046E117BD
:104E400004EB5171C910A4EBC101C1F10702009933
:104E5000114101F0010B0BE01DE02046E11704EBCE
:104E60005171C910A4EBC1020099114101F0010B6D
:104E7000BBF1000F04D00A9ADDE9021000F04AF9F4
:104E8000601CC4B2B442C0DB781CC7B2059887422C
:104E9000B9DB03E002E04FF0FF3055E700BF002030
:104EA00052E70000EC020108DC0801082DE9FF4F81
:104EB00087B0804689461546202D01DB7E2D04DD16
:104EC0004FF0FF300BB0BDE8F08FA5F1200000F0EF
:104ED000FF0A0020069000260590049015980C28E3
:104EE00006D0102805D018283CD0202874D194E092
:104EF00097E04D4800EB0A10069008261020059018
:104F000000272BE00698C05D0390002422E008EB08
:104F1000040080B2029009EB070080B2019016985D
:104F2000012806D1C4F107010398084100F0010BE4
:104F300003E00398204100F0010BBBF1000F01D00A
:104F40000A9800E014980246DDE9011000F0E2F84A
:104F5000601CC4B2B442DADB781CC7B20598874241
:104F6000D0DB5EE00AEB4A00304901EB001006900E
:104F70000C2618200590F01DC11700EB5171C910C7
:104F80000491002745E000243FE008EB040080B2D4
:104F9000039009EB070080B202902046E11704EB72
:104FA0005171C1F3C70101910499019807FB0101F7
:104FB0000698405C0090169801280ED12046E11713
:104FC00004EB5171C910A4EBC101C1F107020099B2
:104FD000114101F0010B0BE020E02046E11704EB4A
:104FE0005171C910A4EBC1020099114101F0010BEC
:104FF000BBF1000F01D00A9800E014980246DDE9E9
:10500000021000F087F8601CC4B2B442BDDB781C0B
:10501000C7B205988742B6DB03E002E04FF0FF30ED
:1050200050E700BF00204DE7EC020108DC08010852
:105030002DE9FF4F83B006460F460598841B06985E
:10504000C51B002C01DB012001E04FF0FF30029076
:10505000002D01DB012001E04FF0FF300190002C1A
:1050600001DB204600E060420446002D01DB2846BB
:1050700000E0684205464CB945B939463046109AB9
:1050800000F048F8002007B0BDE8F08FAC421FDD0B
:10509000204604EBD0714FEA6108B146BA464FF0A2
:1050A000000B12E01FFA8AF11FFA89F0109A00F043
:1050B00031F802988144A8EB0508B8F1000F02DA34
:1050C00001988244A0440BF1010BA345EADD1FE0E7
:1050D000284605EBD0714FEA6108B146BA464FF059
:1050E000000B12E01FFA8AF11FFA89F0109A00F003
:1050F00011F801988244A8EB0408B8F1000F02DA15
:1051000002988144A8440BF1010BAB45EADD00BFD6
:105110000020B8E7FEB505460E46144601AB02AACC
:105120003146284600F068F901231A46BDF80410FC
:10513000BDF8080000F088F920128DF80000E0B2F8
:105140008DF801000221684600F000FA0020FEBD43
:105150002DE9FF4F85B0054688461446DDF8489096
:10516000AA46CDF81080B9F10C0F09D0B9F1100F93
:1051700007D0B9F1180F0BD0B9F1200F10D10EE004
:1051800013E04FF0080B10200390092611270CE0C4
:105190004FF00C0B182003900D26192705E004E0B2
:1051A0004FF0FF3009B0BDE8F08F00BF18E0207865
:1051B0000A2806D1AA460498384480B20490641C98
:1051C0000EE01398CDE9009022785046089B049990
:1051D000FFF7AEFD0AEB06001FFA80FA641C00BF61
:1051E00020780028E3D100BFDCE72DE9FF4F85B030
:1051F000054688461446DDF84C90AA46C346B9F1E8
:105200000C0F09D0B9F1100F07D0B9F1180F0BD05E
:10521000B9F1200F10D10EE013E008200490102007
:105220000390092611270CE00C200490182003900D
:105230000D26192705E004E04FF0FF3009B0BDE866
:10524000F08F00BF1AE020780A2806D1AA460BEB9F
:1052500007001FFA80FB641C10E012991498CDE936
:1052600000190290227859465046089BFFF71EFE0F
:105270000AEB06001FFA80FA641C00BF20780028A1
:10528000E1D100BFDAE7000010B58AB004464E480D
:10529000047000224FF480414C48FDF745FA32205B
:1052A000FCF7F6FF012291034848FDF73DFA322052
:1052B000FCF7EEFF362000F00DF934B1012C08D0D8
:1052C000022C0AD0032C10D10BE0082000F020F9AA
:1052D0000CE0602000F01CF908E0A02000F018F9B4
:1052E00004E0C82000F014F900E000BF00BF3A203D
:1052F00000F0F0F8052000F00BF9B22000F0EAF819
:1053000033A103C9CDE90801052108A800F01EF961
:10531000B72000F0DFF8352000F0FAF8BB2000F0ED
:10532000D9F8192000F0F4F8C02000F0D3F82C20B0
:1053300000F0EEF8C22000F0CDF8012000F0E8F80F
:10534000C32000F0C7F8122000F0E2F8C42000F0FB
:10535000C1F8202000F0DCF8C62000F0BBF80F20D8
:1053600000F0D6F8D02000F0B5F8A42000F0D0F876
:10537000A12000F0CDF8E02000F0ACF816A090E8F5
:105380000E00C068CDE90523049107900E2104A802
:1053900000F0DCF8E12000F09DF813A30FCB8DE8BE
:1053A0000F000E21684600F0D1F8212000F092F89D
:1053B000112000F08FF87820FCF76AFF292000F018
:1053C00089F800200AB010BD98000020000C0140B0
:1053D0000C0C003333000000D0040D11132B3F548C
:1053E0004C180D0B1F230000D0040C11132C3F444C
:1053F000512F1F1F2023000010B5044611480078CC
:1054000030B1012807D002280AD0032814D10CE0BB
:105410001480198013E01180C4F1EF0018800EE0B1
:10542000C1F1860010801C8009E0C4F18600108064
:10543000C1F1EF00188002E01480198000BF00BFA6
:10544000002010BD980000202DE9FC5F06460F46A5
:105450009046994606F1340084B204EB0800401EE1
:105460001FFA80FA07F1280085B205EB0900401EFB
:105470001FFA80FB2A2000F02DF820128DF804007E
:10548000E0B28DF805004FEA2A208DF806000AF0F8
:10549000FF008DF80700042101A800F057F82B2029
:1054A00000F018F828128DF80000E8B28DF801001D
:1054B0004FEA2B208DF802000BF0FF008DF803005F
:1054C0000421684600F042F82C2000F003F8002088
:1054D000BDE8FC9F01B500224FF480710A48FDF73A
:1054E00023F900224FF480510848FDF71DF90123EC
:1054F0001A4669461846FBF701FF012211030348CB
:10550000FDF712F9002008BD00080140000C014021
:1055100001B5012211020B48FDF706F900224FF4F4
:1055200080510948FDF700F901231A4669461846DB
:10553000FBF7E4FE012211030348FDF7F5F8002014
:1055400008BD000000080140000C014070B5044691
:105550000D462946204600F003F8002070BD0000EB
:1055600070B504460D46012211020E48FDF7DCF825
:1055700000224FF480510C48FDF7D6F801232A464B
:1055800021461846FBF7BAFE00BF0120FBF796FE46
:105590000128FAD1012201030348FDF7C5F80020D4
:1055A00070BD000000080140000C014010B5094822
:1055B000FCF71EFC012802D04FF0FF3010BD06485A
:1055C000FCF716FC012802D04FF0FF30F6E7002070
:1055D000F4E70000504C0108604C010870B5044627
:1055E0000E4604B116B94FF0FF3070BDFBF766FFF1
:1055F00028B9FBF777FF4AA004F0B2FA02E054A002
:1056000004F0AEFA202104F10800FAF733FEFFF7A8
:10561000CDFFFBF74FFF083020602068427801463D
:10562000574802F0D7FC10B14FF0FF30DDE7554886
:10563000816B00208847206890F8580010B101283D
:105640002CD10FE0FD214E48406880F827107C21C6
:105650004B48406880F82E10FC214948406880F88B
:1056600022101CE0206890F85A00801CC1B2444807
:10567000406880F82710206890F85A00801CC1B25A
:105680003F48406880F82E10206890F85A00801C2F
:10569000C1B23B48406880F8221000E000BF00BF64
:1056A000374A526802F11D00364A516C8847344827
:1056B00040680078022803D1314803F043F920E024
:1056C0002F484068007801281BD1206890F85800C6
:1056D00010B1012809D102E02B48057807E02068C5
:1056E000B0F85A00801C85B201E0002500BF00BF61
:1056F000002D05DDEAB204F12801214803F05EF92E
:1057000000BF0120FFF7C0FD00F0E0FB40F2DC50DD
:10571000FCF7BEFD204600F0ADF9002065E7000073
:105720005B4D5231365D20466C61736820636F6E4D
:1057300066696720696E76616C69642C207573698F
:105740006E672064656661756C74730D0A000000F5
:105750005B4D5231365D20436F6E666967206C6F1A
:10576000616465642066726F6D20466C61736820A9
:105770007375636365737366756C6C790D0A0000ED
:10578000E02C0020341C0108040000202DE9F04129
:1057900004469D48007800287ED0002501E0681C62
:1057A000C5B29A48007885420FDA9948405D2028B2
:1057B000F5D09748405D0928F1D09548405D0D2807
:1057C000EDD09348405D0A28E9D0904800788542A2
:1057D00013DA8F48405D612803DB8D48405D7A28ED
:1057E00007DD8B48405D412807DB8948405D5A282A
:1057F00003DC0020874908700CE08448007800280A
:1058000008DD824802788249204600F013F9012021
:10581000804908707F480078002850D17B48007884
:10582000002822DD7948007840281ED27748027887
:1058300077497948FAF705FD00207749734A1278CD
:1058400088547248067804E00021701E0646724AA9
:105850001154002E08DD701E6F49085C0D28F3D02E
:10586000701E085C0A28EFD002E000206A49087028
:105870006A48816B0020884703F0A8FF8046042017
:1058800004F0B8F803F0E8FF00206549087001272C
:1058900000BF4FF4807200E015E061495E48FCF7FC
:1058A0003BFA07465E48007818B15D495DA004F0F8
:1058B00057F900205A490870012FEAD000BF002094
:1058C0005149087000BFFBF774FD0646FAF7BEFFAA
:1058D00005465549FAF79BFEA060FBF76AFDD4E93F
:1058E0000423861A61EB03013046FAF7AFFF054641
:1058F0004D49FAF78CFEA061FBF75BFDC4E904019A
:105900004A4840680078022837D1616AA068FAF7EF
:1059100078FE05464649FAF7F1FF2ED22168B1F824
:105920005C10091284F82810216891F85C20292164
:105930000A55FF222A210A5500222B210A55FF224F
:105940002C210A5500222D210A55216891F8581062
:1059500019B92E490978881C04E02168B1F85A1059
:10596000891C88B2062105E0002304F12802535463
:105970004A1C91B28142F7DB00BF206890F85800C2
:1059800010B1012835D112E028484068007801287C
:1059900002D0022808D103E0244802F013FE04E0FC
:1059A000224802F00FFE00E000BF00BF22E01F48C7
:1059B00040680078012802D0022817D103E01B4874
:1059C00002F000FE13E0194802F0FCFDE169A06856
:1059D000FAF717FE05464FF07E51FAF78FFF04D80D
:1059E000204600F0D7FAA168E16100E000BF00BFE7
:1059F00000E000BF00BFFCF79DFE054604F000F884
:105A00000020BDE8F0810000050000200400002017
:105A10003704002009010020EF2D0020341C01086C
:105A20002F2E00202573000000247449E02C002054
:105A3000CDCCCC3D70B504460E4615461CB116B112
:105A40000DB1F52D02DD4FF0FF3070BD2068B0F8CC
:105A50005C00001284F82800206890F85C1029206F
:105A600001552A46314604F12A00FAF7EAFB0020E4
:105A7000EBE700002DE9F04790B004460CB1206838
:105A800020B94FF0FF3010B0BDE8F0870020FFF7DD
:105A9000C3F8002018214DF6A703D6A2CDE90010C7
:105AA00005210846FFF754FBD548007801280BD1A3
:105AB000002018214FF62053D2A2CDE90010052175
:105AC000C820FFF745FB0AE0002018214FF4FC63D3
:105AD000CDA2CDE900100521C820FFF739FB48F21F
:105AE00010401E238722194600900020FFF7A0FADD
:105AF0000020102140F2FF73C4A2CDE9001028213C
:105B00000520FFF725FBC3A64FF6FF79206890F824
:105B1000580010B1012808D103E0C0A64FF6FF7964
:105B200007E0C1A64FF4FC6903E0C1A64AF6555947
:105B300000BF00BF002010214B463246CDE90010C7
:105B400028214120FFF704FB0020102140F2FF73C1
:105B5000B9A2CDE9001041210520FFF7F9FA0FF2B3
:105B6000D02AA7484068407F40B1012809D00328C7
:105B70000AD004280BD10FF2C82A09E00FF2C42A78
:105B800006E00FF2C82A03E00FF2C82A00E000BFC7
:105B900000BF002010214FF6FF735246CDE90010E0
:105BA00041210846FFF7D4FA0020102140F2FF738C
:105BB000AAA2CDE900105A210520FFF7C9FA9048A2
:105BC0004068A84A0023D0E912713846FAF7F8FA7B
:105BD000CDE90A01A4A2CDE900010F210CA803F030
:105BE000CFFF002010214FF6FF730CAACDE9001063
:105BF0005A213220FFF7ACFA23258148007801288A
:105C000067D10020102140F2FF7399A2CDE9001066
:105C100073210520FFF79CFA2068B0F85C3096A24B
:105C20000A2109A803F0ACFF002010214FF6FF73F2
:105C300009AACDE9001073214120FFF789FA05F187
:105C4000190085B20020102140F2FF738CA2CDE92B
:105C5000001028217820FFF77BFA6948406890F906
:105C6000503089A20A2106A803F08AFF00201021E3
:105C70004FF6205306AACDE900102821B420FFF7E3
:105C800067FA05F1190085B2206890F858000128DC
:105C90001ED10020102140F2FF737DA2CDE900103B
:105CA00041217820FFF754FA2068B0F85A307BA2DF
:105CB0000A2103A803F064FF002010214FF62053AF
:105CC00003AACDE900104121BE20FFF741FA00BF31
:105CD0008EE00020102140F2FF7371A2CDE9001088
:105CE00029467820FFF734FA05F1140085B26FA237
:105CF000142107A8D4F8A83003F042FF0020102197
:105D00004FF4FC6307AACDE9001029467820FFF77D
:105D10001FFA05F1140085B2AC20035965A21421C5
:105D200007A803F02DFF002010214FF4FC6307AA01
:105D3000CDE9001029467820FFF70AFA05F1140092
:105D400085B2B02003595DA2142107A803F018FF03
:105D5000002010214FF4FC6307AACDE9001029466A
:105D60007820FFF7F5F90020102140F2FF7355A2CB
:105D7000CDE9001073210520FFF7EAF92068B0F89B
:105D80005E303DA2142107A803F0FAFE0020102186
:105D90004FF6FF7307AACDE9001073214120FFF7EA
:105DA000D7F92068B0F8603033A2142107A803F0B7
:105DB000E7FE002010214FF6FF7307AACDE900107F
:105DC00073217D20FFF7C4F92068B0F862302AA261
:105DD000142107A803F0D4FE002010214FF6FF7312
:105DE00007AACDE900107321B920FFF7B1F900BF70
:105DF000002048E64D5231362053746174757300AB
:105E0000E02C002054580000525800004D6F64658B
:105E10003A000000554E4B4E4F574E0056415249E6
:105E200041424C45000000004649584544000000EE
:105E30004E4F4E4500000000526164696F3A000009
:105E4000424C45004746534B000000004C4F524126
:105E500000000000464C524300000000467265718D
:105E60003A00000040420F00256C6C754D487A00E6
:105E7000545849443A000000307825303458000026
:105E8000506F7765723A0000256464426D0000002F
:105E9000446174614C656E3A000000002564420064
:105EA0007278636F756E743A000000006368313A6F
:105EB000256C75006368323A256C75006368333A67
:105EC000256C7500727869643A0000000EB50020F8
:105ED000FEF7A2FE0020102140F2FF731EA2CDE9C2
:105EE000001077216E20FFF733F901204DF6A7014E
:105EF00020223023CDE900210290002211461A48C9
:105F0000FEF7BCFE6420FCF7C3F901204DF6A701A3
:105F10001C221346CDE900210290042230211348AF
:105F2000FEF7ACFE6420FCF7B3F9002018214DF613
:105F3000A7030FA2CDE900103021FFF709F90020D7
:105F400018214DF6A7030EA2CDE900104821FFF756
:105F5000FFF800200EBD0000496E697469616C692C
:105F60007A696E672E2E2E00AC1A01086C1B010890
:105F70004D5231362D2D576972656C657373000073
:105F80007472616E736D697373696F6E20746F6F75
:105F90006C00000030B589B004461CB94FF0FF30EA
:105FA00009B030BD2148007803283DD123251435A0
:105FB0001FA2142104A8D4F8A83003F0E1FD0020AA
:105FC0001021CDE900014FF4FC6304AA2946029098
:105FD0007820FFF70AF91435AC20035916A21421D2
:105FE00004A803F0CDFD00201021CDE900014FF4FD
:105FF000FC6304AA294602907820FFF7F6F81435CE
:10600000B02003590EA2142104A803F0B9FD00200A
:106010001021CDE900014FF4FC6304AA2946029047
:106020007820FFF7E2F800BF0020B9E7E02C00205D
:106030006368313A256C75006368323A256C7500E7
:106040006368333A256C750010B504462046FBF7AB
:1060500001FF0346012B01D8062010BD032B01D8F8
:106060000720FAE7052B01D80820F6E7072B01D80F
:106070000920F2E7092B01D80A20EEE70F2B01D8FF
:106080001720EAE72820E8E708B500BF1E48406966
:1060900040F001001C4948610846406900F00100D9
:1060A000009000BF00BF002205210C20FCF7CEFBB2
:1060B0000C20FCF7BBFB002205210D20FCF7C6FBE2
:1060C0000D20FCF7B3FB002205210E20FCF7BEFBE0
:1060D0000E20FCF7ABFB002205210F20FCF7B6FBDE
:1060E0000F20FCF7A3FB002205211020FCF7AEFBDC
:1060F0001020FCF79BFB002205211120FCF7A6FBDA
:106100001120FCF793FB08BD0010024010B5064AB1
:106110000021064805F05DF905490860054A00219F
:10612000054805F056F910BD94020108058B0008DA
:1061300000000020704C0108298F000800B585B0D0
:106140000020019002900390049000BF49488069AC
:1061500040F02000474988610846806900F020002F
:10616000009000BF00BF00BF0846806940F00400F7
:1061700088610846806900F00400009000BF00BFFD
:1061800000BF0846806940F00800886108468069C1
:1061900000F00800009000BF00BF00224FF488719B
:1061A0003548FCF7C1FA002245F219213348FCF7C3
:1061B000BBFA4FF4887001900120029000200390F8
:1061C0000220049001A92C48FCF716F90120019047
:1061D000029003900220049001A92848FCF70CF9D2
:1061E0004FF4A4400190012002900020039002206F
:1061F000049001A92148FCF7FFF84FF4805001906A
:106200001F4802900020039001A91B48FCF7F4F8F6
:10621000182001900120029002200390049001A90F
:106220001648FCF7E9F8E020019016480290022099
:10623000039001A91148FCF7DFF84FF4807001903A
:10624000002002900220039001A90C48FCF7D4F82A
:10625000002205211720FCF7F9FA1720FCF7E6FACF
:10626000002205212820FCF7F1FA2820FCF7DEFAAD
:1062700005B000BD0010024000080140000C0140C4
:10628000000021100000111010B50E480E490860E2
:106290004FF48270486000210B488160C160016149
:1062A00041614FF4007181611021C16100210162DF
:1062B000416281620A21C162FCF72CFF08B1FBF741
:1062C0005BFC10BD003001403001002010B50E48CD
:1062D0000E4908604FF48270486000210B488160CD
:1062E000C160016141614FF4007181610821C161A8
:1062F00000210162416281620A21C162FCF70AFF4A
:1063000008B1FBF739FC10BD0038004088010020BF
:1063100000B595B0002011901290139014900F903A
:1063200010901C2108A8F9F7A5FF20216846F9F76D
:10633000A1FF2A482A490860002048600021284817
:1063400081605921C1600021016141618161FDF7D6
:1063500083FC08B1FBF710FC4FF48050119011A999
:106360001F48FDF7EFFC08B1FBF706FC1C48FDF7E2
:106370001FFE08B1FBF700FC00200F9010900FA942
:106380001748FDF727FC08B1FBF7F6FB60200890E3
:10639000002009900A900C900D900E900C2208A9F4
:1063A0000F48FDF783FD08B1FBF7E6FB00200090E6
:1063B00001900290039004904FF40050059000204B
:1063C000079069460648FDF7CBFB08B1FBF7D4FB05
:1063D0000348FDF73FFD15B000BD0000002C014053
:1063E000AC02002010B50C480C4908600C4848600D
:1063F00000210A4881604FF40051C160C910016159
:106400000C21416100218161C161FEF7C7F908B12A
:10641000FBF7B2FB10BD000000380140380500203A
:10642000A086010010B51148114908604FF4E13011
:10643000486000210E488160C16001610C2141610A
:1064400000218161C161FEF7A9F908B1FBF794FB56
:10645000FF2208490648FEF79FFA05480068C06811
:1064600040F0100002490968C86010BD00440040B7
:10647000800500203803002000BFFEE700BFFEE7D4
:1064800010B50220034908700846007801F022FC8C
:1064900010BD0000C000002010B5044604200349D0
:1064A00008700846007801F015FC10BDC0000020FF
:1064B00010B50320034908700846007801F00AFC73
:1064C00010BD0000C000002010B505A003F048FB7F
:1064D0000520074908700846007801F0FBFB10BD55
:1064E0005B54585D2054585F444F4E450D0A0000E0
:1064F000C000002010B505A003F032FB06200849BB
:1065000008700846007801F0E5FB10BD5B54585D4B
:106510002054585F54494D454F5554210D0A0000F1
:10652000C000002008B508490968C9084FF47A720C
:10653000B1FBF2F14143009100BF00BF00994A1E38
:1065400000920029F9D108BD1400002010B50248BE
:10655000FCF746FD10BD00003001002010B50248D8
:10656000FCF73EFD10BD00008801002070B5054617
:106570006C6A0020E087E0862046FCF711FD70BDC4
:1065800070B505466C6A2068406820F003002168F9
:106590004860606D40F010006065012084F8510093
:1065A0002046FCF7FDFC70BD70B50446656A2846C0
:1065B000FCF702FF70BD70B50446656A2846FDF71A
:1065C00061FA70BD70B50446656A2846FDF792FA17
:1065D00070BD70B505466C6AFCF7ACF806462868D5
:1065E000006800F0200020282BD02068406820F0B0
:1065F000200021684860A06850B96068B0F5827FCB
:1066000006D12068406820F003002168486005E05A
:106610002068406820F0010021684860324664210B
:10662000204600F085F808B1202060650020E08752
:10663000012084F85100606D18B12046FCF7B0FCD1
:1066400070BD2046FCF79CFE00BFF9E7F8B5054693
:106650006C6AFCF76FF806462868006800F02000B6
:1066600020282DD02068406820F020002168486054
:106670002068406820F002002168486032466421AA
:10668000204600F091F818B1606D40F02000606580
:10669000A06850B900BF002000902068C06800903A
:1066A00020688068009000BF00BF0020E0860120C5
:1066B00084F85100606D18B12046FCF771FCF8BDFC
:1066C0002046FDF7C9F900BFF9E770B505466C6AC9
:1066D000FCF730F806462868006800F02000202803
:1066E00021D02068406820F02000216848603246B0
:1066F0006421204600F058F818B1606D40F0200089
:1067000060652068406820F0030021684860002030
:10671000E086E087012084F85100606D18B12046C2
:10672000FCF73EFC70BD2046FDF7C8F900BFF9E755
:10673000F8B504460E4615466068B0F5827F0DD167
:10674000A068B0F5004F03D0A068B0F5806F05D108
:106750002068006820F04000216808606068B0F59B
:10676000827F11D1A068B0F5806F0DD13346002231
:1067700001212046009500F04DF898B1606D40F081
:10678000200060650320F8BD3346002280212046AA
:10679000009500F03FF828B1606D40F02000606582
:1067A0000320F0E70020EEE7F8B504460E46154654
:1067B0003346012202212046009500F02BF828B133
:1067C000606D40F0200060650320F8BD3346002274
:1067D00080212046009500F01DF828B1606D40F042
:1067E000200060650320F0E70020EEE70146074A3D
:1067F0000868904201D100207047054A086890421D
:1068000001D10120F8E70320F6E700000030014045
:10681000003800402DE9F84F04460D4690461E46CC
:10682000DDF82890FBF786FFA0EB0900371AFBF78D
:1068300081FF82462C480068C0F3CB30784300903B
:1068400045E0701C002842D0FBF774FFA0EB0A0063
:10685000B84200D2A7BB2068406820F0E000216861
:1068600048606068B0F5827F0DD1A068B0F5004F38
:1068700003D0A068B0F5806F05D12068006820F0D3
:10688000400021680860A06AB0F5005F0DD100BF2C
:106890002068006820F400502168086020680068C3
:1068A00040F400502168086000BF012084F85100C6
:1068B00000BF002084F8500000BF0320BDE8F88F1F
:1068C000FFE7009800B900270098401E009020685C
:1068D00080682840A84201D1012000E00020404506
:1068E000AFD10020EAE700001400002030B50346D5
:1068F0000C461546002207E0184600F008F824F878
:1069000012009B1C501C82B2AA42F5DB30BD01462E
:10691000088870472DE9F05F80468A461746B8F12F
:10692000006F02D33A48804501D3BDE8F09FFBF7E2
:1069300025FDA8F1006B4FEA9B25CBF34809C9F56B
:106940000074A74200DC3C465CE04FF0006101EBC4
:1069500085208A142F49FFF7C9FF00260BE009EBB9
:1069600006002C4931F810004FF6FF71884200D024
:1069700003E0701C86B2A642F1DB00BFA64225DA16
:106980004FF0006101EB8520FBF784F94CF25030A9
:10699000FBF748F92048006920F002001E49086111
:1069A000002608E03AF8160006EB0901194A22F819
:1069B0001100701C86B2A642F4DB4FF0006101EBBF
:1069C00085208A14134900F029F808E04CF2503071
:1069D000FBF728F922465146404600F01FF8A7422F
:1069E00000D110E06D1C4FF000090AEB440A08EBDF
:1069F0004408381B87B2B7F5007F02DD4FF40074FE
:106A000000E03C46A1E700BFFBF756FC00BF8CE767
:106A100000000108681F0020002002402DE9F0411D
:106A200004460E46174600250AE036F815C06246B1
:106A3000002321460120FBF749FCA41C681C85B2F9
:106A4000BD42F2DBBDE8F08101B582B09DF80800DF
:106A5000C0F3401040019DF80810C1F3001140EA56
:106A600001109DF80810C1F3C00140EAC1009DF873
:106A70000810C1F3800140EA81009DF80810C1F3BD
:106A8000400140EA41009DF8081001F0010108436F
:106A90000190012201A9892000F0D2FB0EBD38B57A
:106AA0000446200A8DF80000E0B28DF801000222B1
:106AB0006946972000F0C4FB38BD10B54FF4AA70AA
:106AC00000F02CFB044640F2531000F027FB44EA90
:106AD000002010BD2DE9F04F85B0002004908246C3
:106AE00000210C460D4600F01FFA032853D004DCA9
:106AF000002851D0012850D104E004284AD00F28A2
:106B00004BD146E040F6541000F008FB8DF8100021
:106B100040F6551000F002FB8DF8110040F65610BB
:106B200000F0FCFA8DF812009DF8100000049DF8AA
:106B3000111040EA01209DF8121040EA010ACAF340
:106B4000130A00F047F88346F9F78EFE06463246F0
:106B50000B4600201449F9F70AFE80460022134B29
:106B6000F9F793FDCDE902011421504601F086FFAB
:106B70008046F9F779FE06460D4A0E4BF9F785FD7A
:106B8000CDE90001DDE90223F9F7F1FD04460D46E8
:106B900003E000BF00BF00BF00BF00BF2046294682
:106BA00005B0BDE8F08F00000000994000408F4024
:106BB000CDCCCCCCCCCCF83F08B502226946152010
:106BC00000F074FA9DF801009DF8001040EA0120E1
:106BD00008BD000000200B4909780A290BD01829AC
:106BE00007D0262903D0342907D1074807E00748F2
:106BF00005E0074803E0074801E0002000BF00BFB0
:106C000070470000C600002075190300EA32060034
:106C1000D4650C00A8CB180001480078704700002C
:106C2000C40000201CB50446052269461D2000F062
:106C30003DFA00F079F920702078032870D003DC49
:106C400038B1012857D157E004286AD00F28F9D16C
:106C500061E19DF80010484200EBD071491049B243
:106C600061709DF80110484200EBD07149104AB2A2
:106C7000A2709DF802008009E17860F30001E170E4
:106C80009DF802004009E17860F34101E1709DF850
:106C900002000009E17860F38201E1709DF80200D2
:106CA000C008E17860F3C301E1709DF8020080083C
:106CB000E17860F30411E1709DF802004008E1788A
:106CC00060F34511E1709DF80200E17860F38611F0
:106CD000E1709DF803004009217960F30001217102
:106CE0009DF80300217960F3410121719DF80400B2
:106CF00000F00700607114E19DF80010484200EBBD
:106D0000D071491049B261709DF80120802A09DADA
:106D10009DF80110CA1701EB92729210A2700BE05D
:106D20004DE0ADE09DF80120A2F58070C21700EBA8
:106D30009272921053B2A3709DF802008009E1781C
:106D400060F30001E1709DF802004009E17860F312
:106D50004101E1709DF802000009E17860F38201D1
:106D6000E1709DF80200C008E17860F3C301E170B2
:106D70009DF802008008E17860F30411E1709DF84D
:106D800002004008E17860F34511E1709DF80200CF
:106D9000E17860F38611E1709DF8030040092179E4
:106DA00060F3000121719DF80300217960F3410136
:106DB00021719DF8040000F007006071B1E09DF8BA
:106DC0000010484200EBD071491049B261709DF843
:106DD0000110484200EBD07149104AB2A2709DF8F0
:106DE00002008109E07861F30000E0709DF8020084
:106DF0004109E07861F34100E0709DF8020000096C
:106E0000E17860F38201E1709DF80200C008E1784A
:106E100060F3C301E1709DF802008008E17860F33F
:106E20000411E1709DF802004008E17860F345111B
:106E3000E1709DF80200E17860F38611E1709DF841
:106E400003008109207961F3010020719DF803009E
:106E50004009217960F3820121719DF80300000946
:106E6000217960F3C30121719DF80300217960F35A
:106E7000041121719DF8040000F00700607150E0DA
:106E80009DF80010484200EBD071491049B2617082
:106E90009DF80110484200EBD07149104AB2A2702F
:106EA0009DF802008009E17860F30001E1709DF82F
:106EB00002004009E17860F34101E1709DF80200B1
:106EC0000009E17860F38201E1709DF80200C008DA
:106ED000E17860F3C301E1709DF802008008E17879
:106EE00060F30411E1709DF802004008E17860F35E
:106EF0004511E1709DF80200E17860F38611E170C0
:106F00009DF8030000F0010020719DF8040000F0DE
:106F10000700607105E000202060A0800F20207035
:106F200000BF00BF1CBD0000014800787047000092
:106F3000C5000020F8B505460C46164669462046B1
:106F400000F01DF82078B04201DD0120F8BD227864
:106F500029469DF8000000F071F80020F6E708B51A
:106F600000200090012269461F2000F09FF89DF844
:106F70000000414201EBD170401040B208BD38B56D
:106F800004460D4602226946172000F08FF8FFF7ED
:106F9000CBFF01280DD140F6031000F0BFF801210E
:106FA000B1EBE01F05D140F6011000F0B7F82070FA
:106FB0000BE0FFF7B9FF042804D19DF80000801C06
:106FC000207002E09DF8000020709DF801002870FC
:106FD00038BD1CB500200190012201A9C02000F09D
:106FE00065F89DF8040000909DF8001008461CBD4F
:106FF00010B54FF480710648FAF746FF0446802129
:107000000348FAF741FF44EA4000C0B210BD000057
:10701000000C014010B5044600F0C4F8204600F012
:1070200001F810BD10B504460022802102482368F3
:10703000FAF732FF10BD0000000C01402DE9F041CD
:1070400005460E461446E71C1B20154908700846E5
:1070500045700020887000BF05E00022C11C104B65
:107060005A54411C88B2A042F7DB00F0B3F800226A
:1070700010210C48FAF72EFF3A460B49084801F058
:107080001DFD22460849C91C3046F9F7DAF80122ED
:1070900010210448FAF71EFF00F09CF8BDE8F081CB
:1070A0007024002000080140702800202DE9F041E4
:1070B00005460E461446A01C87B2154805700020F0
:1070C0001349487000BF05E00022811C104B5A5440
:1070D000411C88B2A042F7DB00F07CF800221021AE
:1070E0000C48FAF7F7FE3A460B49094801F0E6FC6E
:1070F00022460949891C3046F9F7A3F801221021DC
:107100000448FAF7E7FE00F065F8BDE8F0810000FA
:1071100070240020000801407028002038B5044683
:1071200001226946204600F003F89DF8000038BDB2
:107130002DE9F04104460E461546281D87B2192058
:1071400015490870200A48708C700020C87000BF74
:1071500005E00022011D104B5A54411C88B2A84280
:10716000F7DB00F037F8002210210C48FAF7B2FEE6
:107170003A460B49084801F0A1FC2A460849091D76
:107180003046F9F75EF8012210210448FAF7A2FE12
:1071900000F020F8BDE8F0817024002000080140D4
:1071A0007028002010B51420FBF772F8002201218E
:1071B0000748FAF78FFE3220FBF76AF801221146E2
:1071C0000348FAF787FE1420FBF762F810BD0000B1
:1071D000000C014010B500BF4FF480710248FBF76E
:1071E0009BFA0128F8D010BD000C01402DE9F041B8
:1071F00004460E461546AF1C1A200F49087020128F
:1072000048702A4631460C48801CF9F71AF8FFF7F7
:10721000E1FF002210210948FAF75CFE39460648D2
:1072200001F03AFC012210210448FAF753FEFFF75F
:10723000D1FFBDE8F081000070240020000801406B
:107240002DE9F04105460E461446601C87B2FFF753
:10725000C1FF002210210C48FAF73CFE0B480570D4
:1072600022463146401CF8F7ECFF3946074801F04A
:1072700013FC012210210448FAF72CFE842D01D0C2
:10728000FFF7A8FFBDE8F08100080140702400204E
:1072900013B50446012201A9204600F001F81CBDE7
:1072A0002DE9F04104460E461546E81C87B2182029
:1072B0000F490870200A48708C702A4631460C48E5
:1072C000C01CF8F7BEFFFFF785FF00221021094818
:1072D000FAF700FE3946064801F0DEFB01221021D4
:1072E0000448FAF7F7FDFFF775FFBDE8F0810000ED
:1072F000702400200008014010B5044602480460D4
:107300000248FFF787FE10BDD0000020C800002013
:1073100010B505480078012802D10449087001E041
:1073200000F006F810BD0000C7000020CC000020CF
:1073300070B50F25FFF770FC00B970BDB24800783A
:1073400001280AD1B1480078012805D172B6002081
:10735000AE49087062B600E0EFE7FFF7E5FD0546CD
:10736000FFF72AFC04464FF6FF70FFF798FB35B194
:10737000012D7CD0032D03D0042D79D101E000BF75
:1073800000BFA3480078042862D0052871D104F01A
:10739000020002282CD104F0400040280CD19D4866
:1073A000006828B39B480068806908B39948006862
:1073B0008169022088471BE004F0080008280CD1EE
:1073C00094480068A0B193480068806980B19148F2
:1073D00000688169012088470AE08E48006838B15A
:1073E0008C480068406818B18A4909684868804735
:1073F00004F0040004280AD18648006838B18548A2
:107400000068806818B1834909688868804704F07B
:10741000080008280BD17F48006840B17D4800680B
:10742000806920B17B48006881690120884704F4A5
:107430008040B0F5804F0AD17648006838B1754871
:107440000068406918B1734909684869804723E0BA
:1074500004F0010050B16F48006838B16D48006811
:10746000006818B16B4909680868804702E015E0B8
:10747000C5E010E004F48040B0F5804F0AD16548C3
:10748000006838B163480068006918B1614909684B
:107490000869804700E000BF00BFB1E05C480078A9
:1074A000042854D0052802D006286FD16FE004F0DC
:1074B000020002281BD104F0400040280CD155489E
:1074C0000068A0B153480068806980B151480068E5
:1074D0008169022088470AE04E48006838B14D486B
:1074E0000068406818B14B4909684868804704F053
:1074F000100010280AD14748006838B14548006894
:10750000C06818B143490968C868804704F0200082
:1075100020280BD13F48006840B13E480068806990
:1075200020B13C48006881690020884704F480400D
:10753000B0F5804F0AD13748006838B13548006847
:10754000406918B1334909684869804755E004F03B
:10755000010050B12F48006838B12E48006800681B
:1075600018B12C4909680868804704F48040B0F5D8
:10757000804F0AD12748006838B126480068006962
:1075800018B1244909680869804736E034E004F4FA
:107590008050B0F5805F1ED104F40050B0F5005F5C
:1075A0000CD11C48006830B31A480068C06910B399
:1075B00018480068C169012088471CE01548006828
:1075C000C8B114480068C069A8B112480068C16910
:1075D000002088470FE004F48040B0F5804F0AD1C6
:1075E0000C48006838B10B480068406918B1094977
:1075F00009684869804700E000BF00BF00E000BFA5
:1076000000BF00BF99E60000C7000020CC000020AA
:10761000C4000020D000002037B504460D4629469E
:10762000204600F0BFF9029800F0FCFA3EBD01B51B
:10763000012269469E20FFF703FE08BD38B50546C6
:10764000A5F1210084B2200A8DF80000E0B28DF887
:107650000100022269469820FFF7F2FD38BD10B5FF
:107660000446210E40F6CF10FFF712FEC4F3074187
:107670004FF41D60FFF70CFEC4F3072140F6D11054
:10768000FFF706FEE1B240F6D210FFF701FE10BD93
:1076900010B50248FFF7E3FF10BD0000D6BE898E8B
:1076A00038B505460C468DF800508DF80140022291
:1076B00069468F20FFF7C4FD38BD000010B50022D9
:1076C0001146C520FFF7BCFD06200149087010BD1A
:1076D000C400002001B5012269468820FFF7B0FDF3
:1076E00006200149087008BDC400002038B50446D2
:1076F000200A8DF80000E0B28DF80100FFF714FCBD
:1077000010B1032808D100E000BF0222694640F60C
:10771000C610FFF7C5FD00E000BF00BF38BD38B59B
:107720000446200A8DF80000E0B28DF80100FFF752
:10773000FBFB10B1032808D100E000BF022269461C
:1077400040F6C810FFF7ACFD00E000BF00BF38BD39
:107750002DE9FC4107460C4615461E46380A8DF8B1
:107760000000F8B28DF80100200A8DF80200E0B2A6
:107770008DF80300280A8DF80400E8B28DF80500A2
:10778000300A8DF80600F0B28DF80700082269462D
:107790008D20FFF755FDBDE8FC81000010B50022EB
:1077A0001146C120FFF74CFD03200149087010BDB0
:1077B000C40000200020014908707047C700002065
:1077C00001B5012269469B20FFF73AFD08BD000084
:1077D00038B50446207827490978884202D02078B5
:1077E00000F0D2F82078032820D003DC38B101283B
:1077F00038D10EE0042823D00F2833D12AE0607856
:107800008DF80000A0788DF80100E0788DF8020076
:1078100028E020798DF8000060798DF80100A079CA
:107820008DF802006079144908701BE0E0798DF84A
:107830000000207A8DF80100607A8DF8020011E0D6
:10784000A07A8DF80000E07A8DF80100207B8DF899
:10785000020007E000208DF800008DF801008DF88F
:10786000020000BF00BF032269468B20FFF7E8FC3F
:1078700038BD0000C5000020C60000201CB504462D
:10788000207840490978884202D0207800F07CF8BE
:107890002078032834D003DC38B101286AD11AE0FB
:1078A000042843D00F2865D154E060788DF800009B
:1078B000A0788DF80100E0788DF8020020798DF82D
:1078C000030060798DF80400A0798DF80500E07957
:1078D0008DF806004EE0207A8DF80000607A8DF871
:1078E0000100A07A8DF80200E07A8DF80300207B79
:1078F0008DF8040000208DF805008DF8060039E0B1
:10790000607B8DF80000A07B8DF80100E07B8DF896
:107910000200207C8DF80300607C8DF80400A07CC0
:107920008DF80500E07C8DF8060023E0207D8DF8C1
:107930000000607D8DF80100A07D8DF80200E07DE3
:107940008DF8030000208DF804008DF805008DF8F7
:1079500006000FE000208DF800008DF801008DF882
:1079600002008DF803008DF804008DF805008DF8F5
:10797000060000BF00BF072269468C20FFF760FCAD
:107980001CBD0000C500002001B59DF800000449A1
:107990000870012269468A20FFF752FC08BD0000EA
:1079A000C500002070B504460D462A462146002039
:1079B000FFF71CFC70BD00000120014908707047F2
:1079C000C700002010B500240AE0074A02EB840239
:1079D0009178054A32F82400FFF75AFC601C04B283
:1079E000002CF2D010BD0000301C010801B50122AE
:1079F00069469620FFF724FC08BD00002DE9FE4FE4
:107A000083464FF0000A0022164B1046590303F03C
:107A100093FD02460B46CDE9000100201249F8F71C
:107A2000A6FE06460F465846F8F72FFF8046324618
:107A30003B46F8F79CFE0446F8F734FF82464FEACF
:107A40001A408DF808004FEA1A208DF809000AF054
:107A5000FF008DF80A00032202A98620FFF7F0FB41
:107A6000BDE8FE8F00003240A8CB884101B582B04E
:107A70009DF808008DF80400BDF80A00000A8DF892
:107A80000500BDF80A00C0B28DF806004FF6FF7081
:107A9000FFF705F8032201A98220FFF7D1FB05209B
:107AA000014908700EBD0000C40000207CB50646E8
:107AB0000C4615468DF80060200A8DF80100E0B2F2
:107AC0008DF80200280A8DF80300E8B28DF8040052
:107AD000052269469420FFF7B3FB05200149087091
:107AE0007CBD0000C400002010B500221146D52046
:107AF000FFF7A6FB10BD000001B582B09DF808009D
:107B0000C007000F9DF80810C1F3400140EA810052
:107B10009DF80810C1F3800140EA41009DF808106B
:107B2000C1F3C001084301900020044908700122FC
:107B300001A98420FFF784FB0EBD0000C4000020D3
:107B400001B5012269468020FFF77AFB9DF800000D
:107B500018B901200349087002E0022001490870A9
:107B600008BD0000C40000202DE9F04105460E4686
:107B70000027FFF7D9F920B1032818D0042835D100
:107B80002AE00527012D04D0022D05D0032D09D1AF
:107B900005E040F6CE1408E040F6D31405E040F6C8
:107BA000D81402E00120BDE8F08100BF20E00427E6
:107BB000012D04D0022D05D0032D09D105E040F69A
:107BC000CF1407E040F6D41404E040F6D91401E0E5
:107BD0000120E8E700BF0BE00427012D02D140F6A9
:107BE000CF1401E00120DEE700BF01E00120DAE769
:107BF00000BF3A4631462046FFF752FB0020D2E74D
:107C000010B5044640F6CD10FFF788FA00F0F000FA
:107C100004F00F0140EA0104214640F6CD10FFF7C1
:107C200037FB10BD01B582B09DF808008DF8040047
:107C3000BDF80A00000A8DF80500BDF80A00C0B2C0
:107C40008DF806004FF6FF70FEF729FF032201A909
:107C50008320FFF7F5FA0420014908700EBD0000EB
:107C6000C400002010B500221146D220FFF7E8FA28
:107C700010BD10B500221146D120FFF7E1FA10BD6A
:107C800038B505460C4605F11200C0B28DF800006B
:107C90008DF80140022269468E20FFF7D1FA38BDE7
:107CA00010B50446FFF740F920B1032803D004289B
:107CB00008D101E000BF00BF214640F6C510FFF724
:107CC000E7FA00E000BF00BF10BD10B500F00AFFEA
:107CD00010BD00002DE9F8438046A8F102000628F7
:107CE0006BD2DFE800F0035F697596B15BA001F02D
:107CF00037FF00206249087062487F22036E6248A5
:107D000098475F4800787F2805DA00205E495C4A82
:107D10001278885403E000205B4981F87E005A48BD
:107D200040785949097840EA0126002436E057484E
:107D300000685E3030F8140040B1544800685E308E
:107D400030F814004FF6FF71884200D125E04F480B
:107D500000685E3030F81400B0421DD14B48A830A6
:107D600050F82400401C4949A83141F824004748F4
:107D700081684162022001F03DFE01F06DFD434843
:107D8000A83050F8240000903D4803783246611C2A
:107D90003FA001F0E5FE03E000BF641C032CC6DB3E
:107DA00000BF56E048A001F0DBFE032001F022FEF8
:107DB0004F4800F0C7FD4CE000E049E04DA001F065
:107DC000CFFE032001F016FE494800F0BBFD40E065
:107DD00053A001F0C5FE012001F00CFE01F03CFDB6
:107DE0002A48006890F8580010B95848057805E00E
:107DF00026480068B0F85A00801C85B2294654A075
:107E000001F0AEFEEAB221492831394800F0D6FD32
:107E10001FE055A001F0A4FE032001F0EBFD1B487C
:107E2000006890F8580010B94848077805E01748EE
:107E30000068B0F85A00801C87B2FAB213492831A2
:107E40002B4800F0BBFD04E053A001F089FE00E0E8
:107E500000BF00BF0020BDE8F88300000D0A5B52A0
:107E6000585D203C3C3C205061636B65742052653A
:107E7000636569766564203E3E3E0D0A00000000A1
:107E800008010020341C0108702D0020302F002034
:107E90005B636825645D204865616465723A2030E3
:107EA0007825303458207C2053697A653A2025643F
:107EB000206279746573207C20436F756E743A205C
:107EC00025640D0A000000000D0A5B52585D202E4B
:107ED0002E2E2054696D656F757420285265737459
:107EE000617274696E67205258290D0A0000000003
:107EF000E02C00200D0A5B52585D202121212045F5
:107F000052524F52202D20526563657074696F6E16
:107F1000204661696C6564202121210D0A00000062
:107F20000D0A5B54585D203C3C3C205061636B65FE
:107F3000742053656E74205375636365737366753F
:107F40006C6C79203E3E3E0D0A00000004000020CB
:107F50005B54585D204C656E6774683A2025642038
:107F600062797465730D0A000D0A5B54585D202117
:107F700021212054494D454F5554202D20547261E4
:107F80006E736D697373696F6E204661696C6564A9
:107F9000202121210D0A00000D0A5B4341445D2090
:107FA0004368616E6E656C204163746976697479AB
:107FB0002044657465637465640D0A00014611B957
:107FC0004FF0FF3070470248007808720020F9E750
:107FD000C00000202DE9FC4704460E4615461CB99A
:107FE0004FF0FF30BDE8FC87666060684570FFF7C2
:107FF0006CFE4FF4FA70FAF74BF992480168924818
:10800000884792A001F0ACFD91A001F0A9FDA0A0CD
:1080100001F0A6FD8EA001F0A3FDA8A1AEA001F085
:108020009FFD8849086B804707463946B2A001F09A
:1080300097FD87A001F094FD35B1012D0ED0022DE2
:1080400016D0032D28D11DE0B4A001F089FD042035
:10805000616881F835006168487720E0BBA001F0D5
:108060007FFD0120616881F835006168487716E07E
:10807000C0A001F075FD0020616881F835006168DD
:1080800048770CE0C5A001F06BFD0320616881F822
:1080900035006168487702E04FF0FF30A2E700BF8B
:1080A0006848816B00208847626892F83500654A0D
:1080B000D16B8847626802F13500624A116C8847CB
:1080C000626802F11D005F4A516C88476268906CDB
:1080D0005C4A916C88475B480021C26C0846904717
:1080E000636893F8511093F95000564B1A6D9047FE
:1080F00060684078022812D16068811C5148826D06
:10810000012090476068C11D4E48826D0220904753
:10811000606800F10C014B48826D03209047606855
:108120004078032814D1606800F111014548826D40
:1081300001209047606800F115014248826D0220DD
:108140009047606800F119013E48826D0320904716
:108150003C49C86E80473DA001F002FD9EA001F0A1
:10816000FFFCADA001F0FCFC9BA001F0F9FC6068F5
:10817000D0E912211046F8F769FB8046B149F8F7BB
:1081800046FA0746F8F7A7FBCDE900016068D0E999
:1081900012733A46ACA001F0E3FC606890F950100D
:1081A000B4A001F0DDFC7F21BAA001F0D9FC606829
:1081B000407801281ED1606890F83910BDA001F008
:1081C000CFFC606890F83A10C1A001F0C9FC60686B
:1081D00090F83B10C5A001F0C3FC606890F8251032
:1081E000C9A001F0BDFC606890F82710CDA001F097
:1081F000B7FC1BE060684078032817D1606890F8EE
:108200003C10CFA001F0ACFC606890F83D10D3A00A
:1082100001F0A6FC606890F82A10BBA001F0A0FC59
:10822000606890F82E10BFA001F09AFCD2A001F077
:1082300097FC69A001F094FCD7A001F091FC00200C
:10824000D0E60000341C01089C0000200D0A00004C
:108250003D3D3D3D3D3D3D3D3D3D3D3D3D3D3D3D4E
:108260003D3D3D3D3D3D3D3D3D3D3D3D3D3D3D3D3E
:108270003D3D3D3D3D3D3D3D3D3D3D3D3D3D3D3D2E
:108280003D3D3D3D3D3D3D3D3D3D3D3D0D0A0000FB
:108290002020202020202020202020202020535873
:1082A0003132383120526164696F20496E697469D6
:1082B000616C697A6174696F6E0D0A004669726D4E
:1082C000776172652056657273696F6E3A20313737
:1082D000303931394100000020204170706C6963F1
:1082E0006174696F6E2056657273696F6E203A20F3
:1082F00025730D0A0000000020204669726D776129
:1083000072652056657273696F6E202020203A20B6
:108310003078253034580D0A000000000D0A5B2A21
:108320005D20526164696F204D6F64653A20424C54
:10833000452028426C7565746F6F7468204C6F77A8
:1083400020456E65726779290D0A00000D0A5B2AC7
:108350005D20526164696F204D6F64653A204C4F17
:10836000524120284C6F6E672052616E6765290D5F
:108370000A0000000D0A5B2A5D20526164696F20CB
:108380004D6F64653A204746534B2028476175730B
:108390007369616E2046534B290D0A000D0A5B2A52
:1083A0005D20526164696F204D6F64653A20464CD0
:1083B0005243202846617374204C6F6E67205261CF
:1083C0006E676520436F6D6D756E69636174696F6B
:1083D0006E290D0A000000002D2D2D2D2D2D2D2D87
:1083E0002D2D2D2D2D2D2D2D2D2D2D2D2D2D2D2DBD
:1083F0002D2D2D2D2D2D2D2D2D2D2D2D2D2D2D2DAD
:108400002D2D2D2D2D2D2D2D2D2D2D2D2D2D2D2D9C
:108410002D2D2D2D0D0A0000202020202020202091
:1084200020202020202020202020436F6E666967B6
:1084300075726174696F6E2053756D6D6172790D1F
:108440000A0000000024744920205246204672652C
:108450007175656E6379202020203A20256C6C753B
:1084600020487A2028252E3166204D487A290D0A89
:10847000000000002020545820506F7765722020A3
:108480002020202020203A2025642064426D0D0AFF
:108490000000000020204275666665722053697AEC
:1084A0006520202020203A2025642062797465739D
:1084B0000D0A000020204C6F5261205346202020DE
:1084C0002020202020203A2025640D0A00000000F2
:1084D00020204C6F52612042572020202020202055
:1084E00020203A2025640D0A0000000020204C6F57
:1084F00052612043522020202020202020203A209A
:1085000025640D0A000000002020507265616D6234
:108510006C65204C656E202020203A2025640D0AD1
:108520000000000020205061796C6F6164204C6570
:108530006E20202020203A2025640D0A0000000033
:108540002020464C524320426974526174652F4288
:1085500057203A2025640D0A000000002020464CD8
:1085600052432043522020202020202020203A2047
:1085700025640D0A0000000020204D6F6465202056
:10858000202020202020202020203A20494E544521
:1085900052525550540D0A000D0A5B2A5D20535863
:1085A0003132383120496E697469616C697A61745D
:1085B000696F6E20436F6D706C657465210D0A0DD7
:1085C0000A00000010B50446FEF7B2FE2046FFF791
:1085D000F5FC002010BD000070B504460D4614B92E
:1085E0004FF0FF3070BD606880F852501A48816BC0
:1085F00000208847032D20D01FDA606890F85200D1
:1086000000EB40001549095C606880F83F10606825
:1086100090F8520000EB400010490844417860682F
:1086200080F84010606890F8520000EB40000B4961
:1086300008448178606880F84110626892F83500DB
:10864000054AD16B8847626802F13500024A116C15
:1086500088470020C6E70000341C0108DC1B010825
:1086600070B504460D4614B94FF0FF3070BD606818
:1086700080F855501A48816B00208847042D20D07F
:108680001FDA606890F8550000EB40001549095C5E
:10869000606880F83C10606890F8550000EB40007E
:1086A000104908444178606880F83D10606890F88F
:1086B000550000EB40000B4908448178606880F861
:1086C0003E10626892F83500054AD16B88476268AF
:1086D00002F13500024A116C88470020C6E700000D
:1086E000341C01080F1C010870B504460D4614B96E
:1086F0004FF0FF3070BD606880F854501A48816BAD
:1087000000208847042D20D01FDA606890F85400BC
:1087100000EB40001549095C606880F8361060681D
:1087200090F8540000EB400010490844417860681C
:1087300080F83710606890F8540000EB40000B4957
:1087400008448178606880F83810626892F83500D3
:10875000054AD16B8847626802F13500024A116C04
:1087600088470020C6E70000341C0108001C0108EF
:1087700070B504460D4614B94FF0FF3070BD606807
:1087800080F853501848816B00208847606890F843
:10879000530000EB40001549095C606880F839100F
:1087A000606890F8530000EB40001049084441789D
:1087B000606880F83A10606890F8530000EB400061
:1087C0000A4908448178606880F83B10626892F832
:1087D0003500054AD16B8847626802F13500024ACC
:1087E000116C88470020C9E7341C0108E81B010808
:1087F00070B504460D4614B94FF0FF3070BD4148C6
:10880000816B00208847626892F835003D4AD16B41
:108810008847606845706068407830B101281DD095
:10882000022834D0032866D14BE00420616881F827
:10883000350061684877626892F83500314AD16B3B
:108840008847626802F135002E4A116C88476268D9
:1088500002F11D002B4A516C88474FE001206168EE
:1088600081F8350061684877626892F83500254ADA
:10887000D16B8847626802F13500224A116C884743
:10888000626802F11D001F4A516C884736E00020E3
:10889000616881F83500012061684877626892F864
:1088A0003500184AD16B8847626802F13500154AD5
:1088B000116C8847626802F11D00124A516C8847AA
:1088C0001CE00320616881F8350001206168487769
:1088D000626892F835000B4AD16B8847626802F1F2
:1088E0003500084A116C8847626802F11D00054A8C
:1088F000516C884702E04FF0FF307FE700BF002057
:108900007CE70000341C010870B504460D4614B91C
:108910004FF0FF3070BD0A48816B002088476268C5
:1089200092F83500064AD16B884700206168C1E99A
:1089300012506268906C024A916C88470020E9E707
:10894000341C010838B504460220207061680870A4
:10895000084800231A46456D074801880088A84743
:108960000648006800900348C16D009888470020C1
:1089700038BD0000341C0108BC000020201C010888
:1089800038B504460320207002206168087008484A
:1089900000231A46456D074801880088A847064805
:1089A000006800900248C16D00988847002038BDDB
:1089B000341C0108BC000020241C0108F8B5054641
:1089C0000F4616466868407858B1012807D002283B
:1089D00003D0032807D17C2407E0FC2405E0FD2414
:1089E00003E0FC2401E07C2400BF00BFA64207DDB9
:1089F000224631460EA001F0B3F84FF0FF30F8BD2B
:108A00000120287069680870194800231A46D0F8B8
:108A100054C0184801880088E04717480068009053
:108A20001348436E31463846009A98470020E6E7DF
:108A30005B5358313238315D204552524F523A2003
:108A40007061796C6F6164202564203E206D6178CF
:108A500020256420627974657320666F72206375C7
:108A60007272656E74206D6F6465210D0A000000DE
:108A7000341C0108BE000020281C010810B5024665
:108A800010468B1E02249C40944203D84B1E0224A5
:108A90009C40001B10BD000070B504460D4601202F
:108AA0000549087001232A4621460020F8F726FCD4
:108AB00006F026FD70BD0000D4000020F8B5044685
:108AC0000D46164601200649087033462A462146BF
:108AD00000900020F8F73CFC06F012FDF8BD000005
:108AE000D400002010B5054A02210020F8F7F8FB59
:108AF000034A00210846F8F7F3FB10BDCDEE00084D
:108B0000C1EE000800BF012002F06CFBFBE710B5CE
:108B1000F9F716FE07F05EF9012801D006F074FDA2
:108B200010BD00B58FB0282105A8F7F7A3FB1421CD
:108B30006846F7F79FFB012005900004069040006F
:108B400007900120099002200C90C1030D914FF471
:108B5000E0110E9105A8F9F7F1FF08B1F9F70CF84B
:108B60000F20009002200190002002904FF48060BE
:108B700003900020049002216846F9F7B9FE08B17D
:108B8000F8F7FAFF0FB000BD7047000010B502689B
:108B90001C4B984208D0B0F1804F05D01A4B984238
:108BA00002D01A4B984203D122F070024B681A434C
:108BB000144B984208D0B0F1804F05D0124B984228
:108BC00002D0124B984203D122F44072CB681A4370
:108BD00022F080034C6943EA040202608B68C3629E
:108BE0000B688362074B984201D10B690363012331
:108BF0004361036903F001031BB1036923F001031F
:108C0000036110BD002C014000040040000800403A
:108C100030B501F01F05012404FA05F3046A9C43F2
:108C20000462046A01F01F0502FA05F52C43046290
:108C300030BD70B505466C6A606AA84207D1012054
:108C40002077A86918BB012084F83E001FE0A06AC5
:108C5000A84207D102202077A869C0B901213F208E
:108C6000015514E0E06AA84207D104202077A869E2
:108C700068B901214020015509E0206BA84206D1C6
:108C800008202077A86910B901214120015520460C
:108C9000FBF7C2F90020207770BD70B505466C6AFD
:108CA000606AA84202D10120207710E0A06AA842A1
:108CB00002D1022020770AE0E06AA84202D1042013
:108CC000207704E0206BA84201D1082020772046BD
:108CD000FBF7B4F90020207770BD70B505466C6ACB
:108CE000606AA84204D10120207784F83E001DE08C
:108CF000A06AA84205D10220207701213F2001551A
:108D000014E0E06AA84205D1042020770121402028
:108D100001550BE0206BA84205D1082020770121E6
:108D20004120015502E0012084F83D002046FBF778
:108D30008FF80020207770BD30B50C46816821F493
:108D40007F4142EA032525432943816030BD0A461D
:108D5000816821F0700142F0070319438160704778
:108D600030B5026A056A25F0010505624368846929
:108D700024F0700424F003040D682C4322F0020256
:108D80008D682A430D4DA84206D100BF22F008028B
:108D9000CD682A4322F00402084DA84207D123F4EB
:108DA000807323F400734D692B438D692B4343601B
:108DB00084614D684563026230BD0000002C0140B3
:108DC00030B5026A056A25F01005056243688469BA
:108DD00024F4E04424F440740D6844EA052422F0AD
:108DE00020028D6842EA05120E4DA84207D100BF4D
:108DF00022F08002CD6842EA051222F04002094DBD
:108E0000A84209D123F4806323F400634D6943EA47
:108E100085038D6943EA8503436084614D688563FA
:108E2000026230BD002C014030B5026A056A25F4AB
:108E3000807505624368C46924F0700424F003045B
:108E40000D682C4322F400728D6842EA05220F4D12
:108E5000A84207D100BF22F40062CD6842EA052291
:108E600022F48062094DA84209D123F4805323F4EF
:108E700000534D6943EA05138D6943EA05134360C6
:108E8000C4614D68C563026230BD0000002C014022
:108E900030B5036A056A25F4805505624468C269E5
:108EA00022F4E04222F440720D6842EA052223F4E3
:108EB00000538D6843EA0533064DA84204D124F4DB
:108EC00080444D6944EA85144460C2614D6805647C
:108ED000036230BD002C014030B50B461446026AD7
:108EE000056A25F001050562816921F0F00141EA7A
:108EF000041122F00A021A438161026230BD30B5CA
:108F00000B461446026A056A25F010050562816960
:108F100021F4704141EA043122F0A00242EA031236
:108F20008161026230BD000070B5054602F090F923
:108F30000A4A00210A4802F04CFA0A490860002255
:108F40000A21022002F0F2F90649486002F0CCF949
:108F500002F039FA044602F098FA70BD944C010808
:108F6000698F0008E82F002002F058F90446F7F74F
:108F70008CFC804600222D4BF7F7F9FB0646F7F7ED
:108F800091FC8246002002F02DF902F03AF9834666
:108F900027480068C06840F0100025490968C8608B
:108FA000F8F788FA00F1080421462248FCF716FB7E
:108FB000012000F011FC192000F08EFC40F6B830C2
:108FC00000F012FD002000F015FD00F045FC02F05D
:108FD00018F9054600BF28E0D3441648FCF7D6FB35
:108FE000012002F0FFF802F00CF90646701B0E2873
:108FF0001AD31048006890F8580018B90E48007845
:10900000841C05E00B480068B0F85A00801C84B24C
:1090100000232246074928310120F8F723FA0E35AC
:1090200004488168016200BF00BFD5E700408F405F
:1090300080050020302F00200400002070B5054678
:109040006C6A0020E085E0842046FBF71BFA70BDC7
:1090500070B506460025746A20684069C0F3C015E3
:1090600094F84100212805D125B10020E084204654
:1090700000F0FBF820684069C0F3801594F84200C6
:10908000222805D125B10020E085204600F0A7F870
:10909000606C40F0100060642046FBF7F3F970BD8F
:1090A00070B505466C6A2868006800F0200000284A
:1090B00042D1E08500BF00BF21680C3151E8001F9C
:1090C00021F4807021680C3141E80002002AF3D1BC
:1090D00000BF00BF00BF2168143151E8001F21F01C
:1090E00001002168143141E80002002AF3D100BFD9
:1090F00000BF00BF2168143151E8001F21F040007B
:109100002168143141E80002002AF3D100BF202079
:1091100084F84200206B01280ED100BF00BF2168F7
:109120000C3151E8001F21F0100021680C3141E89A
:109130000002002AF3D100BF00206063206B0128E9
:1091400004D1A18D2046FBF757F902E02046FBF73A
:1091500039FC70BD70B505466C6A01206063206BF8
:10916000012805D1A08D41082046FBF745F902E012
:109170002046FBF741FC70BD70B505466C6A286857
:10918000006800F02000F8B90020E08400BF00BFB4
:109190002168143151E8001F21F08000216814314A
:1091A00041E80002002AF3D100BF00BF00BF2168E0
:1091B0000C3151E8001F41F0400021680C3141E8BA
:1091C0000002002AF3D102E02046FBF7F1FC70BD5B
:1091D00070B50446656A2846FBF704FD70BD00BF04
:1091E00000BF02680C3252E8002F22F4907102682E
:1091F0000C3242E80013002BF3D100BF00BF00BFC8
:109200000268143252E8002F22F001010268143281
:1092100042E80013002BF3D100BF016B01290ED1EE
:1092200000BF00BF02680C3252E8002F22F010018C
:1092300002680C3242E80013002BF3D100BF20215A
:1092400080F8421000210163704710B50446206881
:10925000C06820F040002168C860202084F84100E8
:109260002046FBF7A5FC002010BD00BF00BF026830
:109270000C3252E8002F22F0C00102680C3242E8A2
:109280000013002BF3D100BF202180F8411070475C
:109290000146074A0868904201D100207047054AFC
:1092A0000868904201D10120F8E70320F6E70000AA
:1092B0000044004000380140F8B5044694F84200EC
:1092C000222875D1A068B0F5805F0CD1206950B913
:1092D0000025A66A20684068C0F308003080A06AB4
:1092E000801CA06215E0A56A0026A068B0F5805F2A
:1092F00003D0A06828B9206918B920684068287090
:1093000004E02068406800F07F002870A06A401CDC
:10931000A062E08D401E80B2E085002846D1206822
:10932000C06820F020002168C8602068C06820F470
:1093300080702168C8602068406920F001002168C1
:109340004861202084F8420000206063206B0128DF
:1093500026D10020206300BF00BF21680C3151E8F6
:10936000001F21F0100021680C3141E80002002AA2
:10937000F3D100BF2068006800F0100010280AD167
:1093800000BF0020009020680068009020684068BE
:10939000009000BF00BFA18D2046FBF72DF802E032
:1093A0002046FBF70FFB0020F8BD01E00020FBE7A3
:1093B0000220F9E770B504462168096921F440519B
:1093C000E2681143226811612269A1681143626950
:1093D00041EA02052168C96841F20C6291432943C0
:1093E0002268D1602168496921F44071A269114362
:1093F000226851612D4A2168914202D1F9F754FB4C
:1094000001E0F9F741FB00EBC00101EB00116268DC
:109410009200B1FBF2F100EBC00202EB00126368B4
:109420009B00B2FBF3F26423B2FBF3F202EBC20344
:1094300003EB0212A1EB8201322202EB0111642242
:10944000B1FBF2F101F0F00100EBC00202EB0012FF
:1094500063689B00B2FBF3F26423B2FBF3F201EB0F
:10946000021200EBC00101EB001163689B00B1FB2D
:10947000F3F100EBC00303EB00136668B600B3FB27
:10948000F6F36426B3FBF6F303EBC30606EB031314
:10949000A1EB8301322303EB01116423B1FBF3F150
:1094A00001F00F0111442268916070BD0038014045
:1094B00077B581B0044615460298A062A5850020C4
:1094C0006064222084F842002848E16B88622848C2
:1094D000E16BC8622748E16B08630020E16B4863D9
:1094E00002AE32682368191D2B46E06BF8F782FE46
:1094F00000BF00200090206800680090206840684D
:10950000009000BF00BF206970B100BF00BF21689C
:109510000C3151E8001F41F4807021680C3141E8A2
:109520000002002AF3D100BF00BF00BF2168143140
:1095300051E8001F41F001002168143141E80002A8
:10954000002AF3D100BF00BF00BF2168143151E8E9
:10955000001F41F040002168143141E80002002A58
:10956000F3D100BF002004B070BD0000A19000083E
:109570005591000851900008014691F841002128BA
:1095800028D18868B0F5805F0BD1086948B90A6AAC
:109590001088C0F308000B685860086A801C0862D5
:1095A00005E00B6A581C086218780B685860C88C74
:1095B000401E80B2C88458B90868C06820F0800096
:1095C0000B68D8600868C06840F040000B68D8603D
:1095D000002070470220FCE72DE9F84304460D46C1
:1095E00017469846089E31E0701C70B3F9F7A2F850
:1095F000A0EB0800B04200D816B90320BDE8F883FC
:109600002068C06800F00400F8B1802D1ED0402D05
:109610001CD020680068C0F3C000B0B100BF0020BB
:10962000009020680068009020684068009000BFAB
:1096300000BF2046FFF7D3FD0820606400BF002074
:1096400084F8400000BF0120D8E7FFE720680068E9
:109650002840A84201D1012000E00020B842C3D038
:109660000020CBE710B50248FAF726FF10BD000036
:109670003805002010B50348FAF71EFF014800F036
:109680005BF810BD8005002010B5044604B910BD7C
:109690001E492068884200D0F9E72046FAF7ADFE5F
:1096A0001B4800684068C0F1FF001A49087008466E
:1096B000007800281FDD08460078FF281BDA0846DE
:1096C000017815A000F04CFA4FF4007311480278AD
:1096D00015492046FBF7AAF914A000F041FA1448F6
:1096E000007840B90B4802780F491248F6F7A9FDF7
:1096F00001200F490870FF210B48F6F7BBFDFF2240
:1097000009492046FBF748F900BFC0E70044004084
:10971000C8050020040000205B55415254322052FD
:10972000583A25645D200000380300200D0A00002F
:10973000050000203704002038B5044604B938BDC0
:109740000C492068884212D120680068C0F30010DC
:1097500068B100BF00200090206800680090206879
:109760004068009000BF00BF2046FFF78DFF00BF9C
:10977000E5E700000044004000BFFEE710B5002010
:10978000F7F778FD0C210C48FAF7B2FD00200B49E1
:1097900008700B48006830B10948006800F090FF7D
:1097A0000020074908600020064908800649087023
:1097B000F7F74CFD10BD0000AC020020DF000020D8
:1097C000D8000020DC000020DE00002001480078E6
:1097D00070470000E000002070B5044614B1B4F5F5
:1097E000806F01DD012070BD1748007808B1FFF7D8
:1097F000C5FF164804800088401C00EB4000C500EF
:10980000A80001F071F8124908600846006820B904
:1098100000200E4908800120E5E7002005E0002136
:109820000B4A126842F82010401CA842F7D30120CE
:109830000549087007480068406C40F4004005493D
:10984000096848640020CEE7DE000020DC0000202C
:10985000D8000020AC02002010B5F8F76BFF0149DA
:10986000886010BDE000002010B51748007810B1E6
:109870001648006800B910BD1548007800B1FAE735
:109880001448008800EB40001049096801EB4014BF
:10989000002004E0002144F82010411CC8B2182820
:1098A000F8DB01200A4908700A480088401C00EBD8
:1098B00040004FF6FF7101EAC00204480168002031
:1098C000F7F7ACFC00BFD6E7DE000020D800002090
:1098D000DF000020DC000020642800DD6420014956
:1098E00008737047E0000020F0B504460D46234998
:1098F000097831B1224909888C4202DA2149096884
:1099000001B9F0BD04EB44011E4E366806EB411070
:1099100000210CE0C1F107070126BE4016400EB140
:10992000392600E01C2640F821604E1CF1B20829BF
:10993000F0DB08210CE0C1F10F070126BE402E40EC
:109940000EB1392600E01C2640F821604E1CF1B211
:109950001029F0DB10210CE0C1F117070126BE40F1
:109960001E400EB1392600E01C2640F821604E1C36
:10997000F1B21829F0DB00BFC3E70000DE000020D1
:10998000DC000020D80000202DE9F04304460D46FD
:1099900090461248007810B11148006808B9BDE837
:1099A000F0831048007B6043642190FBF1F000F0ED
:1099B000FF090C48007B684390FBF1F0C7B20948EF
:1099C000007B00FB08F090FBF1F0C6B233463A464C
:1099D00049460020FFF788FF00BFE0E7DE000020D7
:1099E000D8000020E0000020014908607047000016
:1099F000F00000200149087070470000E0000020DE
:109A00002DE9FC4104465148007810B150480068E7
:109A100008B9BDE8FC814F48007800B1F9E74E482D
:109A20004068201AB0F5967F00D2F2E74A480078E5
:109A3000012806D048480078022802D0464800781D
:109A400048B945488068201A44490968884202D9C3
:109A50000320414908704FF49670B4FBF0F000F019
:109A60000105002600273C4800783B494978884298
:109A700005D0012601273848007837494870364814
:109A80008078A8420ED034480078012807D03248A8
:109A90000078022803D030480078042800D101263D
:109AA0002D48857006B9B4E72B48446000780190D2
:109AB0002948807800909DF8040030B900231A46A8
:109AC00019461846FFF710FF3BE09DF804000128F7
:109AD00003D09DF8040002280FD19DF8000028B1A2
:109AE0000022FF211046FFF74FFF2AE000231A460D
:109AF00019461846FFF7F8FE23E09DF804000328F6
:109B000005D100221146FF20FFF73EFF19E09DF826
:109B1000040004280FD19DF8000028B10022B421D0
:109B2000FF20FFF731FF0CE000231A4619461846C4
:109B3000FFF7DAFE05E000231A4619461846FFF73C
:109B4000D3FEFFF791FE00BF63E70000DE000020B8
:109B5000D8000020DF000020E0000020F0000020FE
:109B60000FB4054B10B503A9044A029800F0A6F9FA
:109B700010BC5DF814FB0000A5A600082001002021
:109B80000FB47CB50C0009AD01D0611E00E00021CE
:109B9000CDE90001064B6A462946089800F08EF987
:109BA000002C02D0009A002111707CBC5DF814FBDF
:109BB000C3A50008490050EAC12018BF04204A0D7F
:109BC00018BF40F0010040F2FF72B2EB515F08BFD6
:109BD00040F00200012808BF0520704702480068D5
:109BE000C0F30220704700000CED00E010B5002823
:109BF00004DB0A07130E054A135406E00A07140E85
:109C0000034A00F00F031B1FD45410BD00E400E012
:109C100018ED00E0004870472C010020EFF30580AC
:109C200070472DE9F0414F1E00EBC7010446D1E912
:109C3000000115461E4637F006020DD02A4633466F
:109C4000F6F723FD7F1E04EBC703D3E90023F6F7E5
:109C5000BEFF37F00602F1D1022F25D0042F13D01A
:109C6000062F18BFBDE8F0812A463346F6F70DFDF2
:109C7000D4E90A23F6F7ABFF2A463346F6F705FD8B
:109C8000D4E90823F6F7A3FF2A463346F6F7FDFC8E
:109C9000D4E90623F6F79BFF2A463346F6F7F5FC90
:109CA000D4E90423F6F793FF2A463346F6F7EDFC92
:109CB000D4E90223F6F78BFF2A463346F6F7E5FC94
:109CC000D4E90023BDE8F041F6F781BF0022134636
:109CD00010460149F6F74BBD0000F03FF6F777BF9D
:109CE0000022134610461146F6F741BD40F20132FC
:109CF00000204FF0E041F7F711B80000024A0020C1
:109D00001107F7F70BB8000001FDFFFF02E008C8DC
:109D1000121F08C1002AFAD170477047002001E0E5
:109D200001C1121F002AFBD17047000001490860E1
:109D3000704700002C0100202DE9FF5F82B0002158
:109D4000DDE90430020DDDF840B0034318D044F6DD
:109D50001050A2F2FF3242431514119801281FD06F
:109D6000A5EB0B00401C5FEA000A4FF000064E4FC7
:109D7000DFF83891B046504615D5CAF1000413E01B
:109D8000119801244AA3012801D16FEA0B0102981E
:109D9000119AC0E90031C0E9024206B0BDE8F09F67
:109DA000CBF10000DFE704460021404A491842EBAE
:109DB0000450CDE9001012E0E00707D032463B46E0
:109DC00040464946F6F761FC8046894632463B46A6
:109DD00010461946F6F759FC06460F466410002C4B
:109DE000EAD1DDE90401DDE90023BAF1000F06DA6A
:109DF000F6F74BFC42464B46F6F747FC05E0F6F714
:109E0000B6FC42464B46F6F7B2FC04460E4600222C
:109E1000284BF6F7B3FF03D84FF0FF30014607E0B9
:109E20000022254B20463146F6F7D1FEF6F78DFF8E
:109E3000102409E0002C0ADB0A220023F6F7C0F9FF
:109E4000039B30321A55641E50EA0102F2D1641CA1
:109E5000039AC4F111031444119A012A03D0012278
:109E600008430DD10AE0084304D000204FF0110B45
:109E7000119072E7A3EB0B056D1E0DE05B4504DD51
:109E80004FF0000205F1010504E003DA4FF0000293
:109E9000A5F10105002AECD002981199C0E9023120
:109EA000C0E9004579E70000000014400000F03FE1
:109EB000300000000000F0430000E03F2DE9FF4FBC
:109EC00095B09A46884606460025EEE1252877D1CA
:109ED00000242746F94A0121039400E0044316F8C0
:109EE000013F203B01FA03F01042F7D130782A28D5
:109EF00011D06FF02F033078A0F13002092A16D864
:109F0000039A44F0020402EB820203EB4202104483
:109F1000761C0390EFE758F8042B0392002A03DA2B
:109F2000504244F40054039044F00204761C30780C
:109F30002E2816D116F8010F44F004042A280DD05B
:109F40006FF02F023078A0F13003092B09D807EB0E
:109F5000870302EB4303C718761CF3E758F8047B2A
:109F6000761C30786C280FD006DC4C2817D0682877
:109F70000DD06A2814D104E0742810D07A280FD1AB
:109F80000DE044F400140AE044F4801401E044F4C9
:109F900040147278824202D104F58014761C761C3B
:109FA000307866280BD013DC582877D009DC0028DD
:109FB00075D04528F6D04628F4D047281AD193E129
:109FC00018E0632835D0642879D0652812D18BE158
:109FD000702873D008DC6728F1D069286FD06E280C
:109FE0000DD06F2806D1ACE073282CD0752874D022
:109FF000782853D05246179990476D1C54E1C4F30A
:10A000000250022809D003280DD0D8F800100428E7
:10A010000DD00D6008F1040846E1D8F80010EA17E9
:10A02000C1E90052F6E7D8F800100D80F2E70D7094
:10A03000F0E718F8041B8DF8001000208DF80100DF
:10A04000EB46012003E058F804BB4FF0FF306107F6
:10A050004FF0000102D40DE009F101018946B94237
:10A060000FDA8145F8DB1BF809100029F4D108E06C
:10A0700009F1010189468142FADB1BF80910002928
:10A08000F6D103985346A0EB090721463846179AA4
:10A0900000F080FA284400EB090507E044E008E1FD
:10A0A0000DE01BF8010B524617999047B9F10109D1
:10A0B000F7D2534621463846179AF2E039E00A2192
:10A0C000C4F302524FF0000B0091022A06D058F858
:10A0D000040BC117032A09D00AE023E008F10700A6
:10A0E00020F00702F2E80201904605E000B2C11735
:10A0F000042A01D140B2C117002906DA0A4600211C
:10A10000404261EB02012D2202E0220504D52B2200
:10A110008DF80420012203E0E20701D02022F7E7B6
:10A12000914657E00A2100E010214FF0000B00910A
:10A130000BE010214FF0000B44F0040408270091BD
:10A1400003E008204FF0000B0090C4F30252022AF3
:10A1500005D058F8040B0021032A08D008E008F1C4
:10A16000070020F00702F2E80201904603E080B207
:10A17000042A00D1C0B24FF0000922072AD5327854
:10A18000702A07D0DDF800C08CF0100C5CEA0B0CD4
:10A1900005D00EE040228DF80420012208E050EAAC
:10A1A000010306D030238DF804308DF805200222FB
:10A1B0009146009B83F0080353EA0B030AD150EA4F
:10A1C000010201D1620705D530228DF804204FF03D
:10A1D00001097F1E3278582A04D039A20C920CAAA9
:10A1E00002920BE03BA2F9E75B46009AF5F7E8FF25
:10A1F0000C9B9B5C029A521E0292137050EA010261
:10A20000F2D1029804A9081A00F1200B600702D5C8
:10A2100024F4803400E001275F4502DDA7EB0B004A
:10A2200000E0002000EB0B01009003984944401A25
:10A230000390E00306D453462146179A039800F092
:10A24000A9F90544002706E001A85246C05D179908
:10A2500090476D1C7F1C4F45F6DBE0030CD5534641
:10A260002146179A039800F095F9054404E0302040
:10A270005246179990476D1C0099481E009000297E
:10A28000F5DC08E00298029952460078491C0291D8
:10A29000179990476D1CBBF10001ABF1010BF1DC8C
:10A2A0005BE100F065F90544761C307800287FF406
:10A2B0000DAE19B02846BDE8F08F00000928010056
:10A2C000303132333435363738396162636465662C
:10A2D00000000000303132333435363738394142EE
:10A2E0004344454600000000600700D4062708F1FB
:10A2F000070020F00700F0E80223804603F0004C3E
:10A300005FEA0C0001D097A009E0200501D596A0D6
:10A3100005E0E00701D095A001E0AFF24C001390FA
:10A32000307823F0004365280CD006DC452809D09E
:10A3300046281DD047287FD13BE0662818D06728E3
:10A340007AD136E00021112F01DB112000E0781CCA
:10A35000CDE9000104A90CA8FFF7EEFCDDE90D0131
:10A360000C9A4FF0000B07F10109109200914EE09A
:10A370004FF000400097CDE9011004A90CA8FFF7A9
:10A38000DBFCDDE90D020C9B0F994FF0000B9146B1
:10A390001093009211B9791C00EB0109B7EB090089
:10A3A00003D4C0F1FF3B07F10109A9EB07000190BD
:10A3B00042E0012F00DA01270021112F01DD1120D9
:10A3C00000E03846CDE9000104A90CA8FFF7B4FC71
:10A3D000DDE90D010C9A00914FF0000BB946109287
:10A3E00021070FD4009A4A4503DA914601E0A9F10A
:10A3F0000109B9F1010F05DD109AA9F10101515CC4
:10A400003029F4D0B84202DA10F1040F03DA012146
:10A41000CDE9011010E0002803DC8344A9EB000122
:10A4200002E0411C494500DD8946A0EB0B00401CC1
:10A4300001904FF000400290200705D40198484554
:10A4400002DB4FF0FF30019000208DF84B000298A6
:10A450000DF14B07B0F1004F25D002200C902B20BE
:10A460000D90029800280CDA404202902D200D90A9
:10A4700007E00A210298F6F74BFA3031029007F80C
:10A48000011D0C99481E0C900029F2DC029800284E
:10A49000EFD1791E0D980870307800F0200040F060
:10A4A000450007F8020D11A8C01BC01D02901398AB
:10A4B000007800B1012000EB0901019801EBE07187
:10A4C000029801440398401A401E0390E00306D40A
:10A4D00053462146179A039800F05CF805441398F8
:10A4E000007818B15246179990476D1CE00323D5A8
:10A4F00053462146179A039800F04CF805441BE098
:10A50000BBF1000F07DB0098584504DD1098179940
:10A5100010F80B0001E0179930205246904701983F
:10A520000BF1010B401E05F10105019004D12E2015
:10A530005246179990476D1CB9F10001A9F1010924
:10A54000DEDC05E017F8010B5246179990476D1CA9
:10A550000299481E02900029F4DC53462146179ABE
:10A5600003989EE62D0000002B0000002000000054
:10A570002DE9F041044600251E461746880404D400
:10A5800005E039462020B0476D1C641EF9D52846E9
:10A59000BDE8F0812DE9F041044600251E469046B5
:10A5A000C80301D5302700E02027880404D505E042
:10A5B00041463846B0476D1C641EF9D52846BDE8B3
:10A5C000F0814A68002A06D00A68531C0B6010709C
:10A5D0004868401E486070472DE9F04106460F4626
:10A5E00014461D460EB104B10DB9BDE8F081681ED8
:10A5F000B84201DD384600E0681E804642463146DA
:10A600002046F5F742FE002004F8080000BFECE702
:10A610002DE9F04707463E4656B900BF502080F36B
:10A620001188BFF34F8FBFF36F8F00BF00BFFEE7EE
:10A6300017480068864201D1002426E004F0AEFCF1
:10A6400075691448D0F800801348D0F8009004F0E1
:10A65000CFFC454501D04D4501D1022415E00F48FE
:10A6600085420BD1B06A38B996F85800012801D15B
:10A6700002240AE0032408E0022406E00848854298
:10A6800000D00DB9042400E001242046BDE8F08785
:10A69000180000201C00002020000020600B00207B
:10A6A0004C0B002073B50D460020F6F7CBFE044698
:10A6B0004FF0FF3301226946FAF7B8F900987CBDE4
:10A6C00010B5002821D0114B0022001F196803E0AB
:10A6D000814203D80A4649680029F9D152B113686A
:10A6E000841A9C4204D1006818441060104602E0AD
:10A6F000506000E0186039B102680B1A934203D130
:10A700000B681A4402604968416010BD24010020B2
:10A71000014611B1012904D101E003A0704705A051
:10A72000FCE706A0FAE700005641524941424C4579
:10A73000000000004649584544000000554E4B4E6D
:10A740004F574E00014631B1012906D0022906D0EB
:10A75000032908D105E005A0704705A0FCE706A085
:10A76000FAE707A0F8E708A0F6E70000424C45002A
:10A770004C4F5241000000004746534B0000000080
:10A78000464C524300000000554E4B4E4F574E0072
:10A790000146012905DB4FF6FE70814201DC0120F4
:10A7A00070470020FCE70146862914D008DC042904
:10A7B0000DD028290CD045290BD0692910D109E0EA
:10A7C000AA2909D0C72908D0EB2909D106E000BF82
:10A7D00000BF00BF00BF00BF00BF00BF0120704727
:10A7E0000020FCE70146862925D00EDC4C291DD02F
:10A7F00006DC042918D0282917D0452922D116E0D3
:10A80000692916D070291DD112E0C72917D006DC9E
:10A810008D290FD0AA2910D0B12913D10CE0CE294F
:10A820000CD0EF290ED10BE000BF00BF00BF00BF6E
:10A8300000BF00BF00BF00BF00BF00BF00BF00BF20
:10A84000012070470020FCE701460A2908D018299A
:10A8500005D0262902D0342904D100BF00BF00BF93
:10A86000012070470020FCE7014601F00F0090B97D
:10A870000811401F08280ED2DFE800F00405060783
:10A8800008090A0B00BF00BF00BF00BF00BF00BF28
:10A8900000BF012070470020FCE7014621B11029CC
:10A8A00003D0202904D101E000BF00BF0120704780
:10A8B0000020FCE7F7F750FFFEF733F9FBF73EFC0B
:10A8C000FBF7E2FBFBF724FDFBF7DEFCFBF7FEFCEE
:10A8D000FBF788FDFBF7A6FD00F0A4FCFBF716FCD8
:10A8E00000F0D2FC00BFFEE7F0B50B30154D20F0B4
:10A8F00007010024144A0FE003688B420BD38B42FC
:10A9000005D95E1A43184768C3E9006700E0436849
:10A91000136002C004E0021D10680028ECD120463C
:10A92000002802D1286808B10020F0BD064A074877
:10A930001060074A121A22F00702C0E90024012021
:10A940002860D7E728010020240100201C300020C7
:10A95000183200202DE9F04FA5B005460E461746E7
:10A96000002024902390229024AA01213846F7F752
:10A97000A5F9804623AA02213846F7F79FF98146B8
:10A9800022AA03213846F7F799F9824620211AA80E
:10A99000F5F770FC202112A8F5F76CFC20210AA81D
:10A9A000F5F768FCB8F1000F05D020231AAA40463D
:10A9B0002499FFF711FEB9F1000F05D0202312AA48
:10A9C00048462399FFF708FEBAF1000F05D020236F
:10A9D0000AAA50462299FFF7FFFDFEA11AA8F5F733
:10A9E00076FCC0B9FD48F5F75CFCFD490968884272
:10A9F00002D80020FA490860F94BF84A3146284647
:10AA000000F061FD044614B90020F54908602046B5
:10AA100025B0BDE8F08FF3A11AA8F5F758FC98B956
:10AA2000F6F748FD04460068401C2060F6F742FD3A
:10AA3000044638222146ED48FBF76CFFECA2314674
:10AA40002846FFF79DF891E3F1A11AA8F5F73FFC1E
:10AA500068B9F6F72FFD044638222146E348FBF794
:10AA600045FFECA231462846FFF78AF87EE3F2A1C3
:10AA70001AA8F5F72CFC78B9F6F734FDF6F71AFDAD
:10AA800000F108042146EE48FAF7A8FDEDA2314690
:10AA90002846FFF775F869E3F3A11AA8F5F717FC44
:10AAA00000284AD1CBA112A8F5F711FC30B9F04A21
:10AAB00031462846FFF764F80020A9E79DF84800D2
:10AAC00000282CD0EBA112A8F5F701FC68B90020F2
:10AAD000DB49096881F85800D948FBF75BFAE8A21E
:10AAE00031462846FFF74CF840E3EDA112A8F5F7F0
:10AAF000EEFB68B90120D249096881F85800D048B6
:10AB0000FBF748FAE8A231462846FFF739F82DE36B
:10AB100012ABECA231462846FFF732F826E3C849CB
:10AB2000096891F85800FFF7F3FD04462346EBA2AD
:10AB300031462846FFF724F818E3EEA11AA8F5F7E6
:10AB4000C6FB002853D19DF84800D0B300200990DF
:10AB5000002209A912A8F5F7C9FC044612A9099810
:10AB6000884206D112ABE6A231462846FFF708F824
:10AB700026E00CB1752C08D975202346E74A3146EA
:10AB800000902846FEF7FCFF1AE0AD490968A1F8DD
:10AB90005A40AB48FBF7FEF9A9480068B0F85A10D4
:10ABA000A7480068B0F85A00801CCDE90001A4480D
:10ABB0000068B0F85A30DA4A31462846FEF7E0FF1E
:10ABC000D4E2FFE79E480068B0F85A109C4800683D
:10ABD000B0F85A00801CCDE9000199480068B0F82F
:10ABE0005A30D04A31462846FEF7CAFFBEE2CEA10F
:10ABF0001AA8F5F76CFB90BB0120CC494968087096
:10AC00008F48006890F8580010B101280AD102E07E
:10AC1000C74804780DE08A480068B0F85A00801CE4
:10AC200084B206E0C3A231462846FEF7A9FF002001
:10AC3000EEE600BFE2B282492831BC48FDF7BEFE15
:10AC40007F48FAF717FF7E48FBF7A4F90020FEF7CC
:10AC5000D1FEC1A231462846FEF792FF86E2FFE709
:10AC6000C4A11AA8F5F733FBA8B90220AF49496877
:10AC70000870AE48FDF784FE7148FAF7FBFE704895
:10AC8000FBF788F90020FEF7B5FEBBA23146284647
:10AC9000FEF776FF6AE2C1A11AA8F5F718FB48B1E2
:10ACA000C0A11AA8F5F713FB20B1C0A11AA8F5F7A7
:10ACB0000EFBF0B99DF86C00A0F131049DF848003E
:10ACC00050B15F4909685E3101EB440033462A46C2
:10ACD00012A904F079F80BE0594800685E3030F8AA
:10ACE0001400631CB3A2314600902846FEF748FFCB
:10ACF0003CE2B7A11AA8F5F7EAFAB0B99DF8480006
:10AD000098B94F480068B0F862004D490968B1F839
:10AD10006010CDE900104A480068B0F85E30AEA27D
:10AD200031462846FEF72CFF20E2BBA11AA8F5F712
:10AD3000CEFA00284DD19DF8480090B97B48406874
:10AD400048B17A48406890F95030B5A2314628465B
:10AD5000FEF716FF0AE2B8A231462846FEF710FFBA
:10AD600004E200200990002209A912A8F5F786FB49
:10AD7000044612A90998884206D112ABB9A23146FD
:10AD80002846FEF7FDFEA1E114F1120F01DB0D2CA8
:10AD90000BDD0D206FF011012346B9A2CDE90010A3
:10ADA00031462846FEF7ECFE90E14FFA84FB5F48FF
:10ADB000406868B15D48406880F850B05B4B5B68A4
:10ADC00093F85110594B5B6893F95000B84B71E1FF
:10ADD00075E17CE168656C7000000000C83C01080A
:10ADE0000C010020736176650000000000F8000887
:10ADF000436F6E66696775726174696F6E20736107
:10AE000076656420746F20466C617368210D0A00BA
:10AE100067657400436F6E66696775726174696F08
:10AE20006E206C6F616465642066726F6D20466C85
:10AE30006173680D0A00000072657365740000009C
:10AE4000302F0020436F6E66696775726174696F99
:10AE50006E20726573657420746F20646566617519
:10AE60006C7473210D0A00006D6F646500000000B2
:10AE7000545401085641524941424C4500000000DB
:10AE80004461746120666F726D6174207365742013
:10AE9000746F3A205641524941424C450D0A000018
:10AEA00046495845440000004461746120666F7251
:10AEB0006D61742073657420746F3A20464958455B
:10AEC000440D0A00496E76616C696420666F726D8C
:10AED00061743A2025730D0A0000000043757272F8
:10AEE000656E7420666F726D61743A2025730D0A69
:10AEF0000000000066697865646C656E0000000003
:10AF0000496E76616C6964206C656E677468207642
:10AF1000616C75653A2025730D0A0000A454010880
:10AF2000E85301087853010874780000E02C0020F1
:10AF30000400002043616E6E6F74207472616E7342
:10AF40006D69743A20696E76616C696420666F720F
:10AF50006D61740D0A0000005472616E736D697446
:10AF600074696E67207061636B65742E2E2E0D0AF6
:10AF700000000000727800005374617274696E679B
:10AF800020636F6E74696E756F757320726563658B
:10AF90006976652E2E2E0D0A000000007278696415
:10AFA00031000000727869643200000072786964D0
:10AFB0003300000043757272656E74205258494424
:10AFC00025643A203078253034580D0A00000000FE
:10AFD00072786964000000005258204944733A0DA9
:10AFE0000A202052584944313A20307825303458CC
:10AFF0000D0A202052584944323A20307825303406
:10B00000580D0A202052584944333A2030782530D0
:10B0100034580D0A00000000706F77657200000060
:10B0200043757272656E7420706F7765723A202571
:10B03000642064426D0D0A0043757272656E74205F
:10B04000706F7765723A2028726164696F206E6F45
:10B050007420696E697469616C697A6564290D0A86
:10B0600000000000496E76616C696420706F77653E
:10B07000722076616C75653A2025730D0A00000018
:10B08000506F776572206F7574206F662072616EE5
:10B0900067653A20256C642064426D202876616CD7
:10B0A00069643A2025642E2E2564290D0A000000CB
:10B0B000341C01081A6D90472D48FAF76BFF5B4668
:10B0C0002CA231462846FEF75BFD00BF4EE02FA1C3
:10B0D0001AA8F5F7FCF8E8BB2E4949684878FFF74D
:10B0E00031FB04462249096891F85800FFF710FB2C
:10B0F0008346284840680078012801D126A200E054
:10B1000026A22448406890F9500019490968B1F80E
:10B110006210CDE90742CDE9051015480068B0F886
:10B12000601013480068B0F85E3011480068B0F84D
:10B130005C200F480068B0F85A00801CCDE902235B
:10B14000049101900A480068B0F85A005B46144A1E
:10B15000314600E004E000902846FEF711FD05E0CE
:10B160001AAB10A231462846FEF70AFD00204FE434
:10B17000302F0020506F7765722073657420746FD4
:10B180002025642064426D0D0A00000073686F770B
:10B1900000000000E02C002054580000525800002D
:10B1A000D44F0108496E76616C696420636F6D6DE0
:10B1B000616E643A2025730D0A55736520276D7200
:10B1C00031362068656C702720666F722061766169
:10B1D000696C61626C6520636F6D6D616E64730D87
:10B1E0000A00000070B50546FEF718FD10B16FF0BB
:10B1F000050404E0002415B1284603F0F5FF2046BD
:10B2000070BD10B5FEF70AFD18B104F0F9FD044653
:10B2100002E004F0EFFD0446204610BD4FF47A70C2
:10B220007047000010B5FEF7F9FC10B16FF005048F
:10B2300009E00648006820B901200449086000249C
:10B2400001E04FF0FF34204610BD000068000020F0
:10B2500010B5FEF7E3FC10B16FF0050412E004F046
:10B26000B9FD20B1012809D0022806D101E001244E
:10B2700007E004F0F5F8002403E000BF4FF0FF34CE
:10B2800000BF00BF204610BD70B5FEF7C7FC10B16F
:10B290006FF005041FE011480068012819D100BFB4
:10B2A000801F0021002804DB0A07130E0C4A1354E8
:10B2B00006E00A07150E0B4A00F00F031B1FD554BA
:10B2C00000BF00BF02200549086004F06DF80024AB
:10B2D00001E04FF0FF34204670BD00006800002000
:10B2E00000E400E018ED00E010B5FEF797FC10B1A7
:10B2F0006FF0050418E004F06DFD20B101280FD0B7
:10B3000002280CD109E0012404F0C4FE012803D076
:10B3100004F060FD00B9A41E05E0002403E000BFB6
:10B320004FF0FF3400BF00BF204610BD2DE9F843A9
:10B3300005460E4614464FF00009FEF76FFC002844
:10B340003ED1002D3CD0002E3AD0471EBCB1A068A3
:10B3500058B1E068502808D3206930B105FB06F0E9
:10B360006169814201D301270AE0A06840B9E06821
:10B3700030B9206920B9606910B9002700E00027C2
:10B38000012F09D10020009031462846A368226988
:10B3900004F081F9814606E02FB9002231462846A3
:10B3A00004F04CF98146B9F1000F09D014B1D4F87A
:10B3B000008001E04FF000084146484603F0D8FE07
:10B3C0004846BDE8F88310B504F0FEFC044620466C
:10B3D00010BD2DE9FF4780468946144600200390A2
:10B3E000FEF71CFC00284ED1B8F1000F4BD0802690
:10B3F00018258246471E44B3206808B1D4F800A03F
:10B40000A06900B1A5692DB1382D03D8207900F0CD
:10B41000010018B1002004B0BDE8F087606908B1F0
:10B4200060698608A06840B1E0685C2805D320699F
:10B4300018B1606908B1012708E0A06830B9E06878
:10B4400020B9206910B9002700E00027012F0CD196
:10B450002169A0684B463246CDE900510290514621
:10B46000404604F053FC03900DE067B903A8B2B264
:10B470004B465146CDE90050404604F015FC0128EA
:10B4800001D0002003900398C5E72DE9F04106465E
:10B490003746FEF7C3FB10B16FF0050410E017B993
:10B4A0006FF003040CE03846FFF7B2F80546042DB0
:10B4B00004D00024384603F0C5FE01E06FF002041A
:10B4C0002046BDE8F0812DE9F05F81460E46174623
:10B4D0001C463846F4F7E5FE80462068404503D315
:10B4E00000202060BDE8F09F012E01D9701E00E011
:10B4F000002083462068A8EB000ADA4501D25046B6
:10B5000000E05846054695B12068C1192A464846CC
:10B51000F4F797FE002009F8050020682844206011
:10B520002068404501D20120DCE70020DAE7002056
:10B53000206000BFD6E700002DE9F04D1D460C4607
:10B5400098B0174621F0004123F00043002814BFB3
:10B550004FF0010C4FF0000C0CEB440CFE4A0CEBCE
:10B5600002064FEA620C66452BD33E0018BF012647
:10B5700006EB45061644F94A964222D3F84A53EAA6
:10B58000070C02D0944205D148B918B000201146EA
:10B59000BDE8F08D002808BF4FF0000C01D04FF03F
:10B5A000010C0CEB440212F5001F0AD8002F14BF47
:10B5B0004FF0010C4FF0000C0CEB450212F5001F90
:10B5C00007D918B03A462B462146BDE8F04DFEF7A4
:10B5D00085BB0022DFF88CA3002CB8BF534526DAC8
:10B5E000DFF884C36345A8BF022220DADFF870C306
:10B5F0009C451CDCDFF874C30CEB235CBCF1140F1E
:10B6000008DDCCF1340627FA06FC0CFA06F6BE4239
:10B610000DD108E05FB9CCF1140623FA06FC0CFA50
:10B6200006F69E4203D10CF00102C2F1020251EA79
:10B63000000C19D1002D17DA002C18BF022A01D0F6
:10B64000012A07D00220FEF771FB18B0BDE8F04DCB
:10B65000FEF73CBB0220FEF769FBFEF737FB18B094
:10B6600081F00041BDE8F08DB7F1000C6CD153457D
:10B6700025D104F1804212F5801201BF002800207C
:10B68000B74918B008BFBDE8F08DB548884207DC5F
:10B69000002DA1BF6046294618B0BDE8F08D07E037
:10B6A000281E05DA80F0004118B06046BDE8F08D34
:10B6B000AF497944D1E9000118B0BDE8F08DDFF859
:10B6C000A0C2634525D1002D1FDA19B1514512D111
:10B6D000D8B909E0002840F0EC82A24A214618B00F
:10B6E00062F31E01BDE8F08D0020214618B060F322
:10B6F0001E01BDE8F08D08DA18B02346BDE8F04D14
:10B70000024600206146F5F732B818B02146BDE880
:10B71000F08D514518DAB5F1804F0DD0A5F1005CE0
:10B72000BCF1FF5C10D1B4F1000C0DDB18B0614628
:10B73000BDE8F04D03F09EBB234618B00246BDE8BD
:10B74000F04D1946F4F7A1BF060024F0004C3BD1A0
:10B75000D9B1514533D1002C06DD002DA1BF002009
:10B76000514618B0BDE8F08D002C01DD002D1BDB2B
:10B77000002C13DA002D11DB012A4FF0000014BF5A
:10B7800078497C4918B0BDE8F08D022A18BF002C1A
:10B790000AD0012A08D1002C06DA0AE0002CB8BF32
:10B7A000002D11DA012A04D0002018B00146BDE8AE
:10B7B000F08D18B000204FF00041BDE8F08DA1F1F0
:10B7C0004050B0F17F601AD0012000EBE47050EAE5
:10B7D000020421D0624C521E4FF0000B104304BFF4
:10B7E0004FF0000B644C654883427CDD644A654839
:10B7F00093421FDD884217DB002D25DB37E0002C4C
:10B8000000DA4AB1022A0CBF01204FF0FF3018B015
:10B81000BDE8F04DF5F728B80120FEF787FA18B01B
:10B82000BDE8F04DFEF75CBA4D4A8A4202DC002DBD
:10B830000ADC1CE0814202DA002D18DA04E0484BF1
:10B84000994220DD002D12DD0220FEF76FFAFEF78F
:10B850004DFA05460E460022534658462146F4F757
:10B8600014FF18B066F31E012846BDE8F08D0220D3
:10B87000FEF75CFAFEF742FA0A46214618B062F378
:10B880001E01BDE8F08D002230466146F5F740FA12
:10B8900080460E466FF00102F5F740FA4FF0553240
:10B8A000394BF5F738FA42463346F4F7EEFE0022FC
:10B8B000364BF5F730FA824642463346049110463D
:10B8C0001946F4F7E2FE5246049BF4F7DEFE8A4680
:10B8D00000904FF0C0422E4B40463146F4F7D5FE63
:10B8E0002C4A2B4B00E027E0CDE906015146009899
:10B8F000F4F7CBFE82460191274A284B4046314659
:10B90000F4F7C3FE5246019BF5F702FA82460B4656
:10B9100002460591DDE90601F5F759F9DDE906234F
:10B92000002688463046F5F7F3F95246059BF5F7B1
:10B93000F2F9024600F07EB90020B1F5801F07DA67
:10B94000352230466146F5F7E9F906466FF03400D6
:10B9500000EB215024E00000FFFF1F00FFFF0F005D
:10B960000000F03F0000F07F0000404301FCFFFFBB
:10B970008A9600000000F0FF0000F0BF0000E041E8
:10B980000000F043FFFFEF3F5555D53F0000E03F7B
:10B990004715F73FFE822B6544DF5DF80BAE543E42
:10B9A000A0F2FF300190C1F3130040F07F6141F03D
:10B9B00040510291FE498842D8BF002004DDFD4974
:10B9C0008142C8BF012001DD0D9008E000200D90EC
:10B9D0000198401C01900298A0F5801002900299F5
:10B9E000F54878440B910D9900EBC100D0E9002394
:10B9F0000F9330460A920B99F5F78AF9CDE90601C3
:10BA0000DDE90A2130460F9BF5F7E1F802460B46C7
:10BA10000020EA49F4F7ABFE059102460B46009080
:10BA2000DDE90601F4F731FE1490E5488A464FF04F
:10BA3000000878440299006812904FF0005040EAE4
:10BA400061010D980F9B01EB804000F500210991E9
:10BA50000A9A1298F5F75CF932460B9BF5F75BF9F9
:10BA600042465346F4F711FE0646029140465146BF
:10BA7000099B129AF4F709FEDDE90623F5F74BF965
:10BA80003246029BF5F744F9059B009AF4F7FDFD59
:10BA90000091149A0490534610461946F4F7F5FDA8
:10BAA00006460246C7480B46029106217844FEF737
:10BAB000B8F8CDE90510029B324610461946F4F756
:10BAC000E4FDDDE90532F4F7E0FD05910646534655
:10BAD00040461946149AF5F77AF8009B049AF4F751
:10BAE000D4FD3246059BF5F772F8CDE905104246C4
:10BAF000534610461946F4F7C8FD0022B24B029196
:10BB00000A90F5F764F8DDE90532F5F760F80E46BE
:10BB10004246AD4B4046F5F7FBF8029B0A9AF5F713
:10BB2000F7F8DDE90532F5F7F6F8424602910A909A
:10BB3000334610465146F4F7A8FDCDE906015346B9
:10BB4000149A02990A98F4F7A0FD8A4602903346A7
:10BB5000424600990498F4F798FD5346029AF5F787
:10BB600036F882460B4602460591DDE90601F5F7F7
:10BB70002EF8DDE90623002088460646F5F7C8F8CA
:10BB80005246059BF5F7C7F8824609914FF060428F
:10BB90008E4B30464146F4F778FD049006918C4A6E
:10BBA0008A4B50460999F4F770FD82460291894A02
:10BBB000894B30464146F4F768FD5246029BF5F743
:10BBC00006F8864B7B440D9A03EBC203D3E90023AE
:10BBD000F4F7FDFF0E9007910198F4F745FE0591EB
:10BBE000DDE9061382460E9A0498F4F7F0FF7C4ACA
:10BBF0007A440D9B02EBC303D3E900230093029226
:10BC0000F4F7E5FF5246059BF4F7E1FF002688466E
:10BC100052463046059BF5F77BF8009B029AF5F7F4
:10BC200077F8069B049AF5F773F8079B0E9AF5F7D9
:10BC300072F8024600200B46029038462946F4F777
:10BC400024FD824601912B4638461946029AF5F7A3
:10BC50005FF832464346F4F718FD5246019BF4F76D
:10BC6000B6FF07468A463246434629460298F4F70D
:10BC70000CFD05460E463A465346F4F7A8FF594ACE
:10BC80008846914221DBA8EB020353EA000210D15F
:10BC90002A463346F5F73CF8CDE90401524A534BA6
:10BCA00038465146F4F793FFDDE90423F5F766F8CB
:10BCB00021D20220FEF73AF8FEF718F80A4621468C
:10BCC00018B062F31E01BDE8F08D494B28F0004228
:10BCD0009A4210D3474A08EB020353EA00027FF46A
:10BCE000C6AD2A463346F5F713F83A465346F5F7FC
:10BCF00045F87FF6BCAD0022019228F000403E4995
:10BD00003E4A01EB2051824223DA481C4FF4801155
:10BD100021FA00F040443A4AC0F30A517A44394BC0
:10BD2000A1F2FF31CB4020EA0303C0F3130040F43B
:10BD30008010C1F11401C84012680190B8F1000FE1
:10BD4000BCBF4042019028463146F4F7E1FF05466A
:10BD50000E462A46334638465146F4F738FF4FF030
:10BD600000084246284B40460591F4F78EFCCDE989
:10BD70000601264A264B40460599F4F786FC0091B9
:10BD800002902A46334640460599F4F7C1FF3A46E9
:10BD90005346F4F7C0FF1F4A1F4BF4F776FC009B95
:10BDA000029AF4F714FF0746884602460B4635E030
:10BDB0008E9803007AB60B00D29200000000F03F8C
:10BDC0000A930000389200000000084009C7EE3FC7
:10BDD000FD033ADCF5015B14E02F3EBE109100003C
:10BDE000D490000000009040FE822B654715973CE0
:10BDF00000CC904000346F3F01FCFFFF0000E03FAB
:10BE000020900000FFFF0F00432EE63F396CA80C86
:10BE1000615C20BEEF39FAFE422EE63FDDE9060105
:10BE2000F4F7D5FEDDE9062305460E46F4F770FF6C
:10BE30003A464346F4F76FFF0F462A4633460090D2
:10BE400010461946F4F721FC824602462E488846E1
:10BE50000B4605217844FDF7E4FE52464346F4F7CD
:10BE600014FC2A463346F4F756FF80468A463B4682
:10BE700028463146009AF4F708FC3B46009AF4F74E
:10BE8000A6FE0691009000224FF0804340465146A6
:10BE9000F4F73EFF0F460C90424653462846314683
:10BEA000F4F7F3FB3B460C9AF4F761FC069B009A0F
:10BEB000F4F72EFF2A463346F4F72AFF0022134BED
:10BEC000F4F729FF054601980E4601EB00510815CD
:10BED000002810DC28463146019AF4F71FFFFDF7D1
:10BEE00069FE042808BFFDF709FF28463146019A7C
:10BEF000F4F714FF05460B4618B02A46584621466B
:10BF0000BDE8F04DF4F7C1BBC08E00000000F03F6B
:10BF10002DE9F04105460E461648076816480068A8
:10BF2000001D02F0D9FF681C38B936B1124801680B
:10BF3000091D124803F026F81AE07C190E48006823
:10BF40004460BC4207D20C480168091D0C480068D7
:10BF500002F0FEFF0CE008480168091D094800686E
:10BF600002F0F6FF08480068844201D206480460E7
:10BF7000BDE8F0812C00002018000020600B00209C
:10BF8000200000201C0000204800002010B50446BE
:10BF900003F004F824480068401C23490860234843
:10BFA000006840B9214804600846006801280DD1A6
:10BFB00000F03AFA0AE01E48006838B91B480068E9
:10BFC000C06AE16A884201D81848046019480068CC
:10BFD000401C184908600846006860641649E06A19
:10BFE0000968884202D91449E06A0860E16A01EBF5
:10BFF0008101124A02EB8100211D02F0C3FF02F011
:10C00000F7FF0B48006868B108480068C06AE16A39
:10C01000884207D24FF0805009490860BFF34F8F24
:10C02000BFF36F8F10BD0000280000201800002013
:10C03000340000204400002030000020B006002022
:10C0400004ED00E008B502F0A9FF12480068E8B965
:10C05000114802F06DFF114802F06AFF0E481049C6
:10C0600008600E480F49086000200F4B0F4A10214E
:10C0700000900A2003F00FFB06490860084600689C
:10C0800020B10BA10348006803F072F802F0B0FF82
:10C0900008BD00005C000020740B0020880B00200D
:10C0A00054000020580000209C0B0020EC0B0020C6
:10C0B000546D72510000000010B516E002F06EFFE2
:10C0C0000C48C068C468201D02F006FF0A480068DA
:10C0D000401E0949086009480068401E0749086079
:10C0E00002F086FF204600F05FF804480068002850
:10C0F000E4D110BD4C0B00202800002024000020BB
:10C1000070B504460D46206C70B1216CE0680144A6
:10C11000E160D4E90210884201D32168E160284639
:10C12000226CE168F4F78DF870BD2DE9F04104460A
:10C130000F4615464FF00008A66B206C48B92068E2
:10C1400000282CD1A06803F007FF80460020A060E3
:10C1500025E07DB93946226C6068F4F772F8216CED
:10C16000606808446060D4E90101884217D3206800
:10C17000606014E03946226CE068F4F762F8216CE4
:10C18000E068411AE1602168E068884203D2216CCE
:10C19000A068411AE160022D01D106B1761E701C23
:10C1A000A0634046BDE8F08110B5044694F85900FC
:10C1B00030B9206B02F03AFF204602F037FF1AE058
:10C1C00094F85900012803D1204602F02FFF12E015
:10C1D00094F85900022801D1012000E0002050B954
:10C1E00000BF502080F31188BFF34F8FBFF36F8FD4
:10C1F00000BF00BFFEE710BD0146084A1268126882
:10C200000AB9012200E000220A600A6822B9034A42
:10C210001268D268106800E00020704754000020C7
:10C220000146002000220AE00B78202B05D1012ACC
:10C2300004D0431C58B2012200E00022491C0B78B4
:10C24000002BF1D1012A01D1431E58B270470000E2
:10C2500030B54FF44063174800F007042CB1C01DFF
:10C2600020F00700134C041B1B1B0246124C2260DB
:10C270000024114D6C60D018083820F007000F4CD6
:10C28000206000240D4D2D686C600C4D2D682C60D5
:10C290001146441A4C60094C24680C60084D4C68E7
:10C2A0002C60084D4C682C604FF00044064D2C600B
:10C2B00030BD0000441300206C00002074000020FA
:10C2C0007C00002078000020880000202DE9F0414B
:10C2D00006460D4617460E48006810B90D480C4931
:10C2E00008600B48006800682A4641683046F3F74A
:10C2F000CCFF0748006840680549086008460068A8
:10C3000008B9002400E001242046BDE8F0810000C7
:10C3100004010020F400002000BFFFF7CDFE064816
:10C3200000680128F9D94FF0805004490860BFF334
:10C330004F8FBFF36F8FF0E7B006002004ED00E0F1
:10C340002DE9F04106460D4617469846069C0DB964
:10C35000246000E02760E66325640121204603F0A5
:10C360000BFA84F84C80BDE8F0812DE9F05F82463D
:10C370000E4690469B460A9F0C9C4FEA8801A522D8
:10C38000206BF3F770FFA8F10100216B01EB80092E
:10C3900029F0070909F0070008B9012000E0002092
:10C3A00050B900BF502080F31188BFF34F8FBFF307
:10C3B0006F8F00BF00BFFEE786B1002507E0715D0B
:10C3C00004F134004155705D00B902E06D1C102D80
:10C3D000F5D300BF00214320015502E0002084F87E
:10C3E0003400382F00D33727E762E7640020206548
:10C3F000201D02F0AAFD04F1180002F0A6FD246140
:10C40000C7F13800A06164620020606584F85800BC
:10C410005A465146484600F071FB20600B9808B11F
:10C420000B980460BDE8F09F10B5002407E004EB12
:10C4300084010F4A02EB810002F07AFD641C382C63
:10C44000F5D30C4802F074FD0B4802F071FD0B4867
:10C4500002F06EFD0A4802F06BFD0A4802F068FD2A
:10C4600004480949086004480849086010BD0000F4
:10C47000B0060020100B0020240B0020380B0020F9
:10C480004C0B0020600B00201C000020200000202E
:10C4900010B50146164800E0006803688B42FBD3E4
:10C4A0000246436813448B4204D143684C682344DA
:10C4B000436001460A464B6813440468A34211D105
:10C4C0000C4C03682468A34208D04B680468646875
:10C4D00023444B6003681B680B6005E0054B1B6839
:10C4E0000B6001E003680B60884200D0016010BD62
:10C4F0006C000020740000202DE9F04104460D4638
:10C5000016461F464FF0000865602461B5420CD8FE
:10C51000F01BA169884202D34FF0010811E0211DF0
:10C520000948006802F014FD0BE0BE4204D2BD428F
:10C5300002D34FF0010804E0211D0448006802F016
:10C5400007FD4046BDE8F08158000020540000205F
:10C5500070B5054602F022FDA86B08B9012400E081
:10C56000002402F045FD204670BD70B5054602F07E
:10C5700015FDA86BE96B884201D1012400E000247D
:10C5800002F036FD204670BDF8B505460F461A4844
:10C590000068C068C468201D02F09EFC94F8280062
:10C5A00000F00400E8B1A06941192B463A46204644
:10C5B000FFF7A2FFD8B1002003462A4601460090AB
:10C5C000204603F025FE064656B900BF502080F3F2
:10C5D0001188BFF34F8FBFF36F8F00BF00BFFEE71F
:10C5E00005E094F8280020F0010084F82800204697
:10C5F000216A8847F8BD000054000020F0B587B0DC
:10C60000A0E00398002811DA04AE56B900BF50200C
:10C6100080F31188BFF34F8FBFF36F8F00BF00BF50
:10C62000FEE7D6E90020B168904700BF03980028D4
:10C63000E6DB059C606908B9012000E0002010B924
:10C64000201D02F049FC02A800F0DEF80546039820
:10C650000A2875D2DFE800F00905073941630608AA
:10C660003A4200BF00BF00BF00BF94F8280040F06E
:10C67000010084F828000498A269811803462A461C
:10C680002046FFF739FFF8B12046216A884794F821
:10C69000280000F00400B8B1002000900498A169BF
:10C6A000421800231946204603F0B2FD074657B949
:10C6B00000BF502080F31188BFF34F8FBFF36F8FFF
:10C6C00000BF00BFFEE700BF3BE000BF94F82800BA
:10C6D00020F0010084F8280033E000BF94F828001F
:10C6E00040F0010084F828000498A061A06908B116
:10C6F000012000E0002050B900BF502080F31188D5
:10C70000BFF34F8FBFF36F8F00BF00BFFEE7A0697D
:10C7100041192B462A462046FFF7EEFE11E094F819
:10C72000280000F0020018B9204602F07FFC05E066
:10C7300094F8280020F0010084F8280001E0FFE7C9
:10C7400000BF00BF002203A90448006803F0B2F94B
:10C7500000287FF456AF07B0F0BD00005C00002059
:10C76000F8B505460C4602F07BFE684600F04CF832
:10C770000646009820BB44B9B54206D803F08AFCAF
:10C7800031462846FFF700FF1CE03CB10E48006828
:10C79000006808B9012000E000200446A91B2246D9
:10C7A0000A48006802F0FAFC03F074FC50B94FF03C
:10C7B000805007490860BFF34F8FBFF36F8F01E0D0
:10C7C00003F068FCF8BD0000580000205C00002069
:10C7D00004ED00E00A490968096809B9012100E08F
:10C7E000002121B14FF0FF31064A116006E00449F3
:10C7F0000968C968C868034A416811607047000049
:10C800001C0000204800002070B5044603F0F2FA36
:10C81000054607480068854204D200F00BF8012065
:10C82000206001E00020206001480560284670BDBE
:10C83000640000202DE9F84334E025480068C06812
:10C84000056823480068C068C468201D02F044FBE6
:10C850002046216A884794F8280000F0040008B3B5
:10C86000A0694619AE4207D966602461211D1848A7
:10C87000006802F06DFB15E0002003462A460146E1
:10C880000090204603F0C4FC074657B900BF502073
:10C8900080F31188BFF34F8FBFF36F8F00BF00BFCE
:10C8A000FEE700BF0A480068006808B9012000E000
:10C8B00000200028C1D00648D0F800800548006854
:10C8C000034908600348C0F80080BDE8F883000011
:10C8D00054000020580000200E480068401C08B991
:10C8E000012000E0002050B900BF502080F31188E3
:10C8F000BFF34F8FBFF36F8F00BF00BFFEE700BFD6
:10C90000502080F31188BFF34F8FBFF36F8F00BFAC
:10C9100000BFFEE78C00002008B500BF6846FFF7A7
:10C920006BFC044620460099FFF71AFFFFF766FEEE
:10C93000F4E770B5044602F031FB94F9455010E07D
:10C94000606A08B9012000E0002038B904F1240031
:10C9500003F054FB18B102F0E5FC00E003E0681EB0
:10C9600045B2002DECDC00BFFF2084F8450002F04A
:10C970003FFB02F013FB94F9445010E0206908B922
:10C98000012000E0002048B904F1100003F036FB5C
:10C9900008B102F0C7FC681E45B200E001E0002DBE
:10C9A000ECDC00BFFF2084F8440002F021FB70BDE6
:10C9B0002DE9F04104464FF0000802F051FD4948CE
:10C9C000006808B9FFF744FC474800682040002889
:10C9D00070D1D4B1083404F00700B0B104F00700FE
:10C9E000C0F10800044404F0070008B9012000E089
:10C9F000002050B900BF502080F31188BFF34F8F43
:10CA0000BFF36F8F00BF00BFFEE7002C52D0374846
:10CA1000006884424ED8364E3046056801E02E4606
:10CA20002D686868A04202D228680028F7D12D48F6
:10CA3000006885423ED0306800F108082868306000
:10CA40006868001B102819D92F1907F0070008B9CA
:10CA5000012000E0002050B900BF502080F3118871
:10CA6000BFF34F8FBFF36F8F00BF00BFFEE7686853
:10CA7000001B78606C603846FFF70AFD1B49686848
:10CA80000968081A194908600846006819490968C0
:10CA9000884203D215480068164908601249686840
:10CAA0000968084368600020286013480068401C3B
:10CAB0001149086003F0EEFA08F0070008B90120F8
:10CAC00000E0002050B900BF502080F31188BFF370
:10CAD0004F8FBFF36F8F00BF00BFFEE74046BDE83A
:10CAE000F081000074000020880000207800002001
:10CAF0006C0000207C00002080000020001F4FF010
:10CB000080730360001F21F001030360001F034BCB
:10CB1000036014380260203870470000D9C800084C
:10CB200007B5B8B00020379036903590349037AACA
:10CB300001213A98F5F7C2F8339036AA02213A98C3
:10CB4000F5F7BCF8329035AA03213A98F5F7B6F814
:10CB5000319034AA04213A98F5F7B0F830902021AA
:10CB600028A8F3F787FB202120A8F3F783FB2021D7
:10CB700018A8F3F77FFB202110A8F3F77BFB33986D
:10CB800028B1202328AA37993398FDF725FD32983C
:10CB900028B1202320AA36993298FDF71DFD31983F
:10CBA00028B1202318AA35993198FDF715FD309842
:10CBB00028B1202310AA34993098FDF70DFDF8A173
:10CBC00028A8F3F784FBC0B9F748F3F76AFBF749E5
:10CBD0000968884202D80020F4490860F34BF24A01
:10CBE000DDE93801FEF76FFC0F900F9810B90020B7
:10CBF000EE4908600F983BB000BDEDA128A8F3F7FF
:10CC000066FBE0B9E6A120A8F3F761FBB8B9EB48F1
:10CC1000F3F747FBEA490968884202D80020E8494F
:10CC20000860E74BE54ADDE93801FEF74CFC0F9060
:10CC30000F9810B90020E24908600F98DBE7E1A1E6
:10CC400028A8F3F744FBE0B9D5A120A8F3F73FFBF0
:10CC5000B8B9DE48F3F725FBDD490968884202D8F8
:10CC60000020DB490860DA4BD84ADDE93801FEF7DD
:10CC70002AFC0F900F9810B90020D54908600F9832
:10CC8000B9E700200F909DF8400030B10022114616
:10CC900010A8F3F72BFC0F9008E09DF8600028B176
:10CCA0000022114618A8F3F721FC0F90C9A128A86B
:10CCB000F3F70DFB00284BD19DF8800070B9C748F1
:10CCC000406840780D90FDF73DFD0346C4A20E90EC
:10CCD000DDE93801FCF754FF02F004B8C7A120A831
:10CCE000F3F7F5FA10B900200E901FE0C4A120A8B8
:10CCF000F3F7EDFA10B901200E9017E0C2A120A8B9
:10CD0000F3F7E5FA10B902200E900FE0C0A120A8B9
:10CD1000F3F7DDFA10B903200E9007E020ABBEA2B6
:10CD2000DDE93801FCF72CFF002064E7AB480E99E1
:10CD3000FBF75EFD30B920ABBEA2DDE93801FCF7A0
:10CD40001FFF04E0C1A2DDE93801FCF719FFC3E7CA
:10CD500097A128A8F3F7BBFA00286FD19DF88000AF
:10CD600000286DD19D48406890F83500D8B1012861
:10CD70002FD0032843D0042857D19848406890F812
:10CD800041109648406890F84000CDE90001934872
:10CD9000406890F83F000346B3A20E90DDE93801E9
:10CDA000FCF7EEFE47E08D48406890F838108B485D
:10CDB000406890F83700CDE900018848406890F855
:10CDC00036000346B6A20E90DDE93801FCF7D8FE26
:10CDD00031E08248406890F83B108048406890F805
:10CDE0003A00CDE900017D48406890F839000346DB
:10CDF000B9A20E90DDE93801FCF7C2FE1BE07748CE
:10CE0000406890F83E107548406890F83D00CDE9C4
:10CE100000017248406890F83C000346B9A20E90A9
:10CE2000DDE93801FCF7ACFE05E0C3A2DDE938011D
:10CE3000FCF7A6FE00BF00BF0020DCE63EE3FFE7F4
:10CE40006648406890F83500002855D0012872D017
:10CE5000032871D0042870D1C0A120A8F3F737FAB5
:10CE600080B90F98EF2806D9BEA2DDE93801FCF79A
:10CE700087FE0020BFE60F98C1B25848406880F88E
:10CE80003F1038E0C2A120A8F3F721FA80B90F982B
:10CE90000F2806D9C1A2DDE93801FCF771FE002098
:10CEA000A9E60F98C1B24D48406880F8401022E0D2
:10CEB000C5A120A8F3F70BFAA8B90F9860B10F9895
:10CEC000102809D00F98202806D0C1A2DDE938012A
:10CED000FCF756FE00208EE60F98C1B23F4840682E
:10CEE00080F8411007E020ABC6A2DDE93801FCF76D
:10CEF00047FE00207FE6D0E298A120A8F3F7E7F9EB
:10CF000080B90F98EF2806D9C8A2DDE93801FCF7EF
:10CF100037FE00206FE60F98C1B23048406880F8B5
:10CF20003610DDE19AA120A8F3F7D1F9A0B90F9846
:10CF30000F280AD902E0D4E13DE2A7E2C6A2DDE96A
:10CF40003801FCF71DFE002055E60F98C1B22348BA
:10CF5000406880F83710C3E19BA120A8F3F7B7F928
:10CF6000A8B90F9860B10F98102809D00F98202801
:10CF700006D0C4A2DDE93801FCF702FE00203AE643
:10CF80000F98C1B21548406880F83810A8E120AB6E
:10CF9000C9A2DDE93801FCF7F3FD00202BE6000013
:10CFA00068656C7000000000281D01081001002059
:10CFB0006D6F64756C6174696F6E0000C122010849
:10CFC000140100207061636B65740000B42E0108C9
:10CFD000180100206D6F646500000000E02C002047
:10CFE00043757272656E7420726164696F206D6F33
:10CFF00064653A2025730D0A00000000424C45008C
:10D000004C4F5241000000004746534B00000000C7
:10D01000464C524300000000556E6B6E6F776E20D9
:10D02000726164696F206D6F64653A2025730D0A23
:10D0300000000000526164696F206D6F64652073A9
:10D04000657420746F2025730D0A00004661696CB9
:10D05000656420746F2073657420726164696F2049
:10D060006D6F64650D0A00004D6F64756C617469C5
:10D070006F6E28424C45293A2062725F62773D30DC
:10D08000782558206D6F64696E6465783D2575203C
:10D0900073686170696E673D307825580D0A00002D
:10D0A0004D6F64756C6174696F6E284746534B29E8
:10D0B0003A2062725F62773D30782558206D6F6448
:10D0C000696E6465783D25752073686170696E6767
:10D0D0003D307825580D0A004D6F64756C61746998
:10D0E0006F6E284C6F5261293A2073663D30782567
:10D0F000582062773D307825582063723D3078257E
:10D10000580D0A004D6F64756C6174696F6E284626
:10D110004C5243293A2062725F62773D307825583D
:10D120002063723D307825582073686170696E679E
:10D130003D307825580D0A00556E6B6E6F776E2066
:10D140006D6F64756C6174696F6E207061636B657F
:10D150007420747970650D0A0000000062725F62CD
:10D1600077000000496E76616C69642062725F62CC
:10D17000772076616C756520666F7220424C452081
:10D18000286D61783A2030784546290D0A00000064
:10D190006D6F64696E64657800000000496E7661A9
:10D1A0006C6964206D6F64696E6465782076616C6B
:10D1B000756520666F7220424C4520286D61783A73
:10D1C000203135290D0A000073686170696E6700AF
:10D1D000496E76616C69642073686170696E67205E
:10D1E00076616C756520666F7220424C4520283050
:10D1F0007830302F307831302F30783230290D0AA6
:10D2000000000000556E6B6E6F776E206D6F647559
:10D210006C6174696F6E206669656C6420666F72FC
:10D2200020424C453A2025730D0A0000496E766174
:10D230006C69642062725F62772076616C7565202C
:10D24000666F72204746534B20286D61783A203034
:10D25000784546290D0A0000496E76616C696420A4
:10D260006D6F64696E6465782076616C75652066A3
:10D270006F72204746534B20286D61783A20313534
:10D28000290D0A00496E76616C69642073686170CB
:10D29000696E672076616C756520666F72204746FF
:10D2A000534B2028307830302F307831302F307881
:10D2B0003230290D0A000000556E6B6E6F776E20BC
:10D2C0006D6F64756C6174696F6E206669656C64FE
:10D2D00020666F72204746534B3A2025730D0A0093
:10D2E000DBE0F7A120A8F2F7F2FF28BB0F98502847
:10D2F0001BD00F98602818D00F98702815D00F9861
:10D30000802812D00F9890280FD00F98A0280CD00A
:10D310000F98B02809D00F98C02806D0E9A2DDE9FF
:10D320003801FCF72DFC002065E40F98C1B2EC48F1
:10D33000406880F839103DE0EAA120A8F2F7C7FF65
:10D34000C8B90F9834280FD00F9826280CD00F9802
:10D35000182809D00F980A2806D0E3A2DDE9380181
:10D36000FCF70EFC002046E40F98C1B2DC48406890
:10D3700080F83A101EE0E3A120A8F2F7A8FF90B9C8
:10D380000F9810B10F98072806D9DFA2DDE9380100
:10D39000FCF7F6FB00202EE40F98C1B2D04840689D
:10D3A00080F83B1006E0DFA2DDE93801FCF7E8FB7E
:10D3B000002020E471E0AFF25C2120A8F2F787FFA3
:10D3C00028BB0F9804281BD00F98282818D00F9836
:10D3D000452815D00F98692812D00F9886280FD0AD
:10D3E0000F98AA280CD00F98C72809D00F98EB28BF
:10D3F00006D0D3A2DDE93801FCF7C2FB00201DE412
:10D400000F98C1B2B648406880F83C103DE0BDA11D
:10D4100020A8F2F75CFFA8B90F9860B10F98022816
:10D4200009D00F98042806D0CDA2DDE93801FCF719
:10D43000A7FB002024E40F98C1B2A948406880F8F7
:10D440003D1022E0AFF2802120A8F2F740FFA8B9FA
:10D450000F9860B10F98102809D00F98202806D097
:10D46000C6A2DDE93801FCF78BFB002008E40F9829
:10D47000C1B29B48406880F83E1006E0A9A2DDE9F1
:10D480003801FCF77DFB00204FE406E0C4A2DDE993
:10D490003801FCF775FB002047E400BF9048406866
:10D4A00035300E90C648006C0D90DDE90D108847B0
:10D4B000C4A2DDE93801FCF763FB0DE4AFF2FC41E7
:10D4C00028A8F2F704FF002841F0C4809DF88000EE
:10D4D000F0BB83484068407F00B3012848D0032850
:10D4E00066D004287ED17E48406890F834107C488D
:10D4F000406890F833207A48406890F83200CDE9CF
:10D50000012100907648406890F831000346B34A04
:10D510000E90DDE93801FCF733FB7BE07048406892
:10D5200090F824106E48406890F823306C484068AA
:10D5300090F822206A48406890F82100CDE9032342
:10D54000059102906648406890F82010644800E019
:10D5500063E04068C07FCDE9000161484068807F9A
:10D5600003469F4A0E90DDE93801FCF709FB51E0C4
:10D570005B48406890F829105948406890F8282086
:10D580005748406890F827305548406890F8260082
:10D59000CDE90132039100905148406890F8250090
:10D5A0000346904A0E90DDE93801FCF7E9FA31E0D4
:10D5B0004B48406890F830104948406890F82F2058
:10D5C0004748406890F82E304548406890F82D0054
:10D5D000CDE90332059102904148406890F82C1043
:10D5E0003F4800E010E0406890F82B00CDE90001D2
:10D5F0003B48406890F82A0003467B4A0E90DDE9DC
:10D600003801FCF7BDFA05E078A2DDE93801FCF746
:10D61000B7FA00BF00BF00200FE431484068407FE8
:10D62000002849D0012848D0032847D0042840F0DA
:10D63000F88774A120A8F2F74AFE80B90F98042851
:10D6400006D974A2DDE93801FCF79AFA002011E44A
:10D650000F98C1B22248406880F8311039E176A1B4
:10D6600020A8F2F734FE80B90F98012806D975A2D8
:10D67000DDE93801FCF784FA002011E40F98C1B20B
:10D680001748406880F8321023E176A120A8F2F70D
:10D690001EFE80B90F98072806D976A2DDE9380169
:10D6A000FCF76EFA002016E40F98C1B20C484068EF
:10D6B00080F833100DE1EDE00CE1F3E3F3E300005B
:10D6C00073660000496E76616C696420736620762B
:10D6D000616C756520666F72204C4F52410D0A00D7
:10D6E000E02C002062770000496E76616C6964204E
:10D6F00062772076616C756520666F72204C4F52A0
:10D70000410D0A0063720000496E76616C69642005
:10D7100063722076616C756520666F72204C4F5283
:10D72000410D0A00556E6B6E6F776E206D6F6475DC
:10D730006C6174696F6E206669656C640D0A000027
:10D74000496E76616C69642062725F6277207661EF
:10D750006C756520666F7220464C52430D0A0000BE
:10D76000496E76616C69642063722076616C7565C0
:10D7700020666F7220464C52430D0A00496E766156
:10D780006C69642073686170696E672076616C757E
:10D790006520666F7220464C52430D0A000000005F
:10D7A000556E6B6E6F776E2063757272656E742046
:10D7B0007061636B657420747970650D0A000000F8
:10D7C000341C01084D6F64756C6174696F6E20754F
:10D7D0007064617465640D0A000000004C52010819
:10D7E000E05101082851010874510108556E6B6E13
:10D7F0006F776E207061636B657420747970650D4E
:10D800000A000000436F6E6E656374696F6E537437
:10D8100061746500496E76616C696420424C4520F4
:10D82000436F6E6E656374696F6E537461746520C7
:10D8300028302D34290D0A004372634669656C64F3
:10D8400000000000496E76616C696420424C4520FE
:10D850004372634669656C642028302D31290D0AB6
:10D8600000000000426C655061636B657454797010
:10D8700065000000496E76616C696420424C455039
:10D8800061636B6574547970652028302D37290DDC
:10D890000A000000F4A120A8F2F719FD90B90F9832
:10D8A00048B10F98082806D0F2A2DDE93801FCF74C
:10D8B00067F9002038E50F98C1B2F748406880F852
:10D8C000341006E0F5A2DDE93801FCF759F9002033
:10D8D0002AE52EE3F8A120A8F2F7F9FC18BB0F986F
:10D8E000D8B10F98102818D00F98202815D00F986D
:10D8F000302812D00F9840280FD00F9850280CD005
:10D900000F98602809D00F98702806D0ED4ADDE9FD
:10D910003801FCF735F9002006E50F98C1B2DE4862
:10D920004068817705E3E8A120A8F2F7D0FCD0B9E0
:10D930000F9890B10F9802280FD00F9804280CD0A0
:10D940000F98062809D00F98082806D0E2A2DDE932
:10D950003801FCF715F90020E6E40F98C1B2CE4873
:10D960004068C177E5E2EBA120A8F2F7B0FC20BB4C
:10D970000F98D8B10F98102818D00F98202815D0DC
:10D980000F98302812D00F9840280FD00F985028A9
:10D990000CD00F98602809D00F98702806D0E14A63
:10D9A000DDE93801FCF7ECF80020BDE40F98C1B2C6
:10D9B000B948406880F82010BBE2DBA120A8F2F74C
:10D9C00086FCE8BBDB480068017CDA480068C37B62
:10D9D000D8480068827BD7480068407BCDE90B239C
:10D9E0000D910A90D3480068017BD2480068C27A42
:10D9F000D0480068837ACF480068407ACDE9073282
:10DA000009910690CB480068007ACA490968CA792A
:10DA1000C84909688979C74B1B685B79CDE9023130
:10DA2000CDE90420C34800680079C2490968C97873
:10DA3000CDE90010BF48006880780346BE4A00E088
:10DA400006E00E90DDE93801FCF79AF800206BE45F
:10DA5000BAA120A8F2F73BFCE0BB9DF8600020B320
:10DA60000022114618A8F2F741FD0E900E98000E04
:10DA7000B049096888700E98010CAE480068C17002
:10DA80000E98010AAB48006801710E98C1B2A9480E
:10DA9000006841710021A74800688171AAA20E9B0D
:10DAA000DDE93801FCF76CF81BE0A24800688079DA
:10DAB000A04909684A799F49096809799D4B1B6803
:10DAC000DB78CDE90031CDE902209A480068807802
:10DAD000034600E007E0A5A20E90DDE93801FCF75F
:10DAE0004FF8002020E4ACA120A8F2F7F0FBE0BB47
:10DAF0009DF8600020B30022114618A8F2F7F6FC4A
:10DB00000E900E98000E8B490968C8710E98010C92
:10DB10008848006801720E98010A864800684172C0
:10DB20000E98C1B283480068817200218148006864
:10DB3000C1729CA20E9BDDE93801FCF721F81BE0C5
:10DB40007C480068C17A7B480068827A794800681E
:10DB5000437A78480068007ACDE901320391009059
:10DB600074480068C079034600E007E096A20E9072
:10DB7000DDE93801FCF704F800200CE49DA120A8A1
:10DB8000F2F7A5FBE0BB9DF8600020B30022114630
:10DB900018A8F2F7ABFC0E900E98000E65490968C4
:10DBA00008730E98010C6348006841730E98010ACF
:10DBB0006048006881730E98C1B25E480068C17306
:10DBC00000215C48006801748DA20E9BDDE93801DC
:10DBD000FBF7D6FF1BE057480068027C55480068F9
:10DBE000C17B54480068837B52480068407BCDE984
:10DBF0000131039200904F480068007B034600E02B
:10DC000007E088A20E90DDE93801FBF7B9FF00209C
:10DC100010E48FA120A8F2F75AFB90B90F9848B1F1
:10DC20000F98202806D08CA2DDE93801FBF7A8FF69
:10DC300000201BE40F98C1B21748406880F82110FB
:10DC400077E18EA120A8F2F742FB58B90F9810B1E6
:10DC50000F98FF2807D98BA2DDE93801FBF790FF69
:10DC6000002011E427E11FE157686974656E696E51
:10DC700067000000496E76616C696420424C452063
:10DC800057686974656E696E672028307830302F68
:10DC900030783038290D0A00E02C0020556E6B6E6C
:10DCA0006F776E20424C45207061636B657420660F
:10DCB00069656C640D0A0000507265616D626C6587
:10DCC00000000000004F010853796E63576F7264C3
:10DCD0004C656E6774680000496E76616C696420FB
:10DCE0004746534B2053796E63576F72644C656E91
:10DCF0006774682028307830302F307830322F30F9
:10DD00007830342F307830362F30783038290D0A7B
:10DD10000000000053796E63576F72644D61746345
:10DD2000680000008C4F010853796E63576F72646E
:10DD300000000000302F00200453010853796E6367
:10DD4000576F7264310000004746534B2073796E61
:10DD50006320776F726420312073657420746F20A4
:10DD600030782530386C580D0A0000004746534B78
:10DD70002053796E6320576F726420313A2025302A
:10DD80003258253032582530325825303258253017
:10DD900032580D0A0000000053796E63576F7264A9
:10DDA000320000004746534B2073796E6320776F33
:10DDB000726420322073657420746F2030782530AF
:10DDC000386C580D0A0000004746534B2053796EBB
:10DDD0006320576F726420323A2025303258253044
:10DDE00032582530325825303258253032580D0AF5
:10DDF0000000000053796E63576F726433000000B7
:10DE00004746534B2073796E6320776F72642033DB
:10DE10002073657420746F2030782530386C580D6D
:10DE20000A0000004746534B2053796E6320576F1A
:10DE3000726420333A20253032582530325825304C
:10DE4000325825303258253032580D0A0000000073
:10DE50004865616465720000496E76616C69642092
:10DE60004746534B204865616465722028307830FE
:10DE7000302F30783230290D0A0000005061796C63
:10DE80006F616400496E76616C6964204746534B4C
:10DE9000205061796C6F61642028312D323535292D
:10DEA0000D0A000046E0C7E00F98C1B2FD48406887
:10DEB00080F822103DE0FCA120A8F2F708FAC0B9D2
:10DEC0000F9878B10F9810280CD00F98202809D0FF
:10DED0000F98302806D0F5A2DDE93801FBF750FE97
:10DEE0000020E7E40F98C1B2EE48406880F82310A4
:10DEF0001FE0AFF28C2120A8F2F7E9F990B90F9852
:10DF000048B10F98082806D0F3A2DDE93801FBF7E5
:10DF100037FE0020CEE40F98C1B2E248406880F896
:10DF2000241006E0F6A2DDE93801FBF729FE002007
:10DF3000C0E47EE3AFF2802120A8F2F7C8F988B9E7
:10DF400000BF0F98FF2806D9F4A2DDE93801FBF7DE
:10DF500017FE0020AEE40F98C1B2D248406880F8A6
:10DF6000251068E0AFF2181120A8F2F7B0F990B9C7
:10DF70000F9848B10F98802806D0F0A2DDE938014B
:10DF8000FBF7FEFD002095E40F98C1B2C54840683C
:10DF900080F826104FE0AFF21C1120A8F2F797F995
:10DFA00090B90F9810B10F98FF2806D9ECA2DDE9BF
:10DFB0003801FBF7E5FD00207CE40F98C1B2B948B9
:10DFC000406880F8271036E0B7A120A8F2F77FF963
:10DFD00090B90F9848B10F98202806D0E8A2DDE943
:10DFE0003801FBF7CDFD002064E40F98C1B2AD48C5
:10DFF000406880F828101EE0E9A120A8F2F767F930
:10E0000090B90F9848B10F98402806D0E7A2DDE9F3
:10E010003801FBF7B5FD00204CE40F98C1B2A148D0
:10E02000406880F8291006E0E9A2DDE93801FBF735
:10E03000A7FD00203EE4FCE2AFF2843120A8F2F715
:10E0400046F920BB0F98D8B10F98102818D00F9818
:10E05000202815D00F98302812D00F9840280FD0C4
:10E060000F9850280CD00F98602809D00F9870286E
:10E0700006D0DE4ADDE93801FBF782FD002019E415
:10E080000F98C1B28748406880F82A10C8E2AFF202
:10E09000C83120A8F2F71BF9D8B90F9890B10F98A2
:10E0A00002280FD00F9804280CD00F98062809D00A
:10E0B0000F98082806D0CEA2DDE93801FBF760FDF5
:10E0C000002005E40F98C1B27648406880F82B1014
:10E0D000A6E2AFF2C03120A8F2F7F9F820BB0F9802
:10E0E000D8B10F98102818D00F98202815D00F9865
:10E0F000302812D00F9840280FD00F9850280CD0FD
:10E100000F98602809D00F98702806D0C74ADDE91B
:10E110003801FBF735FD00201EE40F98C1B26148BD
:10E12000406880F82C107BE2AFF2044120A8F2F79F
:10E13000CEF8B8BBBE480068017FBD480068C27E0B
:10E14000BB480068837EBA480068407ECDE908324B
:10E150000A910790B6480068017EB5480068C27D04
:10E16000B3480068837DB2480068407DCDE9043241
:10E1700006910390AE480068017DAD480068C27CFE
:10E18000AB480068807CCDE901210090A848006878
:10E19000407C0346A74A0E90DDE93801FBF7F0FC0E
:10E1A000002054E4FFE7AFF26C4120A8F2F78FF8AB
:10E1B000D8BB9DF8600000B30022114618A8F2F702
:10E1C00095F90E900E98000E9949096848740E98BA
:10E1D000010C9748006881740E98010A9448006801
:10E1E000C1740E98C1B292480068017592A20E9B4C
:10E1F000DDE93801FBF7C4FC15E08D480068017DBE
:10E200008B480068C27C8A480068807CCDE9012187
:10E21000009087480068407C034690A20E90DDE99C
:10E220003801FBF7ADFC002011E4FFE7AFF29841A5
:10E2300020A8F2F74CF8A0BB9DF8600000B30022C4
:10E24000114618A8F2F752F90E900E98010E784870
:10E25000006841750E98010C7548006881750E982C
:10E26000010A73480068C1750E98C1B27048006811
:10E27000017684A20E9BDDE93801FBF781FC19E1F0
:10E280006B480068017E6A480068C27D6848006883
:10E29000807DCDE90121009065480068407D0346FE
:10E2A00002E109E1E02C002043726300496E7661CF
:10E2B0006C6964204746534B2043726320283078B2
:10E2C00030302F307831302F307832302F30783373
:10E2D00030290D0A00000000496E76616C696420E7
:10E2E0004746534B2057686974656E696E672028EE
:10E2F000307830302F30783038290D0A0000000097
:10E30000556E6B6E6F776E204746534B207061637E
:10E310006B6574206669656C640D0A00496E7661F0
:10E320006C6964204C6F526120507265616D626C43
:10E33000652028302D323535290D0A00496E766169
:10E340006C6964204C6F526120486561646572207D
:10E3500028307830302F30783830290D0A0000000E
:10E36000496E76616C6964204C6F5261205061790E
:10E370006C6F61642028312D323535290D0A00007B
:10E38000496E76616C6964204C6F52612043726300
:10E390002028307830302F30783230290D0A0000B4
:10E3A000496E76657274495100000000496E7661CD
:10E3B0006C6964204C6F526120496E7665727449B5
:10E3C000512028307830302F30783430290D0A0031
:10E3D000556E6B6E6F776E204C6F5261207061636B
:10E3E0006B6574206669656C640D0A00BC4E01089B
:10E3F000496E76616C696420464C52432053796EB5
:10E4000063576F72644C656E67746820283078308B
:10E41000302F307830322F307830342F307830361B
:10E420002F30783038290D0A00000000444F0108D1
:10E43000302F00209C520108464C52432073796EC5
:10E440006320776F726420312073657420746F20AD
:10E4500030782530386C580D0A000000464C524385
:10E460002053796E6320576F726420313A20253033
:10E4700032582530325825303258253032580D0A5E
:10E4800000000000464C52432073796E6320776F82
:10E49000726420322073657420746F2030782530C8
:10E4A000386C580D0A000000FAA20E90DDE9380120
:10E4B000FBF766FB002014E5AFF2C86120A8F1F776
:10E4C00006FFD8BB9DF8600000B30022114618A8D3
:10E4D000F2F70CF80E900E98010EF848006841769D
:10E4E0000E98010CF548006881760E98010AF348F1
:10E4F0000068C1760E98C1B2F04800680177F0A2BA
:10E500000E9BDDE93801FBF73BFB15E0EB480068AB
:10E51000017FEA480068C27EE8480068807ECDE955
:10E5200001210090E5480068407E0346EDA20E9070
:10E53000DDE93801FBF724FB0020D2E4FFE7AFF26E
:10E54000F06120A8F1F7C3FE90B90F9848B10F9879
:10E55000202806D0EDA2DDE93801FBF711FB0020F1
:10E56000BFE40F98C1B2F248406880F82D1057E020
:10E57000AFF2F86120A8F1F7AAFE90B90F9810B198
:10E580000F98FF2806D9EBA2DDE93801FBF7F8FA6E
:10E590000020A6E40F98C1B2E548406880F82E102C
:10E5A0003EE0AFF2FC2120A8F1F791FEC0B90F9830
:10E5B00078B10F9810280CD00F98202809D00F9808
:10E5C000302806D0E3A2DDE93801FBF7D9FA0020B4
:10E5D00087E40F98C1B2D648406880F82F101FE03A
:10E5E000AFF67C1120A8F1F772FE90B90F9848B1F0
:10E5F0000F98082806D0E2A2DDE93801FBF7C0FA3F
:10E6000000206EE40F98C1B2C948406880F830100D
:10E6100006E0E5A2DDE93801FBF7B2FA002060E48C
:10E6200007E0AFF68462DDE93801FBF7A9FA0020C4
:10E6300057E400BFBE4840681D300E90E148406C72
:10E640000D90DDE90D108847DFA2DDE93801FBF709
:10E6500097FA47E3E3A128A8F1F739FE002870D123
:10E66000E34920A8F1F733FEB8B9E248F1F719FE03
:10E67000E1490968884202D80020DF490860DE4B82
:10E68000DC4ADDE93801FCF71EFF0C900C9810B94C
:10E690000020D94908600C9823E49DF8800010BB45
:10E6A000A348406840780B90FCF74CF80C90A048C9
:10E6B000406890F855209E48406890F854009C4966
:10E6C000496891F853109A4B5B6893F85230CDE942
:10E6D0000031CDE90202C94A0C9BDDE93801FBF7A4
:10E6E0004FFA002016E44FF0FF300E9072A00D900C
:10E6F0008F484068407830B1012823D002283FD0AD
:10E7000003287CD15BE00F98022807D9BCA20F9B9D
:10E71000DDE93801FBF734FA002009E484490F9859
:10E72000496881F852008248406890F852000146DA
:10E730000C907F48F9F750FF0E90AD485C300D907B
:10E7400064E076E00F98072807D9B9A20F9BDDE9AE
:10E750003801FBF715FA002015E40F98C1B2744890
:10E76000406880F853107248406890F853000146A2
:10E770000C906F48F9F7FCFF0E90B9A00D9045E0A2
:10E780000F98032807D9B8A20F9BDDE93801FBF7E2
:10E79000F7F9002010E40F98C1B26548406880F88E
:10E7A00054106348406890F8540001460C9060484B
:10E7B000F9F79AFF0E908E4868300D9026E00F987A
:10E7C000032807D9B4A20F9BDDE93801FBF7D8F97C
:10E7D000002009E40F98C1B25548406880F85510F0
:10E7E0005348406890F8550001460C905048F9F79E
:10E7F00037FF0E907E4870300D9007E0FFE7B2A221
:10E80000DDE93801FBF7BCF9002005E400BF0E98F4
:10E8100040B90F980090B2A20D9BDDE93801FBF7DB
:10E82000AFF905E0B9A20D9BDDE93801FBF7A8F9C6
:10E8300058E2C0A128A8F1F74AFD48BB9DF8800026
:10E8400060B93B48406890F950000346BBA20D9068
:10E85000DDE93801FBF794F9002010E40F9840B28D
:10E860000E9033490E98496881F85000304840684E
:10E8700090F851000D902E48406890F950000C908F
:10E880005048006D0B90DDE90B200D99904763E136
:10E8900069E10000464C52432053796E6320576F64
:10E8A000726420323A2025303258253032582530D3
:10E8B0003258253032580D0A00000000302F002059
:10E8C000464C52432073796E6320776F7264203315
:10E8D0002073657420746F2030782530386C580DA3
:10E8E0000A000000464C52432053796E6320576F54
:10E8F000726420333A202530325825303258253082
:10E900003258253032580D0A00000000496E7661F9
:10E910006C696420464C52432048656164657220EE
:10E9200028307830302F30783230290D0A0000003E
:10E93000E02C0020496E76616C696420464C52439D
:10E94000205061796C6F61642028312D3235352972
:10E950000D0A0000496E76616C696420464C524392
:10E96000204372632028307830302F307831302FB8
:10E97000307832302F30783330290D0A0000000013
:10E98000496E76616C696420464C52432057686931
:10E9900074656E696E672028307830302F3078309B
:10E9A00038290D0A00000000556E6B6E6F776E20DF
:10E9B000464C5243207061636B6574206669656CD8
:10E9C000640D0A00341C01085061636B657420708B
:10E9D0006172616D657465727320757064617465D0
:10E9E000640D0A0062617564726174650000000064
:10E9F000A0CF0008AF4501081C0100209455010874
:10EA0000496E76616C696420424C45206261756490
:10EA10007261746520696E6465783A20256C752092
:10EA20002876616C69643A20302D32290D0A000085
:10EA3000496E76616C6964204C6F52612062617529
:10EA4000647261746520696E6465783A20256C751E
:10EA5000202876616C69643A20302D37290D0A0030
:10EA60004C6F526100000000496E76616C69642051
:10EA70004746534B20626175647261746520696E0C
:10EA80006465783A20256C75202876616C69643A53
:10EA900020302D33290D0A00496E76616C6964209F
:10EAA000464C524320626175647261746520696EE0
:10EAB0006465783A20256C75202876616C69643A23
:10EAC00020302D33290D0A00556E6B6E6F776E2046
:10EAD000726164696F206D6F64650D0A000000004B
:10EAE00042617564726174652075706461746564F7
:10EAF00020666F72202573206D6F6465202D3E2087
:10EB0000696E64657820256C750D0A004661696C34
:10EB1000656420746F20757064617465206261752E
:10EB2000647261746520666F72202573206D6F6456
:10EB3000650D0A00706F7765720000004375727290
:10EB4000656E7420545820706F7765723A20256482
:10EB50002064426D0D0A000064A20E9BDDE93801BD
:10EB6000FBF70EF8BEE068A128A8F1F7B0FB80BB68
:10EB700000200E900F980D909DF8800050BB022051
:10EB80000C906448406890F8510000F01F0111BBE0
:10EB9000401108281FD2DFE800F004070A0D101307
:10EBA000161902200C9017E004200C9014E00620A7
:10EBB0000C9011E008200C900EE00A200C900BE065
:10EBC0000C200C9008E010200C9005E014200C9014
:10EBD00002E05BE009E000BF00BF4FA20C9BDDE953
:10EBE0003801FAF7CDFF002065E40D980A281CD003
:10EBF00008DC02280DD004280ED006280FD00828E3
:10EC00001FD10FE00C2813D0102814D0142818D1CD
:10EC100014E000200E901BE020200E9018E0402011
:10EC20000E9015E060200E9012E080200E900FE014
:10EC3000A0200E900CE0C0200E9009E0E0200E9085
:10EC400006E03CA2DDE93801FAF79AFF002032E441
:10EC500000BF30490E98496881F851002D4840683E
:10EC600090F851000C902B48406890F950000B90A0
:10EC70003548006D0A90DDE90A200C99904733A2CF
:10EC80000D9BDDE93801FAF77BFF2BE036A128A8C0
:10EC9000F1F71DFB20B136A128A8F1F718FBE0B968
:10ECA0009DF8800060B91B484168D1E9120133A288
:10ECB000CDE90001DDE93801FAF762FF00203CE40C
:10ECC0000F980E9013480E99F9F71EFE32A20E9B74
:10ECD000DDE93801FAF754FF04E035A2DDE9380137
:10ECE000FAF74EFF00BF002027E4000054582070C0
:10ECF0006F7765722073657420746F2025642064BB
:10ED0000426D0D0A0000000072616D7074696D65DE
:10ED100000000000E02C002043757272656E7420C4
:10ED200072616D702074696D653A20256C7520756F
:10ED3000730D0A00496E76616C69642072616D70B2
:10ED400074696D650D0A0000341C010852616D7014
:10ED50002074696D652073657420746F20256C754F
:10ED60002075730D0A0000007266667265710000FE
:10ED700072666672657175656E637900437572724D
:10ED8000656E7420524620667265713A20256C6C5F
:10ED90007520487A0D0A000052462066726571207F
:10EDA00073657420746F20256C7520487A0D0A00F5
:10EDB000556E6B6E6F776E20726164696F20636F42
:10EDC0006D6D616E640D0A002DE9FC4104460D462F
:10EDD00016461F4601AA10A12846F1F78DFABDF884
:10EDE0000400FBF7D5FC60B94FF6FE7001230BA2BF
:10EDF000394600903046FAF7C3FE4FF0FF30BDE8C9
:10EE0000FC81BDF804002080238814A239463046D6
:10EE1000FAF7B6FE0020F2E7256878005258494418
:10EE200020736574206661696C65643A20696E764A
:10EE3000616C69642076616C75650D0A56616C6958
:10EE4000642072616E67653A203078253034582D21
:10EE50003078253034580D0A0000000052584944DB
:10EE60002073657420746F3A203078253034580D43
:10EE70000A0000002DE9F04106460F46F2F752F96C
:10EE8000041E0D4618BF0120284320F00040C0F1A9
:10EE90007F6000F1E040C00F0ED0301C18BF012091
:10EEA000384320F00040C0F17F6000F1E040C00F27
:10EEB00004BF0120FAF73AFF20462946BDE8F08159
:10EEC0000020014908707047D4000020002001494B
:10EED00008707047D400002001460A69D1E901306A
:10EEE0009860D1E9010358605068884201D1886870
:10EEF0005060002008611068401E10601068704764
:10EF0000034B0360034B0B608023136070470000CA
:10EF10008C0C0020E80C0020034B0360034B0B60BB
:10EF20004FF4807313607047E80E0020440F0020F8
:10EF300000F1080141604FF0FF31816000F10801EC
:10EF4000C1600161002101607047002101617047CB
:10EF500010B502460B685C1C0CB9106907E002F1A1
:10EF6000080000E04068446824689C42FAD944687C
:10EF70004C604C68A160886041600A611468641C40
:10EF8000146010BD42684A6093688B609368596052
:10EF90009160086103685B1C0360704700BF5020EC
:10EFA00080F31188BFF34F8FBFF36F8F00BF0E4800
:10EFB0000068401C0C49086008460068012812D10E
:10EFC0000A480068C0B208B9012000E0002050B92A
:10EFD00000BF502080F31188BFF34F8FBFF36F8FB6
:10EFE00000BF00BFFEE770478C00002004ED00E08A
:10EFF0000D48006850B900BF502080F31188BFF35E
:10F000004F8FBFF36F8F00BF00BFFEE70648006859
:10F01000401E054908600846006820B9002080F3BA
:10F02000118800BF00BF70478C00002070B50646F5
:10F030003546002E44D0083D2C46224960680968B8
:10F04000084008B1012000E0002050B900BF502066
:10F0500080F31188BFF34F8FBFF36F8F00BF00BFE6
:10F06000FEE7206808B9012000E0002050B900BF89
:10F07000502080F31188BFF34F8FBFF36F8F00BF15
:10F0800000BFFEE70F49606809680840C0B120680A
:10F09000B0B90C49606809688843606000F0E0F925
:10F0A0000949606809680844074908602046FDF777
:10F0B000EFF906480068401C0449086000F0EAFFC8
:10F0C00070BD00008800002078000020840000202F
:10F0D00000204FF0E02108618861064800684FF485
:10F0E0007A71B0FBF1F0401E4FF0E021486107203B
:10F0F000086170471400002070B5F1F74BF8044622
:10F10000102C16D304F1E02090F8F0531548007845
:10F11000854201DB012000E0002050B900BF5020F3
:10F1200080F31188BFF34F8FBFF36F8F00BF00BF15
:10F13000FEE70D48006800F4E0600C490968884269
:10F1400001D8012000E0002050B900BF502080F31A
:10F150001188BFF34F8FBFF36F8F00BF00BFFEE773
:10F1600070BD0000900000200CED00E09400002035
:10F17000024600200BE0084B53F8303033B9064B01
:10F1800043F8301003EBC0035A6002E0401C08282B
:10F19000F1D300BF70470000700600202DE9F04158
:10F1A00005460E4617462C46FFF7F8FE94F9440034
:10F1B000401C10B9002084F8440094F94500401C1C
:10F1C00010B9002084F84500FFF712FFA06B28B9A2
:10F1D0003A46314604F1240000F0C6F82046FDF717
:10F1E000A8FBBDE8F081000070B504460025D4B14D
:10F1F0001248006808B9012000E0002050B900BFA3
:10F20000502080F31188BFF34F8FBFF36F8F00BF83
:10F2100000BFFEE700F024F900212046FCF778FE4D
:10F2200000F038FF05463DB94FF0805004490860B2
:10F23000BFF34F8FBFF36F8F70BD000050000020F1
:10F2400004ED00E070B50546FFF7A8FE15B92748A4
:10F25000006800E028460446201DFFF73DFEA06A36
:10F2600018B104F11800FFF737FE21480068401C70
:10F270001F4908601D480068844209D1211D1D48AE
:10F28000FFF780FE1C480068401C1B49086009E02D
:10F290001A480068401E194908602046FCF784FFA0
:10F2A000FDF798FAFFF7A4FE15480068E8B10F488B
:10F2B0000068844219D11348006808B9012000E0B1
:10F2C000002050B900BF502080F31188BFF34F8F4A
:10F2D000BFF36F8F00BF00BFFEE74FF080500A49B9
:10F2E0000860BFF34F8FBFF36F8F70BD1800002011
:10F2F000440000204C0B00202400002028000020A7
:10F30000340000205000002004ED00E003490968AB
:10F310000160034909684160704700004000002017
:10F320002C00002001200149086070473C000020AB
:10F3300070B504460D4654B900BF502080F31188C3
:10F34000BFF34F8FBFF36F8F00BF00BFFEE70548CD
:10F35000016818312046FFF7FBFD01212846FCF724
:10F36000D7FD70BD1800002070B505460E46144646
:10F3700055B900BF502080F31188BFF34F8FBFF302
:10F380006F8F00BF00BFFEE70648016818312846AE
:10F39000FFF7F8FD0CB14FF0FF3621463046FCF781
:10F3A000B7FD70BD1800002010B586B00020059094
:10F3B000049003AA04A905A8FFF7A2FD0022DDE935
:10F3C00004101346CDE9002102901EA11F48039AA4
:10F3D00000F09CFC1E4908600846006808B1012442
:10F3E00000E00024012C02D100F0D6FE0446012CDE
:10F3F00015D100BF502080F31188BFF34F8FBFF3AA
:10F400006F8F00BF4FF0FF30124908600120124992
:10F41000086000201149086000F07AF810E0601CD4
:10F4200008B1012000E0002050B900BF502080F357
:10F430001188BFF34F8FBFF36F8F00BF00BFFEE790
:10F4400006B010BD49444C450000000019C3000837
:10F450004C00002048000020340000202C00002038
:10F4600002480068401C01490860704750000020B5
:10F470001E48006818B101201D49086034E00020D2
:10F480001B4908601B4801680CE051B900BF5020BF
:10F4900080F31188BFF34F8FBFF36F8F00BF00BFA2
:10F4A000FEE7491E01EB8100134A52F8200008B91B
:10F4B000012000E000200028E7D101EB81020E4B83
:10F4C00003EB820042685268426000F10802436820
:10F4D000934202D14268526842604268D268074B48
:10F4E0001A600448016000BF70470000500000200F
:10F4F0003C00002030000020B00600201800002052
:10F5000010B500BF0020F1F7D9FE0128FAD110BDD7
:10F510001CB53849084600780190FF200A46107053
:10F520000846007800909DF8000000F0F0009DF87B
:10F530000020904201D1012000E0002050B900BF1E
:10F54000502080F31188BFF34F8FBFF36F8F00BF40
:10F5500000BFFEE79DF8000000F05000264A107042
:10F560000720264A106009E024480068401E234A0C
:10F5700010609DF800004006000E00909DF800000D
:10F5800000F080008028EFD01C480068C0F1070020
:10F59000042801D1012000E0002050B900BF502014
:10F5A00080F31188BFF34F8FBFF36F8F00BF00BF91
:10F5B000FEE7124800680002104A106010460088FA
:10F5C00000F4E06010600B4A019810700C4800686D
:10F5D00040F470000A4908600846006840F0704036
:10F5E0000860FFF775FD002006490860F0F79CFDF4
:10F5F00000201CBD00E400E09000002094000020EA
:10F6000020ED00E08C00002010B500BF502080F3FA
:10F610001188BFF34F8FBFF36F8F00BF00F0FAFB6D
:10F6200018B14FF080500449086000BF002080F3FB
:10F63000118800BF10BD000004ED00E02DE9F84383
:10F6400005460E4617460DB1012000E0002050B9D6
:10F6500000BF502080F31188BFF34F8FBFF36F8F2F
:10F6600000BF00BFFEE705FB06F808F15000FDF7FC
:10F670009FF9044664B1A14609F15009002084F8BD
:10F6800046003B464A46314628460094FCF758FE61
:10F690002046BDE8F8832DE9F84380460E4617461C
:10F6A0001D46DDF82090B8F1000F01D0012000E0E8
:10F6B000002050B900BF502080F31188BFF34F8F56
:10F6C000BFF36F8F00BF00BFFEE70DB1012000E068
:10F6D000002050B900BF502080F31188BFF34F8F36
:10F6E000BFF36F8F00BF00BFFEE707B10EB101206F
:10F6F00000E0002050B900BF502080F31188BFF314
:10F700004F8FBFF36F8F00BF00BFFEE707B90EB981
:10F71000012000E0002050B900BF502080F3118884
:10F72000BFF34F8FBFF36F8F00BF00BFFEE75020C6
:10F7300000900098502801D1012000E0002050B92D
:10F7400000BF502080F31188BFF34F8FBFF36F8F3E
:10F7500000BF00BFFEE700BF2C464CB1012084F87B
:10F7600046004B463A46314640460094FCF7E8FDD9
:10F770002046BDE8F883000070B505460E462C46CD
:10F7800054B900BF502080F31188BFF34F8FBFF3EF
:10F790006F8F00BF00BFFEE7FFF700FCD4E90F1238
:10F7A000206801FB0200A0600020A0632068606068
:10F7B000E06B401E226C216800FB0211E160FF201B
:10F7C00084F8440084F845009EB9206908B90120F6
:10F7D00000E00020A8B904F1100000F00FFC80B197
:10F7E0004FF0805009490860BFF34F8FBFF36F8F10
:10F7F00007E004F11000FFF79BFB04F12400FFF782
:10F8000097FBFFF7F5FB012070BD000004ED00E061
:10F810002DE9FF4383B0064688461D464FF0000998
:10F82000344654B900BF502080F31188BFF34F8F86
:10F83000BFF36F8F00BF00BFFEE7B8F1000F01D12B
:10F84000206C08B9012000E0002050B900BF502012
:10F8500080F31188BFF34F8FBFF36F8F00BF00BFDE
:10F86000FEE7022D02D1E06B012801D1012000E06A
:10F87000002050B900BF502080F31188BFF34F8F94
:10F88000BFF36F8F00BF00BFFEE700F0A3FA08B917
:10F89000059808B9012000E0002050B900BF5020B1
:10F8A00080F31188BFF34F8FBFF36F8F00BF00BF8E
:10F8B000FEE700BFFFF772FBA06BE16B884201D34C
:10F8C000022D28D12A4641462046FCF72EFC074649
:10F8D000606A08B9012000E0002068B904F1240042
:10F8E00000F08CFB88B14FF0805032490860BFF3C4
:10F8F0004F8FBFF36F8F08E03FB14FF080502D491D
:10F900000860BFF34F8FBFF36F8FFFF771FB0120CC
:10F9100007B0BDE8F083059818B9FFF769FB002030
:10F92000F6E7B9F1000F04D101A8FFF7EFFC4FF0A3
:10F930000109FFF75DFBFFF793FDFFF72FFB94F93C
:10F940004400401C10B9002084F8440094F945009C
:10F95000401C10B9002084F84500FFF749FB05A9B9
:10F9600001A800F05BF9F0B92046FCF7FEFDA0B15C
:10F9700004F110000599FFF7DBFC2046FCF7D9FFE6
:10F9800000F088FB002895D14FF0805009490860AD
:10F99000BFF34F8FBFF36F8F8CE72046FCF7C9FF93
:10F9A00000F078FB86E72046FCF7C3FF00F072FB0F
:10F9B0000020ADE704ED00E02DE9F84F07468A4648
:10F9C00090461E463C4654B900BF502080F3118833
:10F9D000BFF34F8FBFF36F8F00BF00BFFEE7BAF1D9
:10F9E000000F01D1206C08B9012000E0002050B9BF
:10F9F00000BF502080F31188BFF34F8FBFF36F8F8C
:10FA000000BF00BFFEE7022E02D1E06B012801D14A
:10FA1000012000E0002050B900BF502080F3118881
:10FA2000BFF34F8FBFF36F8F00BF00BFFEE7FFF73D
:10FA300063FB00BF5021EFF3118081F31188BFF306
:10FA40004F8FBFF36F8F00BF0546A06BE16B8842FD
:10FA500001D3022E25D194F945B0A06B0090324617
:10FA600051462046FCF761FB0BF1010088B9606A42
:10FA700008B9012000E0002050B904F1240000F092
:10FA8000BDFA28B1B8F1000F02D00120C8F800007B
:10FA900004E00BF1010040B284F845004FF0010989
:10FAA00001E04FF0000900BF85F3118800BF484610
:10FAB000BDE8F88F2DE9F74183B005460E464FF0BB
:10FAC00000082C4654B900BF502080F31188BFF3C2
:10FAD0004F8FBFF36F8F00BF00BFFEE70EB9206CE2
:10FAE00008B9012000E0002050B900BF502080F389
:10FAF0001188BFF34F8FBFF36F8F00BF00BFFEE7CA
:10FB000000F068F908B9059808B9012000E0002064
:10FB100050B900BF502080F31188BFF34F8FBFF35F
:10FB20006F8F00BF00BFFEE700BFFFF737FAA76B7C
:10FB3000F7B131462046FCF7E3FA781EA06320694E
:10FB400008B9012000E0002060B904F1100000F0C5
:10FB500055FA38B14FF080502F490860BFF34F8FEE
:10FB6000BFF36F8FFFF744FA012006B0BDE8F081C4
:10FB7000059818B9FFF73CFA0020F6E7B8F1000F36
:10FB800004D101A8FFF7C2FB4FF00108FFF730FADC
:10FB9000FFF766FCFFF702FA94F94400401C10B925
:10FBA000002084F8440094F94500401C10B900205E
:10FBB00084F84500FFF71CFA05A901A800F02EF80B
:10FBC000F0B92046FCF7C4FCA0B104F1240005996B
:10FBD000FFF7AEFB2046FCF7ACFE00F05BFA002816
:10FBE000A3D14FF080500C490860BFF34F8FBFF393
:10FBF0006F8F9AE72046FCF79CFE00F04BFA94E7E3
:10FC00002046FCF796FE00F045FA2046FCF7A0FCE3
:10FC100000288AD00020A8E704ED00E070B5054672
:10FC20000C4655B900BF502080F31188BFF34F8FA9
:10FC3000BFF36F8F00BF00BFFEE754B900BF502075
:10FC400080F31188BFF34F8FBFF36F8F00BF00BFEA
:10FC5000FEE7FFF7A3F9124802686868131A2068E4
:10FC6000401C08B9002617E00E4928680968884238
:10FC700004D06868904201D801260DE020689842BF
:10FC800007D92068C01A20602846FFF73FFB0026EE
:10FC900002E0002020600126FFF7AAF9304670BD7F
:10FCA0002C000020400000202DE9FF4F85B0804649
:10FCB00089461746DDE912ABB800FCF779FE064627
:10FCC00056B15C20FCF774FE04460CB1266304E0D8
:10FCD0003046FFF7ABF900E000248CB1002084F837
:10FCE0005900CDE900ABCDE902403A4649464046CD
:10FCF000089BFCF73AFB2046FCF748F9012501E098
:10FD00004FF0FF35284609B0BDE8F08F2DE9F04FE0
:10FD100085B00746884691469A46DDE90EB6109CA6
:10FD20000EB1012000E0002050B900BF502080F348
:10FD30001188BFF34F8FBFF36F8F00BF00BFFEE787
:10FD40000CB1012000E0002050B900BF502080F32A
:10FD50001188BFF34F8FBFF36F8F00BF00BFFEE767
:10FD60005C20039003985C2801D1012000E0002072
:10FD700050B900BF502080F31188BFF34F8FBFF3FD
:10FD80006F8F00BF00BFFEE700BFB4B1AEB1254624
:10FD90002C462E63022085F85900002004A9534602
:10FDA0004A46CDE900B1CDE9025041463846FCF75C
:10FDB000DCFA2846FCF7EAF801E0002004900498F9
:10FDC00005B0BDE8F08F00000149086870470000E9
:10FDD000180000200549096809B9012005E0044917
:10FDE000096809B9022000E00020704734000020B3
:10FDF0005000002001490868704700002C000020D6
:10FE000070B5FFF779F9002501480468204670BDF8
:10FE10002C0000202DE9F0414FF000084348006815
:10FE200000287BD142480068451C4148056015BB4D
:10FE300040480068006808B9012000E0002050B97F
:10FE400000BF502080F31188BFF34F8FBFF36F8F37
:10FE500000BF00BFFEE737480768374800683549EC
:10FE600008603548076035480068401C3349086021
:10FE7000FCF7B0FC00BF3248006885423BD300BFAE
:10FE80002C480068006808B9012000E0002020B17B
:10FE90004FF0FF302A4908602CE026480068C0680F
:10FEA000C4686668B54202D22548066022E0201D7B
:10FEB000FFF712F8A06A18B104F11800FFF70CF868
:10FEC0002049E06A0968884202D91E49E06A086050
:10FED000E16A01EB81011C4A02EB8100211DFFF761
:10FEE00051F81A49E06A0968C96A8842C8D34FF0D4
:10FEF0000108C5E700BF15480068C06A00EB800034
:10FF0000114951F82000012801D94FF0010810488B
:10FF1000006808B14FF0010805E0FFE70D480068F0
:10FF2000401C0C4908604046BDE8F08150000020AC
:10FF30002C0000201C000020200000204000002099
:10FF40004800002030000020B006002018000020EB
:10FF50003C0000203800002070B505462C460026E5
:10FF6000002D43D022480068844201D1012000E0E6
:10FF7000002050B900BF502080F31188BFF34F8F8D
:10FF8000BFF36F8F00BF00BFFEE7206D50B900BF09
:10FF9000502080F31188BFF34F8FBFF36F8F00BFE6
:10FFA00000BFFEE7206D401E2065E16CE06A8842DC
:10FFB0001CD0206DD0B9201DFEF78EFFE06CE062F2
:10FFC000E06AC0F13800A0610A49E06A0968884225
:10FFD00002D90849E06A0860E16A01EB8101064A3A
:10FFE00002EB8100211DFEF7CDFF0126304670BDDA
:10FFF0001800002030000020B006002070B5064632
:020000040801F1
:10000000F068C46854B900BF502080F31188BFF372
:100010004F8FBFF36F8F00BF00BFFEE704F11800E2
:10002000FEF75AFF15480068A0B9201DFEF754FFDF
:100030001349E06A0968884202D91149E06A0860F8
:10004000E16A01EB81010F4A02EB8100211DFEF7FD
:1000500099FF04E004F118010B48FEF793FF0B49E8
:10006000E06A0968C96A884204D901250120084963
:10007000086000E00025284670BD00005000002008
:1000800030000020B0060020380B002018000020AF
:100090003C00002070B5002400263648006850B9A6
:1000A00000BF502080F31188BFF34F8FBFF36F8FD5
:1000B00000BF00BFFEE7FEF771FF2E480068401E3C
:1000C0002C4908600846006800284ED12A4800687C
:1000D00000284AD023E02948C068C46804F1180009
:1000E000FEF7FAFE201DFEF7F7FE2549E06A0968D3
:1000F000884202D92249E06A0860E16A01EB810185
:10010000204A02EB8100211DFEF73CFF1E49E06AF8
:100110000968C96A884202D301201C49086017484F
:10012000006808B9012000E000200028D3D00CB1FD
:10013000FCF750FB1648056865B100BFFFF76AFE83
:1001400010B10120114908606D1E002DF6D100206C
:100150000F4908600D48006838B1012630070D4985
:100160000860BFF34F8FBFF36F8FFEF741FF30463C
:1001700070BD00005000002028000020380B002037
:1001800030000020B0060020180000203C000020B5
:100190003800002004ED00E010B586B00024FBF725
:1001A00051FF16480068D0B100200590049003AAC2
:1001B00004A905A8FEF7B0FE0222DDE90410002321
:1001C000CDE9002102900EA10F48039AFFF79EFD92
:1001D0000E4908600846006800B1012400BF54B908
:1001E00000BF502080F31188BFF34F8FBFF36F8F94
:1001F00000BF00BFFEE7204606B010BD5C00002037
:10020000546D72205376630019C900086000002005
:100210002DE9FF4704460D4616461F46DDF830809F
:100220004FF0000954B900BF502080F31188BFF38C
:100230004F8FBFF36F8F00BF00BFFEE71448006809
:1002400010B3009501960294062D15DAFFF7C2FD52
:10025000022808D10023424669460D480068FFF78E
:10026000D7FA814610E000231A466946084800681C
:10027000FFF7CEFA814607E000233A466946044874
:100280000068FFF799FB8146484604B0BDE8F08757
:100290005C000020D04D01080000000000000000BC
:1002A0000000000000000000000200001800000034
:1002B0000000000000000000020304050607080912
:1002C0000A0B0C0D0E0F10100102000000000000C0
:1002D00000000102030406070809000000000102F3
:1002E00003040000AC0200200C000000000000002D
:1002F00000000000000000000000000000000008F6
:1003000008080808080800001818000000486C24B5
:1003100012000000000000000000000000000024A7
:1003200024247F1212127F12121200000000081CF7
:100330002A2A0A0C1828282A2A1C08080000002249
:10034000251515152A585454542200000000000C9D
:100350001212120A76252911916E00000006060479
:10036000030000000000000000000000004020101A
:1003700010080808080808101020400000020408AF
:1003800008101010101010080804020000000000EF
:1003900008086B1C1C6B080800000000000000002F
:1003A000080808087F08080808000000000000008E
:1003B000000000000000000006060403000000002A
:1003C00000000000FE00000000000000000000002F
:1003D0000000000000000000060600000000804051
:1003E0004020201010080804040202000000001839
:1003F00024424242424242422418000000000008C7
:100400000E08080808080808083E00000000003C24
:100410004242422020100804427E00000000003CBE
:100420004242201820404042221C000000000020D0
:100430003028242422227E20207800000000007E24
:100440000202021A26404042221C0000000000382E
:100450002402021A26424242241800000000007EB4
:100460002222101008080808080800000000003CBC
:100470004242422418244242423C0000000000183C
:100480002442424264584040241C00000000000006
:1004900000001818000000001818000000000000FC
:1004A00000000008000000000008080400000040F0
:1004B0002010080402040810204000000000000082
:1004C00000007F0000007F0000000000000000022C
:1004D0000408102040201008040200000000003C26
:1004E0004242464020101000181800000000001C76
:1004F000225A555555552D42221C00000000000877
:1005000008181414243C224242E700000000001F97
:100510002222221E22424242221F00000000007CB2
:100520004242010101010142221C00000000001FA3
:100530002242424242424242221F00000000003F4B
:100540004212121E12120242423F00000000003FFF
:100550004212121E12120202020700000000003CAA
:100560002222010101712122221C0000000000E76B
:10057000424242427E42424242E700000000003EC8
:100580000808080808080808083E00000000007C69
:1005900010101010101010101010110F0000007724
:1005A00022120A0E0A12122222770000000000070F
:1005B0000202020202020202427F000000000077F3
:1005C000363636362A2A2A2A2A6B0000000000E333
:1005D00046464A4A52525262624700000000001CDE
:1005E0002241414141414141221C00000000003FA5
:1005F000424242423E020202020700000000001C8A
:100600002241414141414D53321C60000000003FF6
:100610004242423E1212222242C700000000007CE9
:100620004242020418204042423E00000000007F87
:100630004908080808080808081C0000000000E72E
:100640004242424242424242423C0000000000E735
:100650004242222424141418080800000000006BF1
:10066000494949495555362222220000000000E739
:10067000422424181818242442E7000000000077C0
:100680002222141408080808081C00000000007E3C
:100690002120101008040442423F0000007808089E
:1006A000080808080808080808087800000002027E
:1006B000040408080810102020204040001E1010DC
:1006C000101010101010101010101E0000384400F0
:1006D000000000000000000000000000000000001A
:1006E0000000000000000000000000FF00060800FD
:1006F00000000000000000000000000000000000FA
:100700000000003C4278444242FC0000000000032C
:100710000202021A26424242261A0000000000008D
:10072000000000384402020244380000000000606B
:10073000404040784442424264D80000000000003B
:100740000000003C427E0202423C0000000000F03B
:100750008808087E08080808083E0000000000001D
:100760000000007C22221C023C42423C00000003AC
:100770000202023A4642424242E700000000000CF8
:100780000C00000E08080808083E000000000030B9
:1007900030000038202020202020221E00000003EE
:1007A00002020272120A1612227700000000000EE6
:1007B0000808080808080808083E000000000000B3
:1007C0000000007F9292929292B700000000000019
:1007D0000000003B4642424242E7000000000000A9
:1007E0000000003C42424242423C00000000000047
:1007F0000000001B26424242221E020700000000A9
:100800000000007844424242447840E0000000008A
:10081000000000774C040404041F000000000000E6
:100820000000007C42023C40423E0000000000000C
:100830000008083E08080808083000000000000012
:10084000000000634242424262DC000000000000FF
:10085000000000E742242414080800000000000003
:10086000000000EB4949555522220000000000001D
:100870000000007624181818246E00000000000004
:10088000000000E7422424141808080700000000B4
:100890000000007E22100808447E000000C02020D6
:1008A00020202010202020202020C0001010101018
:1008B0001010101010101010101010100006080862
:1008C0000808081008080808080806000C32C200CA
:1008D0000000000000000000000000000000000018
:1008E0000000000000000000000000000000000008
:1008F00000000000000000000000000000000000F8
:1009000000000000000000000000000000000000E7
:100910000000000060006000600060006000600097
:1009200060004000200020002000000000000000C7
:100930006000600060000000000000000000000097
:100940006006600630039801880044000000000043
:100950000000000000000000000000000000000097
:100960000000000000000000000000000000000087
:10097000000000001002100210021002FE07FE0725
:1009800008020801080108010801FE07FE0704012A
:100990000401040104010000000000000000000048
:1009A000000040004000F00158034C03CC034C0011
:1009B00058007000E000C001C00140034C035C031C
:1009C0004C034801F000400040000000000000001F
:1009D000000000000E010A019100910091005100F9
:1009E00051003A00AE03A0025004500448044804E9
:1009F000480484028403000000000000000000009E
:100A00000000000038006C006C006C006C006C0092
:100A10002C0098071C011A01330133016301E30024
:100A2000C308C6093C0700000000000000000000E9
:100A30000C001C0010001000080004000000000062
:100A400000000000000000000000000000000000A6
:100A50000000000000000000000000000000000096
:100A600000040002000180008000400040002000DF
:100A70002000200020002000200020004000400036
:100A8000800080000001000200040000000000005F
:100A900002000400080010001000200020004000A8
:100AA0004000400040004000400040002000200086
:100AB0001000100008000400020000000000000008
:100AC00000000000000000004000C0004000460C94
:100AD0004E0FD001F0015E0F460C40004000400078
:100AE0000000000000000000000000000000000006
:100AF0000000000000000000000040004000400036
:100B000040004000FE0F4000400040004000400018
:100B100000000000000000000000000000000000D5
:100B200000000000000000000000000000000000C5
:100B300000000000000000000000000000000000B5
:100B40000C001C0010001000080004000000000051
:100B50000000000000000000000000000000000095
:100B600000000000FE070000000000000000000080
:100B70000000000000000000000000000000000075
:100B80000000000000000000000000000000000065
:100B90000000000000000000000000000000000055
:100BA0001C001C001C0000000000000000000000F1
:100BB0000004000600020003000100018000800024
:100BC00040004000600020002000100010000800DD
:100BD00008000C00040006000200000000000000F5
:100BE000000000000000F00098010C030C03060652
:100BF00006060606060606060606060606060C0392
:100C00000C039801F000000000000000000000004C
:100C100000000000000040007C00600060006000F8
:100C200060006000600060006000600060006000C4
:100C300060006000FC0300000000000000000000F5
:100C4000000000000000F800840102030603060310
:100C5000000300018001C0006000200010000802B5
:100C600004020602FE030000000000000000000075
:100C70000000000000007800C600860186018001A7
:100C80008001C00070008001000100030003060322
:100C900006038601F80000000000000000000000CC
:100CA00000000000000080018001C001A001A0013F
:100CB00090018801880184018201FE0F800180017A
:100CC00080018001E007000000000000000000003B
:100CD000000000000000FC03040004000400040005
:100CE0000400F4008C010403000300030603060360
:100CF00082018401F80000000000000000000000F4
:100D0000000000000000E00118030C030C000400C8
:100D10000600E60116030E0606060606060604068B
:100D20000C021803F00000000000000000000000AA
:100D3000000000000000F8070C0604020401000196
:100D40000001800080004000400040006000600022
:100D50006000600060000000000000000000000073
:100D6000000000000000F8010C0306060606060657
:100D70000C021C03F000C8010C030606060606065A
:100D800006060C03F0010000000000000000000057
:100D9000000000000000F0000C010C030602060633
:100DA0000606060606078C06780600060003000302
:100DB0000C018C0178000000000000000000000021
:100DC0000000000000000000000000000000000023
:100DD000E000E000E0000000000000000000000073
:100DE000E000E000E0000000000000000000000063
:100DF00000000000000000000000000000000000F3
:100E00006000600000000000000000000000000022
:100E10000000600060004000200020000000000092
:100E200000000000000400020001800040002000DB
:100E3000100008000400080010002000400080009E
:100E4000000100020004000000000000000000009B
:100E50000000000000000000000000000000000092
:100E6000FE07000000000000FE0700000000000078
:100E70000000000000000000000000000000000072
:100E80000000000004000800100020004000800066
:100E90000001000200040002000180004000200068
:100EA0001000080004000000000000000000000026
:100EB000000000000000E0031806040C040C0C0CF9
:100EC0000C0C0007800140004000400000000000C2
:100ED000E000E000E0000000000000000000000072
:100EE00000000000E00018030C02CC056405660554
:100EF000A605B604B604B604B604B602E4010C04B2
:100F00000C021803F00000000000000000000000C8
:100F1000000000000000600060005000D000900061
:100F20009000880088010801F8010403040304020A
:100F3000020202060F0F0000000000000000000087
:100F4000000000000000FE008C030C030C030C03E7
:100F50000C038C01FC000C030C020C060C060C06A6
:100F60000C060C03FE010000000000000000000061
:100F7000000000000000E00318030C060C04040449
:100F800006000600060006000600060006040C0423
:100F90000C021803F0000000000000000000000038
:100FA0000000000000007F008C010C030C030C0605
:100FB0000C060C060C060C060C060C060C060C03A4
:100FC0000C038C017F000000000000000000000006
:100FD000000000000000FF030603060406040600EC
:100FE00086008600FE008600860086000600060455
:100FF00006040602FF0300000000000000000000DD
:10100000000000000000FF030603060406040600BB
:1010100086008600FE008600860086000600060028
:10102000060006001F000000000000000000000095
:10103000000000000000F00018010C020C02040285
:101040000600060006000600C60F060306030C0392
:101050000C031803F0000000000000000000000076
:101060000000000000000F0F060606060606060632
:1010700006060606FE070606060606060606060617
:10108000060606060F0F000000000000000000002A
:10109000000000000000FC036000600060006000D1
:1010A0006000600060006000600060006000600040
:1010B00060006000FC030000000000000000000071
:1010C000000000000000F807C000C000C000C00021
:1010D000C000C000C000C000C000C000C000C00010
:1010E000C000C000C000C60066003C000000000058
:1010F000000000000000CF038601C6004600260065
:10110000160036002E006E004600C60086008601DE
:10111000060106038F070000000000000000000029
:101120000000000000001F00060006000600060088
:10113000060006000600060006000600060006047B
:1011400006040602FF03000000000000000000008B
:101150000000000000000707860386038E038E034D
:101160004E034E034A035A035A033A03320332032F
:101170003203120387070000000000000000000097
:101180000000000000008E0F0C021C021C02340242
:101190003402640264024402C402840284038403AD
:1011A000040304031F020000000000000000000010
:1011B000000000000000F00098010C030C0206067D
:1011C00006060606060606060606060606060C02BD
:1011D0000C039801F0000000000000000000000077
:1011E000000000000000FF000603060606060606D3
:1011F000060606068603FE00060006000600060038
:10120000060006001F0000000000000000000000B3
:10121000000000000000F00098010C030C0206061C
:1012200006060606060606060606060676064C02AC
:10123000CC039801F00080070003000000000000CC
:10124000000000000000FF01060306060606060671
:1012500006060603FE004600C60086008601060359
:10126000060306060F0E000000000000000000004C
:10127000000000000000F8020C030602060206004F
:101280000E003C00F800E00380030007020602069F
:1012900006060C03F0010000000000000000000042
:1012A000000000000000FE076204610861086000A1
:1012B000600060006000600060006000600060002E
:1012C00060006000F8010000000000000000000065
:1012D0000000000000001E070C020C020C020C02B1
:1012E0000C020C020C020C020C020C020C020C028E
:1012F0000C021801F00000000000000000000000D7
:101300000000000000000F070602040104010C01A8
:101310000C01880088009800980050005000700070
:10132000300020002000000000000000000000004D
:10133000000000000000F70E620442044604460468
:1013400064026402E402E4029C029C019801980198
:1013500088018800880000000000000000000000F4
:101360000000000000009E070C0108011801900019
:10137000B0006000200060006000D0009000880194
:10138000080104038E0700000000000000000000B8
:101390000000000000000F0F060404020C02080108
:1013A0001801B800B00070006000600060006000CC
:1013B00060006000F8010000000000000000000074
:1013C000000000000000FC070C020603020180017F
:1013D0008000400040002000200010001800080499
:1013E0000C040402FE0300000000000000000000E6
:1013F000E00320002000200020002000200020002A
:1014000020002000200020002000200020002000DC
:101410002000200020002000E00300000000000069
:101420000000000004000400080008001000100084
:1014300010002000200040004000C000800080001C
:101440000001000100020002000200040000000090
:101450007C00400040004000400040004000400050
:10146000400040004000400040004000400040007C
:1014700040004000400040007C0000000000600090
:1014800090000801000000000000000000000000C3
:10149000000000000000000000000000000000004C
:1014A000000000000000000000000000000000003C
:1014B000000000000000000000000000000000002C
:1014C000000000000000000000000000000000001C
:1014D00000000000000000000000FF0F00000000FE
:1014E0001800600000000000000000000000000084
:1014F00000000000000000000000000000000000EC
:1015000000000000000000000000000000000000DB
:1015100000000000000000000000000000000000CB
:10152000F0010C030C030003E0031C030E0306038D
:1015300006038E0B7C0E000000000000000000007F
:101540000000000008000E000C000C000C000C0055
:10155000CC013C031C060C060C060C060C060C0603
:101560000C021C03E4010000000000000000000069
:10157000000000000000000000000000000000006B
:10158000F0008C018C0186010600060006000602B0
:101590000C020C01F0000000000000000000000040
:1015A000000000000002C00300030003000300036A
:1015B00078038C030C0306030603060306030603E5
:1015C00004038C0778010000000000000000000008
:1015D000000000000000000000000000000000000B
:1015E000E001180308020C060C06FC070C000C00B6
:1015F00018041802E00100000000000000000000D4
:10160000000000000000C00360063006300030001B
:10161000FE0130003000300030003000300030007B
:1016200030003000FC01000000000000000000005D
:1016300000000000000000000000000000000000AA
:10164000F007D8068C018C018C019801F8000C0081
:10165000FC00CC03060306038E03F8000000000024
:101660000000000008000E000C000C000C000C0034
:10167000EC011C030C030C030C030C030C030C0304
:101680000C030C039E070000000000000000000097
:10169000000000000000600060000000000040004A
:1016A0007C0060006000600060006000600060001E
:1016B00060006000FC03000000000000000000006B
:1016C000000000000000C001C00100000000000197
:1016D000F001800180018001800180018001800192
:1016E0008001800180018001CC007C0000000000AE
:1016F0000000000008000E000C000C000C000C00A4
:101700008C038C008C004C006C005C008C008C0105
:101710000C010C039E070000000000000000000008
:101720000000000040007C0060006000600060007D
:1017300060006000600060006000600060006000A9
:1017400060006000FC0300000000000000000000DA
:101750000000000000000000000000000000000089
:101760003707EE06660666066606660666066606BF
:1017700066066606FF0F0000000000000000000083
:101780000000000000000000000000000000000059
:10179000EE011C030C030C030C030C030C030C03E1
:1017A0000C030C039E070000000000000000000076
:1017B0000000000000000000000000000000000029
:1017C000F00098010C030606060606060606060645
:1017D0000C030C03F00000000000000000000000FB
:1017E00000000000000000000000000000000000F9
:1017F000EE011C030C060C060C060C060C060C066F
:101800000C031C03EC010C000C003E000000000067
:1018100000000000000000000000000000000000C8
:1018200078028C030C030603060306030603060373
:1018300004038C03780300030003C00700000000CA
:101840000000000000000000000000000000000098
:101850009F035806380618001800180018001800D2
:1018600018001800FF000000000000000000000049
:101870000000000000000000000000000000000068
:10188000F0031C030C020C023800F000C003040338
:1018900004038C03FC0100000000000000000000B5
:1018A0000000000000000000200020003000300098
:1018B000FE013000300030003000300030003000D9
:1018C00030023002E00100000000000000000000D3
:1018D00000000000000000000000000000000802FE
:1018E0008E030C030C030C030C030C030C030C03FE
:1018F0000C039C07780100000000000000000000BD
:1019000000000000000000000000000000000000D7
:101910001E070C020801080118019000B000B00079
:1019200060006000200000000000000000000000D7
:1019300000000000000000000000000000000000A7
:10194000F70E6204460464026402EC029C019801F2
:10195000980198010800000000000000000000004D
:101960000000000000000000000000000000000077
:10197000BC0718011001B00060006000E00090009A
:10198000080108039E07000000000000000000009E
:101990000000000000000000000000000000000047
:1019A0009E0708010801080190009000B000600047
:1019B000600060002000200024001C0000000000E7
:1019C0000000000000000000000000000000000017
:1019D000FC018401C40044006000200030001802B3
:1019E00008020C03FC0100000000000000000000E1
:1019F0000003800080008000800080008000800064
:101A000080004000200040008000800080008000B6
:101A10008000800080008000000300004000400043
:101A200040004000400040004000400040004000B6
:101A300040004000400040004000400040004000A6
:101A40004000400040004000400040000000000016
:101A50000C0010001000100010001000100010000A
:101A600010002000400020001000100010001000A6
:101A700010001000100010000C00000000001C00FE
:101A80002204C204800300000000000000000000E7
:101A90000000000000000000000000000000000046
:101AA00000000000000000000000000001F800003D
:101AB000FFC007FC0001FFE00FFF0007FFF01FFF62
:101AC000800FFFF03FFFC01FFFF83FFFE07FFFF8F0
:101AD0003FFFF0FFFFF83FFFFBFFFFF83FFFFFFF77
:101AE000FFF83FFFFFFFFFF83FFFFFFF9FF83FFFBB
:101AF000FFFF0FF83FF3FFFC0FF83FF1FFF80FF87F
:101B00003FF0FFE00FF83FF07F800FF83FF01E003E
:101B10000FF83FF008000FF83FF000000FF83FF01B
:101B200000000FF83FF0000E0FF83FF0001E0FF816
:101B30003FE0007E0FF83FE000FE0FF83FE001FEBF
:101B40000FF83FE003FE0FF83FE007FE0FF83FE01D
:101B500007FE0FF83FE003FE0FF83FE001FE0FF82D
:101B60003FE000FE0FF83FE0007E0FF800000000AD
:101B700007FFFF800FFFFFE01FFFFFF01FFFFFF8D1
:101B80003FFFFFFC00001FFC00000FFC00000FF8EF
:101B900000001FF800003FF01FFFFFE03FFFFFC005
:101BA0003FFFFF807FFFFF007FFFFE007FF1FE0011
:101BB000FFE0FC00FFE07C00FFC07E00FFC03E00B5
:101BC000FFC03F00FF801F00FF800F80FF800F805D
:101BD000FF0007C00000000000000000CE01208DC3
:101BE00001204C0120000000C03407A03404B00ADA
:101BF00003801806801801601801500A04500A0179
